:100000002029FE1F61950000BD8F00005D95000056
:100010005D9500005D9500005D950000000000000A
:100020000000000000000000000000005D950000DE
:100030005D950000000000005D9500005D950000EA
:10004000017E0000D57E0000357F0000194C0000C5
:100050009D420000913B0000393700006D3A0000DE
:1000600005390000852300006122000019230000EB
:1000700099210000F116000049170000E515000065
:10008000852300006122000019230000992100004F
:10009000852300006122000019230000992100003F
:1000A000E9260000F12400007D240000ED25000079
:1000B000FFFFFFFFFFFFFFFFFFFFFFFFFFFFFFFF50
:1000C000FFFFFFFFFFFFFFFFFFFFFFFFFFFFFFFF40
:1000D000FFFFFFFFFFFFFFFFFFFFFFFFFFFFFFFF30
:1000E000FFFFFFFFFFFFFFFFFFFFFFFFFFFFFFFF20
:10040000FFFFFFFFFFFDFFFFFFFFFFFFFFFFFFFFFE
:10041000FFFFFFFFFFFFFFFFFFFFFFFFFFFFFFFFEC
:10042000FFFFFFFFFFFFFFFFFFFFFFFFFFFFFFFFDC
:10043000FFFFFFFFFFFFFFFFFFFFFFFFFFFFFFFFCC
:10044000FFFFFFFFFFFFFFFFFFFFFFFFFFFFFFFFBC
:10045000FFFFFFFFFFFFFFFFFFFFFFFFFFFFFFFFAC
:10046000FFFFFFFFFFFFFFFFFFFFFFFFFFFFFFFF9C
:10047000FFFFFFFFFFFFFFFFFFFFFFFFFFFFFFFF8C
:10048000FFFFFFFFFFFFFFFFFFFFFFFFFFFFFFFF7C
:10049000FFFFFFFFFFFFFFFFFFFFFFFFFFFFFFFF6C
:1004A000FFFFFFFFFFFFFFFFFFFFFFFFFFFFFFFF5C
:1004B000FFFFFFFFFFFFFFFFFFFFFFFFFFFFFFFF4C
:1004C000FFFFFFFFFFFFFFFFFFFFFFFFFFFFFFFF3C
:1004D000FFFFFFFFFFFFFFFFFFFFFFFFFFFFFFFF2C
:1004E000FFFFFFFFFFFFFFFFFFFFFFFFFFFFFFFF1C
:1004F000FFFFFFFFFFFFFFFFFFFFFFFFFFFFFFFF0C
:100500000C06FE1F8A003000F005FE1F8D0030181B
:10051000CC05FE1F8E003020E805FE1FB6002B30F4
:100520000806FE1F01000600C405FE1F7008150026
:10053000B805FE1F6D0815089005FE1F6F08151001
:100540009405FE1F6E081518EC05FE1F77011408B0
:10055000F805FE1F74011410D005FE1F760114204B
:10056000DC05FE1F75011428D405FE1F8009141038
:100570000406FE1F82091420F405FE1F81091428B9
:10058000FC05FE1F9B1914080006FE1F9819141085
:10059000E005FE1F9A191420B405FE1F99191428AE
:1005A000D805FE1FA7211408E405FE1FA42114107E
:1005B000C005FE1FA6211420C805FE1FA521142872
:1005C0009805FE1FBF011600BC05FE1FBC011610DA
:1005D0001006FE1FC00116186405FE1FBD0116207F
:1005E00020000000200001002F0000002F0001006B
:1005F0000C0001001100000030000000300001007C
:100600002400000024000100240002002400030054
:10061000240004002400050013000000170000005F
:10062000230000002100000021000100070000005D
:100630000700010007000200070003000700040094
:100640000700050007000600070007001200000071
:1006500044000000080000000B0000004100000002
:1006600040000000400001000400000043000000C2
:100670002B0000002B000A002B000B002B000C00AD
:100680002B000D002B0001002B0002002B000300AB
:100690002B0004002B0005002B0006002B00070098
:1006A0002B0008002B0009000600000006000A00CD
:1006B00006000B0006000C0006000D0006000E00F0
:1006C00006000F00060001000600020006000300FD
:1006D00006000400060005000600060006000700EC
:1006E00006000800060009001500000015000100C2
:1006F00015000200310000002A0000004500000043
:1007000010000000030100000300000003000100CE
:100710000F0000000D0000002D000000420000004E
:100720002C0000002C0001002C0002002C00030013
:100730003200000028000000180000001400000033
:10074000140001001400020014000300140004004F
:10075000140005001400060014000700140008002F
:1007600014000900340000003400010016000000ED
:1007700016000100350000003600000036000100C0
:1007800022000000330000003301000029000000B7
:1007900010B5054C237833B9044B13B10448AFF3BB
:1007A00000800123237010BDDC04FE1F0000000048
:1007B00090FA0000084B10B51BB108480849AFF388
:1007C00000800848036803B910BD074B002BFBD01D
:1007D000BDE81040184700BF0000000090FA00007C
:1007E000E004FE1F3404FE1F0000000040B101239E
:1007F0000921052201704370C37082700020704788
:10080000012070472DE9F04F89B03C4C9DF84CB069
:10081000069007910492059302468BF00103A0FB1A
:100820000401374D129E0393CDE90001A0464FEA23
:10083000122A4FF0000903E0324B06359D4256D094
:100840002A79EB781343039A9342F5D1079B2F88BB
:1008500003FB07F7069BB3FBF7F404F1FF3BBBF187
:10086000FF0FE9D85B4607FB04F4AB464D46B9469B
:100870001F461DE0B4FBFAF27F2A02FB03F33AD9CC
:10088000002BB8BFFF331B12A3F5C333A03B002BD3
:10089000B8BF5B42984506DD05991546049AC1F834
:1008A00000B0984617703560C9EB04041FB3013FD0
:1008B000E317DDE9000122460BF03EF9A0F5C33055
:1008C000A03800F5C333A033002ED3D10028B8BF21
:1008D00040428045A9465D46AEDD059B1D60049BF8
:1008E0001F70084B06359D428046B146A8D1404650
:1008F00009B0BDE8F08FA9465D469DE7A0860100DE
:100900008CE30000DAE300002DE9F04182B002AC94
:10091000002544F8045D1E4D089E2F6915462246A9
:100920009846B8479DF804403470074600BB66B24D
:10093000002E21DB730904F01F0420331549012226
:10094000A24041F82320BFF34F8FBFF36F8F304693
:1009500008F0C8FC06F160432D0103F56143EDB2D8
:1009600083F800530C4B1B6853F83630C3F80080F3
:10097000384602B0BDE8F081304608F0B3FC074BC2
:1009800004F00F042D012344EDB21D76EAE700BF09
:1009900050E5000000E100E04CEB0000FCEC00E062
:1009A00030B129B11D4B42689A4203D007207047ED
:1009B0000120704770B58268002382B004460E465D
:1009C0004B600B602AB391681068009301938B69A8
:1009D00069469847E278009B02F0030203FB02F3AA
:1009E0007360E06888B1836800689B6900250095A2
:1009F000019569469847E278009B02F0030203FBE9
:100A000002F32846336002B070BD4FF0FF3333600D
:100A1000F9E74FF0FF334B60E3E700BF554943531D
:100A200050B149B142B110B40B4B44689C4205D05F
:100A300007205DF8044B704701207047C37803F02E
:100A40000303022B01D00020F3E7114311F0010F43
:100A50000CBF00200320ECE755494353F0B583B0A9
:100A600004460E461546FFF7DBFF98B9E278A36807
:100A700002F0030283B199680090013A01908F69F6
:100A800018686946D540B847009B9D4212D8A178A6
:100A900029B1082003B0F0BD184603B0F0BDA3682B
:100AA0000122A2709A6818685468ABB23246A04717
:100AB00003B0F0BD012003B0F0BD00BF30B59468B5
:100AC00083B0002C32D01468002C2FD052686AB347
:100AD00012685AB30978D57894786FF387156FF355
:100AE00045140229D570947023D0D1786FF3051185
:100AF000D17019460346124A1B7802A80024142517
:100B000001940094ADF8063000F8045D13696A465C
:100B100098479DF90030213308D0069ABDF802307D
:100B20001380079B20461C7003B030BD012003B02A
:100B300030BDE9B2012464F30511D170D9E700BFDB
:100B400050E5000010B50C4620B1836813B1DB6995
:100B500000689847236833B19A6822B1D26918684F
:100B6000BDE81040104710BD2DE9F04184B043F6B8
:100B700097250A9CAC4203D9032004B0BDE8F0815C
:100B80000028F9D0054604A8002400F8084D98462E
:100B900017460E4608F0C6F9124B03949B699DF860
:100BA000080003A9984704460028E5D101230193D2
:100BB0000398CDF800803B4629463246FFF722FED7
:100BC0000A9B984201DC0020D7E73B460398CDF80A
:100BD0000080019429463246FFF714FE0A9B8342A7
:100BE000CADBF0E7F8E50000F0B1E9B1414B42683B
:100BF0009A421BD02DE9F0473F4B90B005460E4678
:100C00000878DA681421002304930793ADF81200E2
:100C10008DF81010089309930A9304A807A9904728
:100C200030B110B0BDE8F087012070470820704750
:100C3000079F6F6204A808F095FB0028F1D1BDF86A
:100C400022202E490590C2F3810242F210738A5C81
:100C50006A70326AEB62002A38D0137B92F80090F7
:100C60006BBBE97863F38201E97098461369244A03
:100C7000EB62FF218DF80F1006927068B9F1000F3A
:100C80002BD005F11B03F27B009301212B4604A816
:100C9000FFF73AFE05F11803327B009304A8022106
:100CA0002B46FFF731FE044660B3A86805F10C013E
:100CB000FFF748FF04A808F089FB2046B1E7EB786E
:100CC00043F00403EB700DF11408CFE7FF200C494B
:100CD0008DF80F0070680691904600930DF10F019A
:100CE00006AA4346FFF740FF04460028DDD18146AF
:100CF000C7E700BF5549435350E50000DCE300005F
:100D00008CE3000005F11903727B009304A8052110
:100D10002B46FFF7F9FD04460028C6D105F11A035A
:100D2000B27B009304A804212B46FFF7EDFD044697
:100D30000028BAD13269EB787169AA60012262F3A6
:100D40000103EB70327AE960022A03D1EB7862F397
:100D50000103EB70D6F810C0BCF1000F3DD0DCF8F9
:100D600004400FCC0DF12C0AD646AEE80F000CAAB9
:100D7000246800920DF1320301936246CEF80040E0
:100D8000304606F108010223FFF798FE04460028CA
:100D90008BD1326969785368E8781B68002900F0C4
:100DA000928100F003000228696A00F08A81113103
:100DB0005960916893F802E0DC7810680A680221B3
:100DC00061F3830E6FF38304DC70514683F802E015
:100DD0009047044600287FF468AFD6F814C0BCF1F1
:100DE000000F3ED0DCF804400FCC0DF12C0AD646A3
:100DF000AEE80F000CAA246800920DF132030193B3
:100E00006246CEF80040304606F108010523FFF7A0
:100E100055FE044600287FF448AF7269697853682C
:100E2000E8781B68002900F0658100F003000228C3
:100E3000696A00F064810F319960916893F802E06B
:100E4000DC7810680A68022161F383046FF3830E73
:100E5000DC70514683F802E09047044600287FF496
:100E600024AF04A808F006FA00233B70BB703A795F
:100E700002B13B71F223FF22BB714FF4784A7A70C2
:100E800000234FF0400E03240620BA740699FB712C
:100E90009DF80FC03B727B72BB72FB723B737B731E
:100EA0003B73A7F814A07B8387F813E03C7738776F
:100EB000B9F1000F40F0D280BB7823F00303BB7080
:100EC00087F801C0FB798A7823F0400302F0010221
:100ED00043EA8213FB71FB79CA7823F0100302F016
:100EE000010243EA0213FB710A79FB7902F0010265
:100EF00023F0080343EAC203FB714B79397803EA14
:100F0000040221F0030313433B70B8F1000F0AD031
:100F1000D8F80030FF2B00F2C680FA79DBB242F03D
:100F20000402FA71BB746A786B6A2AB39A8A42F037
:100F300001029A829A8A42F002029A823269002A57
:100F400000F0C8809A8A22F470629A8269789A8A3C
:100F5000013901F00F01C2F30B0242EA01329A8219
:100F60009A8A42F004029A829A8A5207FCD49A8A98
:100F700022F0F0029A826B6A1A78717A42EA0112C0
:100F8000D2B21A70327A012A00F08480022A00F06C
:100F90008F80B17A1A7801F0010122F0080242EA4A
:100FA000C1021A70F27A1AB15A7B42F002025A73E5
:100FB000316AD9B1DA79887802F07F0242EAC01248
:100FC000DA71DA79C87822F0200200F0010042EAF2
:100FD00040120020DA7118724A78997898780A439A
:100FE00002F0030120F003020A439A7033782B7059
:100FF000F369B2692B620023EA612B616B61AB700C
:10100000BB8A23F00803BB82BB7843F01003BB709C
:101010002A7EE97E53B2002B08DB02F01F025B0937
:1010200001203D4C00FA02F244F823204BB2002B81
:1010300007DB01F01F015B09012237488A4040F8B5
:101040002320BB78354943F04003BB706A6A93782C
:1010500043F02003937000206960E2E57A70FB7929
:1010600023F04003FB71FB7923F00803FB713B780D
:1010700023F003033B70BB7823F0030343F0020328
:10108000B9F1020FBB707FF44EAFFB7943F0100350
:10109000FB7148E71A7842F040021A709A7942F0E0
:1010A00010029A7175E7FB7923F00403FB713AE7AC
:1010B0001A7822F040021A709A7922F010029A717E
:1010C00067E7103174E600F003000128696AF8D17F
:1010D00005316DE66A78316A013A92B299B10879C0
:1010E000998A024002F00F0021F4706242EA002265
:1010F0009A822BE700F003000128696A01D00E31C3
:101100009AE6033198E6998A02F00F0221F47061A1
:1011100041EA02229A8219E700E100E0554943536F
:1011200078B138B54268454B9A4201D0072038BDA6
:1011300011F0FD0F04460D4605D00620012D66D99D
:1011400038BD01207047426A937803F07B039370A7
:1011500090F9190008F0C6F8627E53B2002B18DB34
:101160005B0920330121364802F01F0201FA02F226
:1011700040F82320BFF34F8FBFF36F8F627E53B2CF
:10118000002B06DB5B09603302F01F02914040F840
:10119000231094F91A0008F0A5F8A27E53B2002B90
:1011A00018DB5B0920330121254802F01F0201FAF8
:1011B00002F240F82320BFF34F8FBFF36F8FA27E60
:1011C00053B2002B06DB5B09603302F01F02914033
:1011D00040F82310E06898B183680068DB6898479E
:1011E00063783BB1626A938A43F004039382938AE3
:1011F0005B07FCD400232361636100289ED038BDC7
:101200006378002BEED123616361184696E7A068EE
:1012100070B10023A37083680068DB689847637827
:10122000002B8DD0626A938A43F00203938238BD0B
:101230006378002BF6D1184682E700BF5549435327
:1012400000E100E0002878D03D4B42689A4201D08E
:101250000720704770B50022436A42609A7802F016
:101260000B029A70017E4AB2002A82B00DDB52094D
:1012700020320124334D01F01F0104FA01F145F839
:101280002210BFF34F8FBFF36F8FC17E4AB2002A87
:101290000DDB5209203201242A4D01F01F0104FA0E
:1012A00001F145F82210BFF34F8FBFF36F8F417EDE
:1012B0004AB2002A0DDB520920320124214D01F0EF
:1012C0001F0104FA01F145F82210BFF34F8FBFF35D
:1012D0006F8F817E4AB2002A0DDB52092032012431
:1012E000184D01F01F0104FA01F145F82210BFF377
:1012F0004F8FBFF36F8F04469A78987802F00201FF
:1013000020F003020A439A7004F10C0102AEA068B7
:10131000FFF718FC00251423019506F8043DE5614C
:101320002378A5623046ADF8063007F09FFF3046BF
:1013300008F04CF8284602B070BD0120704700BF8D
:101340005549435300E100E0C378427803F00303BA
:10135000022B10B4036918D01978436A8CB27AB1A1
:101360001A79D209FCD0DC81C2780469416902F0A3
:101370000303C91A2344416103615DF8044B7047BC
:101380001A79D209FCD0D970EEE71C88436A002A8A
:10139000E6D11A79D209E6D11A79D209F9D0E2E771
:1013A0002DE9F04182B004460E461546FFF738FBA2
:1013B00010B92369082013B102B0BDE8F081676A53
:1013C000BA7802F07B02BA70E268266165611AB3EE
:1013D000E1789068009301F003086361019308F1DC
:1013E000FF3E83691068694625FA0EF59847009B11
:1013F0009D4240D86378002B3FD1013DC4F8148052
:101400000AD006EB0801E3689A6818685668ABB220
:101410000022B0470028CFD194F9190007F062FFED
:10142000627E53B2002B0FDB5B099B0003F160432C
:10143000012103F5614302F01F0201FA02F2C3F831
:101440008021617801B11A60BB7843F0A003BB70C2
:10145000637873B9636993B9627E53B2002B08DB7A
:1014600002F01F025B090121074801FA02F240F86D
:1014700023200020A0E701209EE73146C3E7204655
:10148000FFF762FFE8E700BF00E100E028B3384B58
:1014900042689A4201D007207047F0B5456AAB78A0
:1014A00013F0030387B01AD1C278059302F0040247
:1014B00002F0FF06AAB904462E4FE36A0093FF2309
:1014C00008468DF80F300DF10F0104AA334604973A
:1014D000FFF74AFB38B107B0F0BD0120704701208B
:1014E000F9E705AEE7E7AB789DF80F1003F00B03C3
:1014F000AB702061AB78049A23F00303AB70697082
:10150000EB79917823F0400301F0010143EA811364
:10151000EB71EB79D17823F0100301F0010143EA7C
:101520000113EB711179EB7901F0010123F008034C
:1015300043EAC103EB715379297803F0030221F0E8
:10154000030313432B7046B13368FF2B0AD8EA79A3
:10155000DBB242F00402EA71AB74AB7843F05003A3
:10156000AB70B8E7EB7923F00403EB71F5E700BF4C
:10157000554943538CE3000070B5054684B0437869
:10158000296A00780090802203916C6AADF80420EB
:1015900083B9EB7803F00303022B0CBF228A627934
:1015A000EB690CBF92B2D2B213B10292684698476F
:1015B00004B070BDFE26267103E0238AEA699BB25F
:1015C0004AB9E38ADA06F8D1BF2323712379DB070E
:1015D000F1D404B070BDC3F308030293684690478A
:1015E000EFE700BFF0B585B0EFF30380103840B2ED
:1015F00007F078FEEFF303833B4A103B5BB21268BF
:1016000052F833301C6824B1E568666A1DB163691D
:101610003BB105B0F0BD6378002B4BD16369002B63
:101620005ED194F91A0007F05DFEA27E53B2002B42
:1016300009DB5B09603302F01F0201212B4801FA2C
:1016400002F240F82320B37803F07F0343F0040351
:10165000B370627E53B2002B0DDB5B092033012196
:10166000224802F01F0201FA02F240F82320BFF3E1
:101670004F8FBFF36F8FA27E53B2002B08DB02F0B7
:101680001F025B090121194801FA02F240F82320E8
:10169000E36900222261002BBBD02178206A0091EF
:1016A0004FF4807103900292ADF804106846984799
:1016B00005B0F0BDF78AC7F30427DF1B002F02DC5B
:1016C00009E0BD4207D063690135002BF9D02046FF
:1016D000FFF73AFEF5E7337903F07F03337196E7BE
:1016E0002046FFF731FE92E74CEB000000E100E0FE
:1016F00010B584B0EFF30380103840B207F0F2FD6C
:10170000EFF303830F4A103B5BB2126852F8333099
:10171000186828B183780278012B03D0FFF72CFFDB
:1017200004B010BDC169002484700029F8D0006A9B
:10173000039000920294ADF804306846884704B0E4
:1017400010BD00BF4CEB000030B585B0EFF3038354
:10175000194A103B5BB2126852F833301B681BB356
:10176000596A1C788A7802F07B028A70997E4AB2A4
:10177000002A0DDB520920320120104D01F01F011B
:1017800000FA01F145F82210BFF34F8FBFF36F8FBE
:10179000DA694AB11B6A0393002102230094029183
:1017A000ADF8043068469047EFF30380103840B23C
:1017B00007F098FD05B030BD4CEB000000E100E003
:1017C00020B1034B1B680360002070470120704765
:1017D00018E400002DE9F04F00F1380683B004460C
:1017E00030468A46914698469DF830B09DF8347050
:1017F00007F0A4FD054620B10A25284603B0BDE840
:10180000F08FD4F818C0CDF804C09CF8023023F053
:1018100040038CF802309CF8023003F07F038CF810
:1018200002309CF8022007F0010322F004028CF839
:101830000220A062E062C4F8308084F835B0C4F8B9
:1018400020A0C4F8249084F8377084F836309CF8CF
:101850000D3023F010038CF80D3094F91E0007F0C2
:1018600041FD94F91D0007F03DFD94F91C0007F0BF
:1018700039FD94F91F0007F035FDB8F5803F57D2C8
:10188000A368DDF804C01BB3A269CDF804C0022F21
:1018900002F1030904BF3F4A226294F83420186819
:1018A0000CBFAA464FF0020A52459A6805D0D36889
:1018B000984700284ED005463BE0D2F804A0216AA4
:1018C0004A461FFA88F3D047DDF804C00028F2D159
:1018D000E3688BB1012F30D09A68A1695768186806
:1018E000626ACDF804C01FFA88F30531B847DDF805
:1018F00004C018B105461CE0012F1ED09CF8023030
:1019000043F040038CF802309CF8023063F07F0310
:101910008CF802309CF8023043F030038CF802302F
:10192000A36893B39CF80530284603B0BDE8F08F58
:101930000125304607F012FD5FE79CF8023063F0A6
:101940007F038CF802309CF8023043F020038CF8BF
:101950000230E5E7A068236A4168826809689268F6
:1019600091F803E04B606AF3830E1FFA88F3CB8192
:1019700081F803E0C1F808900068904784F834A02B
:10198000DDF804C00028A3D095E7E368002BC9D197
:1019900033E700BF34E4000008B1012B01D001207F
:1019A00070474AB141B130B54568094CA54283B092
:1019B00004D0072003B030BD184670471C461346BC
:1019C0000A460221019100940021FFF703FFF1E78D
:1019D0005349435308B1012B01D0012070474AB14C
:1019E00030B583B041B14568084CA54206D0072008
:1019F00003B030BD184670471846F9E71C460094FE
:101A0000134601940022FFF7E5FEF1E753494353E3
:101A1000F0B583B09DF8204008B1012C02D0012020
:101A200003B0F0BD4BB141B13AB14668074DAE428B
:101A3000864605D0072003B0F0BD204603B0F0BDB8
:101A400003258DE83000FFF7C5FEE9E7534943530E
:101A5000002800F08280424B42689A4201D0072061
:101A6000704730B58369002242609A7822F04002C4
:101A70009A709A7802F07F029A709A7822F00402A3
:101A80009A70427F53B2002B83B00DDB5B09203389
:101A90000121344C02F01F0201FA02F244F8232023
:101AA000BFF34F8FBFF36F8F027F53B2002B0DDB5D
:101AB0005B09203301212B4C02F01F0201FA02F2D4
:101AC00044F82320BFF34F8FBFF36F8FC27F53B211
:101AD000002B0DDB5B0920330121224C02F01F0299
:101AE00001FA02F244F82320BFF34F8FBFF36F8F48
:101AF000827F53B2002B0DDB5B0920330121194C8F
:101B000002F01F0201FA02F244F82320BFF34F8FC4
:101B1000BFF36F8F02AD00221423019205F8043D3C
:101B200004460378ADF80630284607F09FFBE368CB
:101B30001BB19A681868D3699847A3681BB19A6863
:101B40001868D369984704F1380007F007FC284665
:101B500007F03CFC002003B030BD0120704700BFFF
:101B60005349435300E100E02DE9F04F93B021B316
:101B700018B3144F00230C464FF01408097806934D
:101B80000546ADF81A10FA6809930A930B930C9363
:101B90008DF8188006A809A9904720B10546284667
:101BA00013B0BDE8F08F06A807F0DCFB814658B102
:101BB0000A25284613B0BDE8F08F0125284613B04A
:101BC000BDE8F08F50E5000049463C2228460AF067
:101BD000A3FA099E3A69AE6123780192CDF820906C
:101BE0000DAAADF822308DF82080CDF8349008A8E9
:101BF0000221019B677898479DF834202A770028B6
:101C000040F0688253B2002BC0F2738203F160434C
:101C100003F561433F01FFB283F80073C34A95F9AE
:101C20001C30176857F833200023156008A80D935F
:101C30000521019B94F802800DAA98479DF8343045
:101C40006B77002840F046825AB2002AC0F27082B8
:101C500002F1604303F561434FEA0812D2B283F800
:101C6000002395F91D3057F833200023156008A88C
:101C70000D930421019B94F803800DAA98479DF8C9
:101C80003430AB77002840F025825AB2002AC0F2E7
:101C9000688202F1604303F561434FEA0812D2B251
:101CA00083F8002395F91E3057F833200023156080
:101CB00008A80D930121019B94F804800DAA984770
:101CC0009DF83430EB77002840F004825AB2002AA5
:101CD000C0F2518202F1604303F561434FEA0812FA
:101CE000D2B283F8002395F91F3057F833301D60C6
:101CF0002378039306A807F0BDFA4FF47847002332
:101D0000FF224FF0F20E032140203370B370337185
:101D100086F806E07270B274F37133727372B37244
:101D2000F372337373733373B7827383F0743177E1
:101D3000B37823F04003B370B37803F07F03B3703C
:101D4000B37823F00403B37095F91D0007F0CAFAC5
:101D500095F91C0007F0C6FA95F91F0007F0C2FAC2
:101D600095F91E0007F0BEFA95F81DA04FFA8AFCFF
:101D7000BCF1000F09DB4FEA5C1360330AF01F006F
:101D800001226B49824041F8232095F81CE04FFA6C
:101D90008EF1002908DB4B0960330EF01F0701228A
:101DA0006348BA4040F82320EF7F7AB2002A0ADB6A
:101DB0005309603307F01F090120DFF8748100FA2E
:101DC00009F048F82300AB7F029318465BB2002B62
:101DD0000CDB4FEA531800F01F0B08F160084FF0BE
:101DE0000109534809FA0BF940F82890BCF1000F9B
:101DF0000BDB0AF01F094FEA5C1C4FF00108DFF80B
:101E000030A108FA09F84AF82C8000290ADB0EF004
:101E10001F0E49094FF0010CDFF814810CFA0EFE79
:101E200048F821E0002A08DB07F01F0752090121CA
:101E3000DFF8FCE0B9404EF82210002B08DB029AD4
:101E40003B4902F01F005B090122824041F8232038
:101E5000B38A23F00103B382B37923F00103B37192
:101E6000737A23F001037372337863F07F03337066
:101E7000737B23F001037373236A002B00F02F811F
:101E80001B78002B00F02B81F37943F00403F371EE
:101E9000002308A88DF817300D938DF82030D4F862
:101EA0000C8007F03FF8234B9DF820009B690DA99B
:101EB00098470746002840F01781B8F1000F00F05E
:101EC00013810D98DFF870E03A4639463EF802304B
:101ED00008FB03F3B0FBF3F3013BFE2B02F1060218
:101EE00040F2308101310429F0D10127FF23F2793A
:101EF000520723D5002207929DF8172002EB4202D9
:101F00004FEA08283EF8122002FB08F803FB088875
:101F1000B8FBF0F00790079B7F2B0FD9079BFF2B97
:101F20000CD8079BDBB2B37408E000BF4CEB000099
:101F300000E100E0F8E5000000E40000002F40F0C0
:101F4000D38061692269B2FA82F3081C18BF0120AC
:101F50005B09834200F0D580002845D08B68002BB8
:101F600000F0D1800B68002B00F0CD80486800287D
:101F700000F0C9800268002A00F0C580D37891780B
:101F80004FF0020C67F387136CF3830167F383034D
:101F900067F3051367F34511D37091708646BEE869
:101FA0000F000DF13408A8E80F00DEF80030C8F883
:101FB00000306146019B089706A808AA98479DF93A
:101FC0002030213300F09F8063690F979A68BDF835
:101FD0002210126818688DF83A70ADF838100DA903
:101FE0009047002876D12269002A44D09368002BBC
:101FF00000F097801368002B00F093805768002F43
:1020000000F08F803A68002A00F08B80D3789178B6
:10201000022003F03F0360F3830301F0F3016FF349
:1020200005136FF34511D37091700FCF0DF1340E7E
:10203000AEE80F004FF000083B68CEF8003008AA69
:10204000019BCDF8208006A8052198479DF92030F6
:10205000213366D02369CDF83C809A68BDF82270A0
:10206000126818688DF83A800DA9ADF8387090475D
:10207000002840F08A806379012B4BD0B37823F09D
:102080000303B3706379A279E179012B14BF0023B4
:102090000523012A39D0012914BF43F0800343F0FE
:1020A000C0037373637A1BB9B37943F00803B37148
:1020B0009DF80C30A269E6692B7060692169344B88
:1020C0002A6102226E61E860A96085F834206B60A5
:1020D000002564E5054606A807F078F95FE5F37981
:1020E00023F00403F371D3E606A807F06FF9012586
:1020F00055E5284902F00F023B011144DBB20B7693
:102100008CE50325E7E70125E5E70029C9D143F080
:102110004003C6E7B37823F0030343F00203B37030
:10212000B0E7012563699A681868D3699847D2E7D0
:10213000184A03F00F031A444FEA08185FFA88F3AD
:1021400013768EE5C9B28DF81710D9B29DF8172015
:102150007170317802F0030221F003010A433270FA
:10216000C5E60C4A03F00F031A444FEA08185FFA59
:1021700088F3137696E5074A03F00F031A444FEAF3
:1021800008185FFA88F31376ADE50546CAE700BF85
:1021900053494353FCEC00E010B5EFF30384103CCB
:1021A00064B2204607F09EF82B4B1B6853F834307E
:1021B0001C68E36813B3236BA362A269937803F0EE
:1021C0007F03937094F91D0007F08CF8627F53B27F
:1021D000002B09DB5B09603302F01F0201211F485D
:1021E00001FA02F240F8232094F83730012B04D191
:1021F000A269937843F00403937010BDA368002B89
:10220000D9D1A269537B5B0701D5A36A43B194F886
:102210003730012B1EBF937803F07F039370A36ABE
:10222000226B9A420DD994F836206AB1216AA269CC
:10223000C95C1379DB09FCD0D170A36A226B01332E
:10224000A3629A42D9D1B8E7A2691379DB09FCD01D
:10225000FF23D370F1E700BF4CEB000000E100E08A
:1022600010B584B0EFF30384103C64B2204607F04D
:1022700039F8284B1B6853F834301C68E3680BB3FB
:10228000236BE362A269937823F040039370A26901
:10229000937803F07F039370A269937803F0CF03E0
:1022A0009370236943B121786269019101218DF80E
:1022B0000810039201A8984704F1380007F04EF87F
:1022C00004B010BDA368002BDAD1A169E36A626A89
:1022D0004979D154E36AA16A226B01339142E362E6
:1022E0000ED294F8363073B1236AA269595C13791F
:1022F000DB09FCD0D170A16AE36A226B0131A162D3
:102300009A42DDD1BEE7A2691379DB09FCD0FF2335
:10231000D370F0E74CEB000030B585B0EFF30384E9
:10232000174B103C64B21B6853F834301D68AA691F
:10233000937823F040039370AA69937803F07F03A6
:102340009370AA69937823F004039370AA69937831
:1023500003F0CF0393702B6943B129786A69019127
:1023600001218DF80810039201A8984705F1380063
:1023700006F0F4FF204606F0B5FF05B030BD00BF03
:102380004CEB000030B585B0EFF30383184A103BE7
:1023900012685BB252F833301C682369A569227851
:1023A0005BB101922A7992064CBF062202228DF877
:1023B00008206269039201A8984704F1380006F0EA
:1023C000CDFF2B7903F0C7032B71EFF30380103897
:1023D00040B206F087FFEFF30383103B5BB2054A80
:1023E000C03352F823300093009B05B030BD00BFCE
:1023F0004CEB000000600040826A036B9A423AD2C4
:1024000070B590F8353082B04FF0FF31019193B143
:1024100090F83410036A02FB01F261B1013952FAFB
:1024200081F101311944134401AA13F8014B02F858
:10243000014B8B42F9D10446EFF31086012585F359
:10244000108890F91E0006F04DFFA27F53B2002BBA
:1024500007DB5B09603302F01F020749954041F832
:102460002350A369019A5A6086F31088A36A013346
:10247000A36202B070BD704700E100E030B585B0E6
:10248000EFF30380184B103840B21B6853F830301C
:102490001C68A269137803F00F031370A27F53B274
:1024A000002B0DDB5B0920330121104D02F01F02D0
:1024B00001FA02F245F82320BFF34F8FBFF36F8F6D
:1024C00006F010FF236943B121786269019101216F
:1024D0008DF80810039201A8984704F1400006F017
:1024E0003DFF05B030BD00BF4CEB000000E100E057
:1024F00070B584B0EFF30384103C64B2204606F05C
:10250000F1FE384B1B6853F834301C6894F8365091
:10251000002D42D0236BE362A3691A78120710D50D
:10252000DB789B070DD5A27F53B2002B33DB02F083
:102530001F025B0901212C4801FA02F240F8232016
:1025400029E0A37F58B200280FDB40092030012288
:10255000254903F01F0302FA03F341F82030BFF3CB
:102560004F8FBFF36F8F94F91E0006F0BBFEA26978
:10257000137803F00F031370236943B12178626964
:10258000019101218DF80810039201A8984704F1E8
:10259000400006F0E3FE04B070BDA3695B68E3632E
:1025A0002046FFF729FFE16A206B814216D294F89A
:1025B0003460626A01FB06F376B11A4404F13B0110
:1025C0002B4611F8010F02F8010B94F83400013387
:1025D0008342F6D3E16A206B0131E16288429BD0ED
:1025E00004B070BD4CEB000000E100E010B584B019
:1025F000EFF30384103C64B2204606F073FE384BC0
:102600001B6853F834301C6894F83630A3B9A369BA
:102610001A7812074FD594F83920012A03D01A7876
:1026200022F020021A702046FFF7E6FE226BA36A12
:102630009A4203D004B010BD236BA362A269137841
:1026400023F020031370637F58B200280FDB40098A
:1026500020300122234903F01F0302FA03F341F85B
:102660002030BFF34F8FBFF36F8F94F91D0006F03A
:1026700039FE627F53B2002B09DB5B09603302F045
:102680001F020121174801FA02F240F82320A36932
:102690001B781B0713D594F83930012BCAD1A17FC1
:1026A0004AB2002AC6DB01F01F0152090D488B40D7
:1026B00040F82230BEE7A26A002AB4D0ABE7236913
:1026C00043B121786269019101218DF808100392CC
:1026D00001A8984704F1400006F040FE04B010BD88
:1026E0004CEB000000E100E030B585B0EFF3038370
:1026F0002C4A103B12685BB252F833301C68A26956
:102700002178D378DBB2D8072ED50620BC238DF8EC
:102710000800D370A27F53B2002B0DDB5B0920337E
:102720000120214D02F01F0200FA02F245F8232099
:10273000BFF34F8FBFF36F8FA269137803F00F03BE
:102740001370236923B162690191039201A898472C
:1027500004F1400006F002FEEFF30380103840B2AF
:1027600006F0C0FD05B030BD5D0707D5D8060DD415
:1027700003238DF80830B923D370CBE71B070CD5A2
:102780000520B5238DF80800D370C3E70820AD23DA
:102790008DF80800D370A269EDE702238DF80830A8
:1027A000B8E700BF4CEB000000E100E020B1034BB4
:1027B0001B680360002070470120704754E400004C
:1027C00030B5C26985B0044662B1836BC56B006ADF
:1027D00001905B1B02938DF80C1001A89047002319
:1027E00084F84B30E36A0022DA7194F8332053B254
:1027F000002B0DDB5B0920330121254802F01F026D
:1028000001FA02F240F82320BFF34F8FBFF36F8F1E
:1028100094F8302053B2002B0DDB5B0920330121EB
:102820001B4802F01F0201FA02F240F82320BFF316
:102830004F8FBFF36F8F94F8322053B2002B0DDB14
:102840005B0920330121124802F01F0201FA02F253
:1028500040F82320BFF34F8FBFF36F8F94F83120E0
:1028600053B2002B0DDB5B0920330121084802F035
:102870001F0201FA02F240F82320BFF34F8FBFF38B
:102880006F8F04F1510006F069FD05B030BD00BF47
:1028900000E100E0F0B583B002AD002445F8044D3E
:1028A000134C089E276914462A461D46B8479DF8D2
:1028B0000410317088B94AB2002A10DB02F160427C
:1028C00002F561422401E4B282F80043094B96F913
:1028D00000201B6853F832301D6003B0F0BD064B7A
:1028E00001F00F0124010B44E4B21C76EEE700BFB7
:1028F00050E500004CEB0000FCEC00E070B5044635
:1029000082B038B1806A0F4B984218BF072004D0BC
:1029100002B070BD012002B070BD04F15106304616
:102920008DE8060006F00AFD9DE80600054608B1A0
:102930000820EDE730462181A27206F00FFD2846FF
:10294000E6E700BF4349495230B5456985B00446C2
:1029500035B190F8493003F0FF02002B00F0888178
:10296000A56925B194F84930002B40F06D81E06BEA
:1029700020B994F84C30002B00F08D81E36A0022DE
:10298000DA7194F8332053B2002B0DDB5B0920334E
:102990000121C44802F01F0201FA02F240F823208C
:1029A000BFF34F8FBFF36F8F94F8302053B2002BDB
:1029B0000DDB5B0920330121BA4802F01F0201FA46
:1029C00002F240F82320BFF34F8FBFF36F8F94F8CC
:1029D000322053B2002B0DDB5B0920330121B148BB
:1029E00002F01F0201FA02F240F82320BFF34F8FDA
:1029F000BFF36F8F94F8312053B2002B0DDB5B09CE
:102A000020330121A74802F01F0201FA02F240F828
:102A10002320BFF34F8FBFF36F8FE36A5A785206BC
:102A200000F1B1801A7802F07F021A701978E26A18
:102A3000C9098DF805101978C9098DF805101B789A
:102A4000DB098DF805309DF80530137843F040031D
:102A500013701378E16AC3F380138DF80430137890
:102A6000C3F380138DF804301378C3F380138DF80B
:102A7000043000239DF804204B7294F9330006F0D3
:102A800031FC94F8332053B2002B09DB5B0960332F
:102A900002F01F020121834801FA02F240F82320CC
:102AA00094F9300006F01EFC94F8302053B2002B4D
:102AB00009DB5B09603302F01F020121794801FA4A
:102AC00002F240F8232094F9320006F00BFC94F84F
:102AD000322053B2002B09DB5B09603302F01F0286
:102AE0000121704801FA02F240F8232094F93100E4
:102AF00006F0F8FB94F8312053B2002B09DB5B0998
:102B0000603302F01F020121664801FA02F240F828
:102B10002320E26A137863F07F0313701178E36A6D
:102B2000C9098DF803101178C9098DF803101278BE
:102B3000D2098DF803209DF803201A7822F0400274
:102B40001A701A78C2F380128DF802201A78C2F334
:102B500080128DF802201B78C3F380138DF80230A9
:102B6000204601219DF80230FFF72AFE002394F849
:102B70004610A26BE36384F84C3084F8481022645A
:102B8000122005B030BD9A7812F0070220D0511CF7
:102B90001A7842F020021A701A78C2F340128DF8A7
:102BA00008201A78C2F340128DF808201A78E36AD8
:102BB000C2F340128DF808209DF808201A78950677
:102BC000FCD44A1E12F0FF01E2D11A78D0076BD56F
:102BD0005A7842F008025A705978E26A94F8520022
:102BE000C9B28DF807105978C9B28DF80710597815
:102BF000C9B28DF807109DF80730D17841F0020175
:102C0000D170D37823F00103012808BF43F00103FA
:102C1000D370537943F001035371E36A00228DF8B6
:102C200006205A78110708D40BE05A7A02F0010204
:102C30008DF806205A78120703D59DF80620002A41
:102C4000F3D09DF80620EDE6AB6828689B6900226A
:102C50008DF80E2002A998479DF80E30002B3FF406
:102C600086AEAB6828685B6998470123E36385E615
:102C7000AB6828689B698DF80E2002A998479DF8DB
:102C80000E30002B3FF46CAEAB6828685B69984748
:102C90000123E36364E694F84B30002B7FF46EAEBF
:102CA0006FE700BF00E100E01A7822F010021A700E
:102CB0001A7842F004021A70E36A89E728B1404AA0
:102CC000816A914203D0072070470120704730B5D8
:102CD000044683B0FFF738FEA36900220546A262CE
:102CE0001BB19A681868D369984763691BB19A68E1
:102CF0001868D3699847E36A0022DA7194F83320A0
:102D000053B2002B0DDB5B09203301212D4802F06B
:102D10001F0201FA02F240F82320BFF34F8FBFF3E6
:102D20006F8F94F8302053B2002B0DDB5B092033FA
:102D30000121244802F01F0201FA02F240F8232088
:102D4000BFF34F8FBFF36F8F94F8322053B2002B35
:102D50000DDB5B09203301211A4802F01F0201FA42
:102D600002F240F82320BFF34F8FBFF36F8F94F828
:102D7000312053B2002B0DDB5B09203301211148B8
:102D800002F01F0201FA02F240F82320BFF34F8F36
:102D9000BFF36F8F14F8512B0021152301A8019167
:102DA000ADF806208DF8043006F060FA01A806F0B0
:102DB0000DFB204606F0D2FA284603B030BD00BF16
:102DC0004349495200E100E028B1826A044B9A422B
:102DD00003D00720704701207047FFF7B5BD00BF43
:102DE0004349495210B4C46A90F83320E17953B290
:102DF00041F01F01002BE17108DB02F01F025B09AB
:102E00000121234C01FA02F244F82320C46A90F80D
:102E10003020E17953B241F02001002BE17108DB51
:102E200002F01F025B090121194C01FA02F244F879
:102E30002320C46A90F83220E17953B201F0BF0137
:102E4000002BE1710DDB5B0920330121104C02F0F6
:102E50001F0201FA02F244F82320BFF34F8FBFF3A1
:102E60006F8FC46A90F83120E17953B241F080014C
:102E7000002BE17108DB02F01F025B09012104480D
:102E800001FA02F240F823205DF8044B704700BFBE
:102E900000E100E02DE9F04F97B0002840D0002974
:102EA0003ED0274E4B68B3423AD84B6A002B37D0FE
:102EB000244CE36803930D460023097806931522FA
:102EC000074609930A930B930C93ADF81A108DF8EB
:102ED000182006A809A9039B984730BB6B68B3422A
:102EE00028D006A806F03EFAF8B96A6A099B12785B
:102EF00087F85220FB622A780D90152311901290CA
:102F0000139014908DF83430ADF836200DA811A927
:102F1000039B9847C0B1044606A806F057FA00E0A4
:102F20000124204617B0BDE8F08F0446204617B0B4
:102F3000BDE8F08FBDF82A305B07D2D40324F0E758
:102F400040420F0050E5000007F13003AA7B0093D8
:102F50000DA801213B46FFF79DFC0028DBD107F1BE
:102F60003103EA7B00930DA803213B46FFF792FC57
:102F70000028D0D107F132032A7C00930DA802214A
:102F80003B46FFF787FC0028C5D107F133036A7C75
:102F9000009301463B460DA8FFF77CFC80460028C5
:102FA00040F04B82AC46BCE80F00BE46AEE80F00D6
:102FB000BCE80F00AEE80F009CE803008EE80300B9
:102FC00006A806F057F9FA6A137803F07F03137026
:102FD0001178FB6AC9098DF817101178C9098DF8A5
:102FE00017101278D2098DF817209DF817201A783B
:102FF00042F040021A701978FA6AC1F380118DF814
:1030000016101978C1F380118DF816101B78C3F3D0
:1030100080138DF816309DF8163082F8098097F9E4
:10302000330006F05FF997F8332053B2002B09DB29
:103030005B09603302F01F020121BB4801FA02F272
:1030400040F8232097F9300006F04CF997F830202B
:1030500053B2002B09DB5B09603302F01F02012130
:10306000B14801FA02F240F8232097F9320006F045
:1030700039F997F8322053B2002B09DB5B09603332
:1030800002F01F020121A84801FA02F240F82320B1
:1030900097F9310006F026F997F8312053B2002B4A
:1030A00009DB5B09603302F01F0201219E4801FA2F
:1030B00002F240F82320FB6A9C4A1978926961F079
:1030C0007F0119701978C9098DF815101978C90987
:1030D0008DF815101B780021DB098DF81530119142
:1030E000012011A99DF8153090478246002840F034
:1030F0001281119BD7F804B04FF06408A3FB088934
:103100000126324600234046494608F031FD5A4622
:10311000002308F02DFD63304FF0640241F10001FF
:10312000002308F025FD002908BF41285FFA8AF234
:103130004FEA46060AF1010AC0F00481BAF1080F0D
:10314000DFD17B4B9B4500F0F780FB6A97F852007C
:10315000D97841F00201D970DA7822F00102012811
:1031600008BF42F00102DA705A7942F001025A7146
:10317000FA6A537943F002035371FA6A537943F0C0
:1031800004035371FA6A537923F008035371FA6AFE
:10319000537943F0100353713846FFF723FEFB6A5F
:1031A0001A7822F040021A701978AA69C1F38011C6
:1031B0008DF814101978C1F380118DF814101B7854
:1031C000C3F380138DF814309DF81430002A63D0B7
:1031D000002329780893152207930D930E930F93DC
:1031E0001093ADF822108DF8202008A80DA9039B9C
:1031F0009847002840F09E80AB699A68002A00F04A
:10320000D2801A68002A00F0CE805B68002B00F0A4
:10321000CA801E68002E00F0C68097F93030213336
:1032200000F0C18008A82369012107AA98478646B3
:1032300020B1044606A806F019F86DE6F378B178D7
:10324000FA6ABDF81EC060F38713022060F38301A1
:103250006EF383036EF3051313326EF34511F370AF
:103260007260B170AE69D6F80490B9E80F000DF144
:103270004408A8E80F00D9F80030C8F80030CDF8AD
:103280004CE0B36830681B688DF84AE0ADF848C080
:1032900011A9984700284DD16B69002B00F0B3802D
:1032A000002328780893152207930D930E930F930C
:1032B0001093ADF822000DA98DF8202008A8039BDB
:1032C0009847002840F09D806B699A68002A00F0BA
:1032D000AD801A68002A00F0A9805B68002B00F01E
:1032E000A5801E68002E00F0A18097F931302133AF
:1032F00000F09C80236908A8032107AA9847044688
:10330000002852D0AB699A681868D369984700289A
:1033100018BF04468EE706A805F0A8FF06A8544685
:1033200006F054F8FDE500BF00E100E0F8E500001C
:1033300040420F0004467DE7FA6A537963F07F0349
:10334000537102E7C0F34701431ADBB2062B0DD9D4
:103350003B4883456CD0B2FA82F04009091AC0F1AB
:10336000FD000339034401F0FF01DBB2F86A41F0CC
:10337000E0010174F96A43F0E0034B74F96A8B7859
:1033800002F0070223F0700343EA02138B70FB6A1A
:103390001A7922F003021A715A7942F020025A7106
:1033A000D7F804B0CDE6012444E7F378B178FA6A9F
:1033B000BDF81EE060F38713022060F3830364F31B
:1033C000830164F30513123264F34511F370B17095
:1033D000B260D5F81480D8F804C0BCE80F0011AE74
:1033E0000FC6DCF8003033601394D8F80830D8F8F2
:1033F00000001B688DF84A4011A9ADF848E09847D5
:1034000008B104467EE700200E4B87F85100786330
:1034100087F84900B86387F84A00F86387F84B00DB
:10342000386487F84C000446BB627AE5012469E7FA
:103430000639063BC9B2DBB298E704466CE500BF2B
:10344000801A06004349495210B582B000237C21FE
:103450000122019104468DF8032080F84B3080F85A
:103460004D3080F84E3080F84F3080F8503090F872
:103470004C2094F84610806BE06384F8471084F881
:1034800048302364002A67D1019B6BB1E26A53780C
:10349000DB0903D108E05378DB0905D0019B013B30
:1034A0000193019B002BF6D1019B33B904F151002C
:1034B00005F054FF082002B010BDE36A00225A72E2
:1034C00094F9330005F00EFF94F8332053B2002B2B
:1034D00009DB5B09603302F01F0201213D4801FA5C
:1034E00002F240F8232094F9300005F0FBFE94F836
:1034F000302053B2002B09DB5B09603302F01F025E
:103500000121344801FA02F240F8232094F93200F4
:1035100005F0E8FE94F8322053B2002B09DB5B097A
:10352000603302F01F0201212A4801FA02F240F83A
:10353000232094F9310005F0D5FE94F8312053B2E0
:10354000002B09DB5B09603302F01F0201212148D7
:1035500001FA02F240F82320E36A94F85200D97885
:1035600041F00201D970DA7822F00102012808BF87
:1035700042F00102DA705A7942F001025A71204693
:10358000FFF730FC94F84C30D3B1002384F84C3072
:10359000E3693BB1002002B010BD94F8513003F054
:1035A000FF029BB19DF8033003F0FF02002BF4D122
:1035B00094F84B30002BEDD084F84B2012207AE7A2
:1035C000E26A537843F002035370E1E78DF8032079
:1035D000E8E700BF00E100E0F0B5044685B0A0B127
:1035E0000D4691B18AB1806A2649884218BF0720EA
:1035F0000CD104F1510630468DE80C0005F09EFE1A
:103600009DE80C0020B1082000E0012005B0F0BDCD
:10361000A16959B18F6802900390BF69086802A937
:10362000B8470299009A019B8A421AD2A17A84F87B
:103630004A300123994284F849306563A2632389A3
:1036400014D084F84430DB0903F00E0363F00F0359
:10365000032284F8453084F846202046FFF7F4FE24
:10366000D4E7304605F07AFE1720CFE75B0043F041
:103670000103002284F8461084F8443084F8452081
:10368000EBE700BF43494952F0B5044685B048B165
:103690000D4639B1806A2749884218BF072004D0F7
:1036A00005B0F0BD012005B0F0BD04F15106304673
:1036B0008DE80C0005F042FE9DE80C0008B10820E2
:1036C000EEE7616959B18F6802900390BF6908689D
:1036D00002A9B8470299009A019B8A421CD2A17A9A
:1036E00084F84A3001294FF000036563A263E26366
:1036F00084F8493015D0238984F84430DB0903F07D
:103700000E0363F00F03022284F8453084F846204C
:103710002046FFF799FEC3E7304605F01FFE17204D
:10372000BEE7227A84F84530530084F8461084F8C6
:103730004430EDE74349495230B583B0EFF303809D
:10374000103840B205F0CEFDEFF303836C4A103B16
:103750005BB2126852F833301C6894F84D30002B7D
:103760003BD1A36B012B04D9E26A137943F04003E8
:103770001371E36B012BE36A1A7942F010021A719C
:103780001A79C2F3001251D08DF804201A79C2F3CD
:1037900000128DF804201A79C2F300128DF804206B
:1037A0009DF804201A7922F008021A71A2692AB140
:1037B00094F8493013B1A36B032B4AD8E26A537AC9
:1037C0009906FCD5D37CDBB28DF8033001239DF83C
:1037D000032084F84D3003B030BD94F84E3003BB65
:1037E000E36B002BF7D0032B4FD0022B53D0012BD0
:1037F00040D0606B216CE26A537A9B06FCD5D37C87
:103800004354E36B012B05D1E26A137923F04003A3
:103810001371E36B226C013B0132E363226403B05A
:1038200030BD002384F84E3003B030BD8DF8052044
:103830001A79C2F300128DF805201A79C2F300122A
:103840008DF805209DF805201A7942F008021A71BA
:10385000ACE7916810684D68626B033B9BB2002136
:10386000A847A36B0321033B01222364E16384F88F
:103870004E20A3E794F84A2042B3E16A4A7842F026
:1038800004024A7084F84C30B3E7E26A137943F0DB
:1038900040031371ADE7E36A1A7942F010021A711E
:1038A0001A79C2F300128DF807201A79C2F30012B8
:1038B0008DF807201A79C2F300128DF807209DF8C1
:1038C00007201A7942F008021A7192E7E26A537AE5
:1038D00023F008035372E36A5A7842F008025A70E0
:1038E0005A78D2B28DF806205A78D2B28DF80620D6
:1038F0005B78DBB28DF806309DF8063079E700BFC3
:103900004CEB0000F8B5EFF30380103840B205F03F
:10391000E9FCEFF30383534A103B5BB2126852F8A1
:1039200033301C6894F84750002D3DD194F849304D
:1039300003F0FF0233B994F84F3023B1E36B84F8FE
:103940004F201BB1F8BDE36B002B49D194F8312017
:1039500053B2002B0DDB5B0920330121424802F0FA
:103960001F0201FA02F240F82320BFF34F8FBFF38A
:103970006F8F94F83250E66A6CB2204605F0B2FCC4
:10398000002C4BDB63099B0003F1604303F56143AB
:1039900005F01F050122AA40C3F88021F17941F00A
:1039A0004001F1711A60F8BD94F84630032B25D020
:1039B000012B94F8446004D994F848202ABB94F869
:1039C0004560012D34D0E36A9E7494F8482094F841
:1039D00047300132013B84F8482084F84730F8BD75
:1039E000226C616BE36A8A5C9A74226CE36B01322D
:1039F000013B2264E363002BA4D1A7E794F848209D
:103A0000022A10D094F84460D8E7022AD9D1032BB7
:103A100004BF94F8456046F00106D2E7F37943F01D
:103A20004003F3718EE794F850100029EAD1A0E723
:103A30006269002AC7D094F8493003F0FF07002BD1
:103A4000C1D1A36B002BBED093681068D3F804C01B
:103A5000616BA38F3A46E047A36BE76384F84F504E
:103A60002364B0E74CEB000000E100E010B582B049
:103A7000EFF30383444A103B5BB2126852F83330D1
:103A80001C6894F849301BB194F84730012B6FD073
:103A9000E36BB3B994F84A30002B48D1E36A5A7803
:103AA00042F008025A705A78D2B28DF807205A783C
:103AB000D2B28DF807205B78DBB28DF807309DF825
:103AC0000730E36A5A7A22F040025A72597AE06A61
:103AD00094F83220C1F380118DF80610597AC1F3A1
:103AE00080118DF806105B7AC3F380138DF80630D1
:103AF0009DF80630C17953B201F0BF01002BC171AE
:103B00000DDB5B0920330121204802F01F0201FA7E
:103B100002F240F82320BFF34F8FBFF36F8FEFF314
:103B20000380103840B205F0DDFB02B010BD94F9FF
:103B3000310005F0D7FB94F8312053B2002B09DB9C
:103B40005B09603302F01F020121104801FA02F202
:103B500040F82320E26A537843F004035370E26A8A
:103B60005379012123F00103537184F84C10A8E725
:103B700094F85020002A8BD1E16A4A7842F004027E
:103B80004A7084F850309CE74CEB000000E100E004
:103B900008B5EFF30383304A103B12685BB252F86A
:103BA00033301868C26A537A13F0010304D0537A91
:103BB00023F0010353720123517A890705D5517A05
:103BC00021F0020143F002035172517AC90605D572
:103BD000517A21F0100143F010035172517A4907D4
:103BE00005D5517A21F0040143F004035172517A52
:103BF00011F0080F05D0517A21F0080143F00803B5
:103C0000517213F0130F21D11A0718D5C36A5A7ACB
:103C100022F010025A725A7A22F008025A7290F870
:103C20004930002B14BF02210321FEF7C9FDEFF339
:103C30000380103840B2BDE8084005F053BB90F84F
:103C40004C20002AF3D05B07F1D5DFE7012380F891
:103C50004B30FEF779FEEAE74CEB000070B4104CF5
:103C60002368020A9A4216D26568C0B200F11006B3
:103C7000012355F8225003FA06F62E420BD069B103
:103C800000EB0210A36853F82030C3F34003002078
:103C90000B7070BC7047032070BC70471846FBE780
:103CA000A404FE1F084B1A68000A904201D30320A7
:103CB000704731B1DA684301043200209B580B8011
:103CC00070470120704700BFA404FE1F084B1A680C
:103CD000000A904201D30320704739B1DA684301EA
:103CE000043200209B581B0C0B807047012070474A
:103CF000A404FE1F144A1368F0B4040A9C421DD2A7
:103D00005768C5B205F11006012357F8244003FA9D
:103D100006F6264212D0A1B1D468000A043440014C
:103D200003FA05F2005992B202EA1040904213BF22
:103D3000002000200B700870F0BC70470320F0BC1E
:103D400070471846FBE700BFA404FE1F0C4B10B4DD
:103D50001C68000AA04200D21AB903205DF8044B87
:103D60007047DB685DF8044B083303EB401022EA30
:103D70000103114041EA034141600020704700BF48
:103D8000A404FE1F154BF0B41C68020AA2420AD21A
:103D90005E68C7B207F11005012456F8222004FA24
:103DA00005F5154202D10320F0BC70470129FAD86D
:103DB000DB6800F47F4003F1080303EBD00008D078
:103DC0004368BC4043EA0444240C240444600020BB
:103DD000EAE74468B9400C43A4B2F7E7A404FE1F25
:103DE00040B101230621022201704370C37082702A
:103DF0000020704701207047012901D90320704736
:103E0000114A1368F0B4040A9C4216D25768C5B22E
:103E100005F11006012357F8244003FA06F626425E
:103E20000BD000F47F40AB4051B91B04D268C008EE
:103E3000083219438150002000E00320F0BC704795
:103E400099B20023F2E700BFA404FE1F012901D9A3
:103E5000032070472C4BF0B51C68020AA2424ED2D8
:103E60005D68C0B200F11006012455F82250B4403C
:103E70002C4244D000EB02109C681D6954F820309D
:103E800000293ED043F00401204E0E40EFF310878E
:103E9000012383F310881E4B1A8892B222B94FF087
:103EA000400EEA7085F803E01A88013292B21A8057
:103EB00087F31088CF0354F8202007D5154F22F43C
:103EC00080320F4044F8202044F8207044F82060ED
:103ED000EFF31081012282F310881A880C4892B205
:103EE0001AB10288013A92B202801B889BB213B9C0
:103EF0008022EB70EA7081F310880020F0BD03206F
:103F0000F0BD23F00401BFE7A404FE1FD5FC011F90
:103F1000F804FE1FD5FC001F0AB9032070470B4BA5
:103F200010B41C68000AA04203D303205DF8044BC0
:103F30007047DB6822EA0104400108330A4042EA84
:103F40000442C2505DF8044B00207047A404FE1FD9
:103F50000AB9032070470D4B70B41C68000AA042D8
:103F600002D3032070BC70474001DD682E582B58E7
:103F700002EA01043443A4B261EA02021B0C2240AB
:103F80001B041A432A50002070BC7047A404FE1F73
:103F90002DE9F041002839D009681E4D002701EBBA
:103FA000C000B8464FF0010E8C88002335F813206E
:103FB000A24218D00133032BF8D108318142F3D14A
:103FC000FF43FFB2012005F079FA134A92F8BB349F
:103FD00048EA030808EA070782F8BB740120BDE835
:103FE000F04105F03BBA0A6802F0B852B2F1807FA6
:103FF00005D00EFA03F647EA0602D7B2DAE70EFA60
:1040000003F248EA02085FFA88F8D3E78046FF2700
:10401000D8E700BF94E4000000E0014070B582B032
:1040200002AB002403F8044D054618460E4604F082
:10403000A5FF9DF80430DB0702D4062002B070BD56
:10404000202D02D9032002B070BD012EFAD8084BF2
:104050001A69137805D02B4303F030032046137000
:10406000ECE703F0300323EA050520461570E5E789
:10407000A404FE1F002867D02DE9F84F4368002BE9
:104080005FD00146804631F8040BFFF781FFB8F896
:104090000030002B52D02D4CDFF8B4E0A1460022B6
:1040A00001204FF0400B4FF0800AD8F80430DEF8C2
:1040B000107053F83260DEF8085003EBC2039988A1
:1040C0000B0AC9B201EB0313EFF3108C80F31088D5
:1040D000218889B211B9F97087F803B021880131BC
:1040E00089B221808CF3108816F4803F55F8231094
:1040F00007D021F4803126F4803C45F8231045F8A0
:1041000023C045F82360EFF3108180F310882388E3
:104110009BB22BB1B9F80030013B9BB2A9F800303B
:1041200023889BB213B9FB7087F803A081F3108832
:104130000132B8F8003092B29342B6D80020BDE800
:10414000F88F0120BDE8F88F01207047F804FE1FAA
:10415000A404FE1F002832D04368002B2FD0F0B5F6
:1041600087B006AC002309210193164A04F8141DF8
:10417000154ED7680293054603930493059302A94D
:104180002046B8474FF00A0C029ABDF80C308DF863
:1041900004C002A9F2602046059A72603360B847F5
:1041A0000122029B8DF8052002A92046B360B84782
:1041B000029B33612846FFF75DFF07B0F0BD012089
:1041C000704700BF50E50000A404FE1F2DE9F04138
:1041D000304C2268050A954284B003460CD26268CE
:1041E000C6B20F464FF0010806F1100152F8252023
:1041F00008FA01F1114203D1032004B0BDE8F081B7
:1042000004A902AA41F80C2D4046ADF80C300297E3
:10421000ADF8008006EB0515FFF7BAFE2069A2682D
:10422000EFF3108488F310881B490B889BB213B9F5
:104230004026C370C6700B8801339BB20B8084F399
:104240001088FC0352F8253007D523F4803327F477
:10425000803442F8253042F8254042F82570EFF3CB
:104260001082012383F310880B880B4C9BB25BB93F
:104270000B889BB213B98021C370C17082F3108880
:10428000002004B0BDE8F0812388013B9BB223806D
:10429000EEE700BFA404FE1FF804FE1F00B583B0C4
:1042A000EFF303830C4A103B12685BB252F83330D1
:1042B0001B689A6832B102A8D9685B7C40F8081D77
:1042C00001939047EFF30380103840B205F00AF8ED
:1042D00003B05DF804FB00BF4CEB000038B183680D
:1042E0002BB1C168064A914203D0072070470120D4
:1042F0007047DA6A22F00102DA620020704700BFDC
:104300005450470038B183682BB1C168064A9142C6
:1043100003D00720704701207047DA6A42F001029B
:10432000DA620020704700BF5450470040B139B1F5
:1043300083682BB1C068054A904203D007207047BC
:10434000012070479B6C0B60002070475450470061
:1043500070B169B12DE9F041876882B057B1C26888
:104360001B4B9A4218BF072006D002B0BDE8F0816F
:10437000012070470120F8E77B6E0E4602A9002558
:104380000133B36041F8045DFA6A04461148C2F390
:1043900002688369032098474FEA4808012303FA1B
:1043A00008F2019BB3FBF2F373603B6B03F0010374
:1043B0003370FB6A13F0010F0CBF01232B463373DC
:1043C000237C03EB83035B00B6332846F381CCE701
:1043D00054504700F8E5000020B1034B1B68036010
:1043E0000020704701207047C4E40000FFFFFFFF7A
:1043F0002DE9F04782B002AC002544F8045D3C4D45
:104400008946AF6982469046214603201E464C46A7
:104410000025B847B8F1060F34D8DFE808F00F37A9
:104420004953575B040000214FF47A7202FB09F2F2
:104430000B46019807F09CFB04460D469AF8153090
:10444000012B07D000230A9A00201370346002B0B9
:10445000BDE8F0874FF6FF700021A94208BFA042D7
:104460004FF00003EFD2A208AF0842EA8572B942CA
:1044700003F1010308BF904214463D46DBB2E2D28D
:10448000052BF0D1032002B0BDE8F087019816A3F8
:10449000D3E90023A9FB000107F06AFB04460D469F
:1044A0009AF81530012BD5D04FF0FF300021D4E71A
:1044B0000198104A0023A9FB000107F059FB0446AC
:1044C0000D46EDE701984FF47A72F3E7019CA9FBE2
:1044D0000445E5E72B464A460198002107F048FBD2
:1044E00004460D46AAE700BF00CA9A3B0000000040
:1044F000F8E5000040420F00012A70B506461C4650
:104500002FD02AD3022A15D1A1FB0301194A002377
:10451000002507F02DFB012E0ED0A94208BFA042B6
:1045200015D0002908BFB0F1FF3F10D08D4208BF61
:1045300084420ED2032070BD14F1FF3245F1FF33E7
:10454000101A63EB01018D4208BF8442EED14FF097
:10455000FF30049B1860002070BD08460025002134
:10456000D9E7A1FB030164220023002507F000FB2B
:10457000D1E700BFA086010038B183682BB1214A82
:10458000C168914203D0072070470120704730B5C1
:10459000DA6A22F00102DA62017D4AB2002A83B0AF
:1045A0000DDB520920320124174D01F01F0104FADE
:1045B00001F145F82210BFF34F8FBFF36F8FDA8EF2
:1045C00022F48072DA869A8E044622F4807202A85F
:1045D00000252B219A860195237C00F8041DADF857
:1045E000063004F0F3FE94F91430657413F1210FD2
:1045F00004D0064A126852F833301D600020E06093
:1046000003B030BD5450470000E100E04CEB000027
:1046100038B183682BB1104BC2689A4203D007208F
:1046200070470120704730B4EFF31084012383F307
:1046300010888368DA6AD96A002021F00101D96202
:104640009864DD6A02F0010125F001020A43DA6292
:1046500084F3108830BC704754504700002838D08D
:1046600030B5856885B00346002D34D011B90320DC
:1046700005B030BDC568194CA54218BF0720F7D159
:104680001C460DF10B030025009303AB03958DF839
:104690000B50FFF7ADFE0028EAD1A368DA6AD96AA9
:1046A00021F00101D962D96A9DF80B4021F0E06147
:1046B00004F0070441EA0461D9620399013959669B
:1046C0009864D96A02F0010221F001010A43DA621A
:1046D000CEE7012070470120CAE700BF54504700D1
:1046E00040B3F0B5866885B036B3012B02D90320FC
:1046F00005B0F0BDC568224CA54218BF0720F7D110
:1047000004AF0446002047F8040D1D46736EA07DDB
:1047100000970133FFF7F0FE0028E9D1039AA36860
:1047200062B9A5B1196B21F0407141F000711046DA
:104730001963DDE7012070470120D9E7511C14D02F
:10474000196B65B121F0407119639A65D0E71A6B56
:1047500022F4403242F4003228461A63C8E721F4BA
:104760004031196328465A65C2E71A6B1DB142F001
:1047700040721A63BCE742F4403228461A63B7E736
:1047800054504700002966D0002864D02DE9F0413C
:10479000A84F8AB000230C460546487C04932B2181
:1047A000ADF812008DF81010FA688DF80B300393F5
:1047B000069307930893099304A806A99047064611
:1047C00010B10AB0BDE8F0810AAA069942F8140DAA
:1047D0003B69A96004A80621BDF81E809847BDF872
:1047E0001E309DF814202A755B075CBF01236B7592
:1047F0000DF10B0348BF6E756168227A009328465D
:1048000003ABFFF7F5FD0028DBD16369002B00F057
:10481000618195F91420213229D0A2696A602B6048
:10482000637C2B742278E369012A00F058811F7899
:104830009E781879A8750021022AAF74EE74697405
:1048400006910AD004A804F08DFD074688B108201F
:104850000AB0BDE8F0810120704706AEE168227C15
:10486000039B0096FFF748FE0028EBD0A9E70B203A
:10487000A7E7AE6804A804F0FDFCF16A4FEAD80887
:104880004FF0FF3321F001014FF4254E012028F0B5
:104890000102F162C6F800E0376177617761F76184
:1048A00037627762B762F76230637763B763F76343
:1048B0003764B764F36433657365B3657366B36671
:1048C000C6F88870C6F88C308AB17764F3663367AF
:1048D000F3677367C6F88030B367C6F88430C6F8EC
:1048E0009030C6F89430C6F89830C6F8A070AE681C
:1048F0000698F36A9DF80B10039A23F4E023F36201
:10490000336B43F002033363336B43F001033363D0
:10491000336B23F002033363F36A01F0070123F0E2
:10492000E06343EA0163013A0021F3627266B16415
:10493000E36933B11A78002A40F082809A78002A1D
:1049400036D16369002B00F0D480287D3A4AA37CDD
:10495000126841B20029C0F2B58001F160401B012C
:1049600000F56140DBB280F8003352F8313095F940
:1049700014001D6004F0B6FC2A7D53B2002B0DDB41
:104980005B099B0003F1604303F5614302F01F02E2
:10499000012101FA02F2C3F880211A60E37C1BB105
:1049A000F36A43F00103F362244BEB60002008E755
:1049B000AA68D978938E277801F0010E23F01003AE
:1049C00043EA0E139386938E01F0030E23F0C00387
:1049D00043EA8E139386938E012F43F00C03938644
:1049E00000F09180002F00F08980AB7D002B40F01B
:1049F000DB80938E23F0030343F001039386938EB1
:104A000023F00C0343F008039386136C23F4402334
:104A100043F480231364136B002840F0B78023F025
:104A2000407343F000731363938E43F48073938653
:104A300087E700BF50E500004CEB000054504700F2
:104A4000AA6893F801E0D78E94F800C00EF0010830
:104A500027F0100747EA0817D786D78E0EF003080D
:104A600027F0C00747EA8817D786D78EBCF1010F19
:104A700047F00C07D7866AD0BCF1000F62D0A97D41
:104A8000002940F09E80D18E21F0030141F0010108
:104A9000D186D18E21F00C0141F00801D186116C34
:104AA00021F4403141F480311164116B002874D13C
:104AB00021F4403141F400311163D18E41F4807111
:104AC000D1863BE7534F00F00F001B010744DBB2D8
:104AD0003B764AE72278012A7FF4A2AE99E618785D
:104AE00099786A741A79AA750023A874E9740693F0
:104AF000A8E62378012B7FF451AF26E7938E23F0AD
:104B00000303938690E700231365136C23F440237B
:104B100043F4802313646B7D012B0CBF4FF6FF73AE
:104B20004FF0FF339365938E23F00303002955D193
:104B300043F002039386938E23F00C0343F00403A7
:104B4000938671E7D18E21F00301D186B5E7D16458
:104B5000116C21F4403141F480311164697D0129E7
:104B60000CBF4FF6FF714FF0FF315165D18E21F030
:104B70000301BEF1000F3BD141F00201D186D18E7D
:104B800021F00C0141F00401D18696E7411C39D097
:104B900023F040731363906546E7471C36D021F439
:104BA00040311163506588E7938E23F0030343F08F
:104BB00002039386938E23F00C0343F00403938641
:104BC00023E7D18E21F0030141F00201D186D18E7D
:104BD00021F00C0141F00401D18660E743F00103AC
:104BE0009386938E23F00C0343F0080393861BE710
:104BF00041F00101D186D18E21F00C0141F0080174
:104C0000D1865AE743F0407313630DE741F4403116
:104C1000116352E7FCEC00E010B582B0EFF30383C0
:104C2000164A103B12685BB252F833301C68EFF33F
:104C30000380103840B204F055FBE4B1627CA368F5
:104C400082B1DA6A002122F00102DA629964A27C60
:104C500002B1D964E27C0AB100221A65DA6B22F053
:104C60004002DA63236833B16268009200228DF853
:104C700004206846984702B010BD00BF4CEB00000E
:104C8000024658B1064B07491B68002B08BF0B466C
:104C90000020596803EB81031360704701207047BF
:104CA000B804FE1FF4E6000088B10A4B1B6863B12C
:104CB0005A6800F1100103EB820353F8042F40F807
:104CC000042B8842F9D1002070471C207047012036
:104CD000704700BFB804FE1F70B36AB3174BF0B53E
:104CE0001E681EB3164B07781B68002404E00134CD
:104CF000B44203F1080319D09D79BD42F7D193F86E
:104D000005E04588B5EB9E0FF1D1DD7990F801E023
:104D100005F0070CF445EAD1B1EBD50FE7D19B883C
:104D20001470C3F3090353800020F0BDDF21FF237B
:104D3000117053800B20F0BD012070474405FE1F09
:104D40004CEB000020B1034B1B6803600020704750
:104D50000120704768E5000070B42A4C216851B109
:104D6000234604F57F70002201E053F8041F8342BC
:104D70000A44FAD11AB100BE1D2070BC7047224D02
:104D800022482A600368190CB1F5807F02D0002008
:104D900070BC7047196801390331F8D81C495E6A44
:104DA0008E42F4D12B6001686368486804EB83038A
:104DB00001EB800101F12300233301214FF47E45F3
:104DC00003E0013201310138013B25FA02F4E40726
:104DD00007D5072A10D0082A07D01E780478A642E3
:104DE000C9D11029EDD10020D2E70478372CE8D0C2
:104DF0001E78A642E5D0BEE706781C78A642E0D22F
:104E0000B9E700BFF4E60000B804FE1F9CB17F4084
:104E10005237465300285ED000295CD08B4B2DE9D9
:104E2000F0439A6890F800C003EB82029478A4459E
:104E300037D24FEA1C1802EB88060CF00F073589B1
:104E4000D2F804E025FA07F919F0010F29D0072F4D
:104E5000B67A09D902EB88080CF0070798F80BC05E
:104E60000CF00F0C66442D0ADFF8E481DFF8E4C192
:104E700018F80780754F08EA050524091CF8055045
:104E8000023402EB8402AC1902EB440532F8142020
:104E90006C78C2F30902250603EB820305D4002BCC
:104EA0004BD14FF4AF60BDE8F08317F8222045786E
:104EB0005208FDB14FF0020E012604271C78E407CA
:104EC00005F1FF3552D5052A00F2BE80DFE802F079
:104ED000332D211C1A05012070479A781EFB0264AD
:104EE000033204EB9202920013441A7854082246CB
:104EF000002DE3D1042A00F2A480DFE802F063630E
:104F000063503B000822EFE79A7817FB0262920099
:104F1000EAE793F804C09C7814FB0CF2D41C0CF163
:104F2000030204EB92029200DEE71A79033222F0C8
:104F300003020C32D8E70C22D6E74478B4B9DC7807
:104F4000C4F303144C72DC780125C4F303048C729F
:104F50008D804088002843D137F822200EEB0222B2
:104F60000A609B78CB800872C86015E040F27950E7
:104F7000BDE8F083DA78C2F303124A72DA78C2F33A
:104F800003028A725878C88000228A800A72CA6036
:104F90005B680B608307E9D50020BDE8F083DA7811
:104FA000C2F303124A72DA78C2F303028A725A78A1
:104FB000CA809A788A80043304200022CB60087269
:104FC0000A60E9E7DC78C4F303144C72DC78C4F3BC
:104FD00003048C721D79ACB28C804088844203D863
:104FE00040F27A50BDE8F083DC889E68012A04FB19
:104FF00000640C601CD0022A0AD09C785B780022E6
:1050000043EA0424CC800A72CA60002CE8D0C3E7CB
:105010001C18EA1C247BCC809D780D72920805FB3D
:10502000002003EB80030C33CB60002CD8D0B3E717
:10503000034400221C7BCC800A72CA60002CCFD0B3
:10504000AAE76420BDE8F08300224DE7F4E6000003
:10505000C8E40000D0E40000034B04301B6823F8D0
:1050600020100020704700BFFC04FE1F034B021DF0
:105070001B68002023F82200704700BFFC04FE1FBD
:10508000034B1A68137863F07F0313700020704796
:10509000FC04FE1F034B1A68137803F07F031370A0
:1050A00000207047FC04FE1F20B1034B1B68036007
:1050B000002070470120704788E5000060B101289A
:1050C00008D1094B1B680020402141221871197139
:1050D0001A71704701207047034B1B684021412221
:1050E000987099709A707047FC04FE1F002836D0A3
:1050F00070B51C4986B000230B22019302930393E1
:10510000049305930546CB688DF8042001A802A9F5
:105110009847044608B106B070BD134E029B336039
:1051200001A804F0A7F86B6873B130682346AA6839
:1051300012F8231002EB83020431528820F8212058
:105140006A6801339A42F2D828780028E3D032689E
:105150001378002063F07F03137006B070BD012048
:10516000704700BF50E50000FC04FE1F062070479A
:105170000620704790B10A4B02689A4201D007207E
:10518000704790F90630074AC033116851F8232060
:1051900022F0807241F823200020704701207047E0
:1051A000004354440005FE1F20B1034B1B680360FD
:1051B0000020704701207047B4E5000010B31A4B7F
:1051C00002689A4201D007207047D9B1174B1B687B
:1051D000DB8900229BB28A7190F9062018041AD448
:1051E000134B53F82230D87800F0C00080280BD041
:1051F000DB8940289BB28B8013D038B94FF48033C1
:105200000B607047012070479B898B804FF480733F
:105210000B60002070475BB2934204BF01238B7187
:10522000DEE7DBB28B80F1E7004354440405FE1F48
:105230000000FE1F0346F0B1114A0168914201D0FF
:105240000720704790F9062012F1210F15D030B4D5
:105250000C490D4D0C68C032002154F8220020F09A
:10526000807044F8220093F90620084645F8221081
:10527000196030BC7047012070470B20704700BF99
:10528000004354440005FE1F0000FE1F78B31D4B71
:1052900002689A4201D00720704790F9063013F156
:1052A000210F26D0184A52F823209168F9B151688D
:1052B000E9B1D17801F0300110291CD0202910D09B
:1052C000124AC033126852F8231021F4803142F898
:1052D000231052F8231041F0807142F8231000206F
:1052E00070479168890702D152689207E8D001207F
:1052F00070470B2070479168C907F8D45268D007EF
:10530000DED5F4E7004354440000FE1F0005FE1FF5
:105310002DE9F04182B001919DF820700092BDF816
:10532000245070B190F90640294A52F82410C978E7
:1053300001F0C001802903D0062002B0BDE8F08151
:105340001DB9012002B0BDE8F081002BF9D0214940
:1053500006688E4201D00720EFE71F4E1F49D6F89E
:1053600000E0D1F80080C0345EF8241021F0807194
:105370004EF8241098F8001021F0100188F8001061
:10538000019990F9064019B152F8246001997160B1
:10539000009919B152F824600099B16052F82410B4
:1053A000CC788D81CB818B7BCB7367F30514CC706C
:1053B000FFF76CFF98F80030002843F0100314BF8B
:1053C0001320002088F8003002B0BDE8F08100BF53
:1053D0000000FE1F004354440005FE1F0405FE1F8D
:1053E00000283AD0002938D00B68002B35D0DA7865
:1053F00012F0C00F04D0DB899BB2B3F5807F2CD8AC
:10540000514B02689A422AD02DE9F0474F4E33782B
:1054100086B08046894623B34D4B1D68B9F80460B9
:10542000002302E00133702B35D003F1C004DFB25A
:1054300055F82420C2F308029642F3D1454955F8A5
:10544000242051F82300C2F30802A8F80420002801
:1054500049D0082006B0BDE8F08701207047082039
:1054600070473D4901930822CC680293039304934B
:1054700005938DF8042001A80DEB0201A047002838
:10548000E8D1364D029B2B6001A803F06BFF074665
:1054900058B10A20DEE7D5F87C320B20C3F30803AD
:1054A000A8F8043006B0BDE8F087DFF8A8A001A88E
:1054B00003F0E0FE39464FF4E072504606F02CFE51
:1054C0002B68C3F804A01A7B062542F001021A7368
:1054D0008DF8045001A802A9A0471D4A029D15603D
:1054E000012333709AE7D9F8002000E01032D07819
:1054F00010F0C00F1CBF907BD073907810F0C00FDD
:10550000F4D1164A104D1468227822F0100222704D
:1055100099F80600D9F8002041F8232088F8067091
:10552000C8F8005020B9237843F01003237091E7A6
:105530004046FFF7ABFE2378002843F0100314BF6A
:1055400013200020237085E7004354440805FE1F04
:105550000005FE1F0000FE1F50E500000405FE1FB1
:10556000F0B583B001910092002851D090F9064027
:105570002A4951F82450EA7812F0C00206D1284A8C
:10558000056895420CD0072003B0F0BD13B9132075
:1055900003B0F0BD224E0768B742F4D1802A33D061
:1055A000204D214A2E681568C03456F8242022F078
:1055B000807246F824202A7822F010022A70019A7C
:1055C0004AB390F90620019E51F822406660009C83
:1055D0001CB151F82240009EA66051F82210CA78F2
:1055E00002F0C002802A0DD002B9CB81FFF74EFE37
:1055F0002B78002843F0100314BF132000202B70D9
:1056000003B0F0BD8B81F1E7EA8992B2002AC7D1DD
:10561000012003B0F0BD90F90620D8E70000FE1F7E
:10562000004354440005FE1F0405FE1F20B1034B38
:105630001B6803600020704701207047B8E5000038
:1056400018B10C230370002070470120704700BF81
:10565000A8B183790BB9072070470279036823F852
:10566000121042794AB902795AB91A7942F04002C5
:105670001A710123437100207047002070470120F8
:1056800070471A7962F07F021A71F2E7B0B183793C
:105690000BB907207047027903683AB11A7962F0B2
:1056A0007F021A7101234371002070471A7942F07A
:1056B00040021A7101234371002070470120704796
:1056C000B0B183790BB907207047027903683AB10A
:1056D0001A7902F07F021A7100234371184670474D
:1056E0001A7922F040021A7100234371184670475C
:1056F0000120704719B110B18B78012B01D901201D
:10570000704770B50C4686B03F49002321220193B3
:10571000054602930393049305938DF80420CB6808
:1057200001A802A9984750B9BDF80E30C3F3411340
:105730003BB1DBB222789A4205D340F27A5006B0F0
:1057400070BD0223F6E7029B2B602378ADF806308C
:1057500001A803F007FE0023ADF806300028EED1C3
:1057600001A803F087FD23782E68002B3CD1337904
:1057700023F0400333717379A27803F07F0302F0C2
:10578000010243EAC2137371B379627803F07F03B5
:1057900043EAC213B3712278E378FAB94BB3337A90
:1057A00043F0400333729DF8003006A86FF3000306
:1057B00000F8183D03F0DCFB9DF80030DB0705D551
:1057C000F37923F0070343F00103F37123782B717E
:1057D000012200236B711846AA71B0E773B1337AC6
:1057E00063F07F033372DEE7337903F07F033371B5
:1057F000C1E7337A23F040033372D4E7337A03F0FE
:105800007F033372CFE700BF50E5000028B38379F0
:105810000BB90720704730B50279036883B0BAB17D
:105820001A7902F07F021A7102AD0024212301943B
:1058300005F8043D8471037944712846ADF80630BB
:1058400003F014FD284603F0C1FD204603B030BD2F
:105850001A7922F040021A71E6E70120704700BF72
:10586000094A0A4B12680A48916910B4D469196050
:105870004FF400420021DC60586059619A601A615F
:105880005DF8044B704700BFD404FE1FBC04FE1F2C
:1058900000127A00374B1B6893F8283013F030025F
:1058A0003DD0102A0DD0202A3AD0DFED337A334A8A
:1058B000F0EE676A67EEA67AFCEEE77AC2ED057A4B
:1058C0007047028D2E4902F0030231F812100029B0
:1058D0004CD05B0610B44AD5038D13F0100F0CBFEB
:1058E00003240024254A038D52F824005DF8044B5C
:1058F00007EE900AB8EE677A07EE901AB8EE676A7C
:10590000C3F30523C7EE067A013306EE903AFAEEAA
:10591000EF6A67EEA67AFCEEE77AC2ED057A704789
:1059200090F82B30174A9B0932F813100029F6D053
:10593000124A90F82B30D2ED037A03F01F03B8EE31
:10594000677A06EE903A07EE901AF8EE666AB8EEBD
:10595000676AF7EE007A76EEA76AC7EE067A67EE18
:10596000A67AFCEEE77AC2ED057A70477047032409
:10597000B8E700BFD404FE1F00000000BC04FE1FF7
:10598000E0E50000D8E50000F8B50D4B1B680646C1
:1059900093F8205093F8217000200C4603F08EFD00
:1059A00096F81324E9B2BC400C4022EA010344EA11
:1059B000030186F813140020BDE8F84003F04EBD43
:1059C000D404FE1FF8B50D4B1B68064693F8225011
:1059D00093F8237000200C4603F070FD96F88124A4
:1059E000E9B2BC400C4022EA010344EA030186F814
:1059F00081140020BDE8F84003F030BDD404FE1F40
:105A000038B505460C46002003F058FD052C0AD891
:105A1000DFE804F019242F033A0E95F8323023F012
:105A2000010385F832300020BDE8384003F016BD90
:105A300095F82A3023F0010385F82A300020BDE8CC
:105A4000384003F00BBD95F8363023F0010385F89C
:105A500036300020BDE8384003F000BD95F83830FE
:105A600023F0010385F838300020BDE8384003F00A
:105A7000F5BC95F8903423F0010385F890340020AC
:105A8000BDE8384003F0EABC95F8803423F0010308
:105A900085F880340020BDE8384003F0DFBC00BF4B
:105AA00038B505460C46002003F008FD052C0AD841
:105AB000DFE804F019242F033A0E95F8323043F052
:105AC000010385F832300020BDE8384003F0C6BC41
:105AD00095F82A3043F0010385F82A300020BDE80C
:105AE000384003F0BBBC95F8363043F0010385F82D
:105AF00036300020BDE8384003F0B0BC95F83830AF
:105B000043F0010385F838300020BDE8384003F049
:105B1000A5BC95F8903443F0010385F8903400203B
:105B2000BDE8384003F09ABC95F8803443F0010397
:105B300085F880340020BDE8384003F08FBC00BFFA
:105B400003290ED0052907D009B10020704790F82D
:105B50003C0000F00100704790F83C00C0F340109A
:105B6000704790F83C00C0F3C0007047052937D853
:105B7000DFE801F011181F262D031A4B1B6893F85C
:105B8000283013F0300329D090F82A0000F00100EB
:105B900080F00100704790F8360000F0010080F0BE
:105BA0000100704790F8380000F0010080F001001B
:105BB000704790F8900400F0010080F001007047F9
:105BC00090F8320000F0010080F00100704790F87A
:105BD000800400F0010080F0010070471846704713
:105BE00000207047D404FE1F036A90F826307047E7
:105BF00038B5054600200C4603F060FC95F81334D8
:105C000004F0010123F0400343EA811185F81314E5
:105C10000020BDE8384003F021BC00BF38B5054680
:105C20000020144603F04AFC95F8A22004F00F046B
:105C300022F00F02144385F8A2400020BDE838404E
:105C400003F00CBC084B1B6893F8283013F0300F9E
:105C500004D104288CBF00200120704705288CBF88
:105C600000200120704700BFD404FE1F90F82600DA
:105C700000F00700704700BF38B5054600200C460D
:105C800003F01CFC95F8261004F0070421F007012E
:105C90000C4385F826400020BDE8384003F0DEBB09
:105CA000074B1B6893F828305B0601D4032070472C
:105CB000038D13F0100F0CBF03200020704700BFAE
:105CC000D404FE1F38B5044600200D4603F0F6FB51
:105CD000238D032D0CBF23F0100343F01003238505
:105CE0000020BDE8384003F0B9BB00BF38B5224CF6
:105CF0002DED028B236893F8283003F03003102B2E
:105D00000546B0EE408A1CD0202B02D0BDEC028BA1
:105D100038BD002003F0D2FBFCEEC87A95F82B10BA
:105D200017EE903A013B03F01F0221F01F031343CB
:105D300085F82B30BDEC028B0020BDE8384003F025
:105D40008DBB002003F0BAFB78EE087A2A8DFCEEBA
:105D5000E77A22F47C5217EE903A013B03F03F03BE
:105D600042EA03232B85002003F078FB236893F895
:105D7000283003F03003C7E7D404FE1F70B51E4C73
:105D8000236893F8283003F03003102B82B00546C7
:105D900019D0202B01D002B070BD184B002033F871
:105DA000114003F08BFB95F82B3004F0030403F053
:105DB0003F0343EA8413002085F82B3002B0BDE88E
:105DC000704003F04BBB0E4B0191002033F8116083
:105DD00003F074FB2B8D06F0030623F003031E4330
:105DE0002E85002003F03AFB2368019993F82830B0
:105DF00003F03003CDE700BFD404FE1FF0E5000040
:105E0000E8E5000038B51A4B1A6892F8293092F884
:105E10002A200546180748BF08784FF0000448BFFD
:105E200060F30E34D80644BF487860F30A2498061D
:105E300044BF887860F30614580644BFC87860F3FE
:105E40000204D20744BF0A7962F312441B0644BF1E
:105E50004B7963F31E748B79002063F31A6403F0AB
:105E60002DFB2C620020BDE8384003F0F7BA00BFDC
:105E7000D404FE1F036AC3F302330B70036AC3F337
:105E800002234B70036AC3F302138B70036A03F09F
:105E90000703CB70036AC3F302430B71036AC3F3B6
:105EA00002734B71036AC3F302638B71704700BFC7
:105EB000144B42781B6893F8241091421ED393F838
:105EC000262090ED017A07EE902AF8EE677AF4EE3C
:105ED000C77AF1EE10FA11D493F8253007EE903A14
:105EE000F8EE677AB4EEE77AF1EE10FA06D40078AD
:105EF000032805D0B0FA80F04009704700207047B1
:105F000001207047D404FE1F062921D8DFE801F0E4
:105F1000080C1014181C0400006AC0F302607047DB
:105F2000006AC0F302307047006AC0F30220704775
:105F3000006AC0F302107047006A00F00700704763
:105F4000006AC0F302407047006AC0F302707047F5
:105F50000020704710B50446FFF7D6FF94F82630AE
:105F6000034A03F0070352F8233023FA00F010BD70
:105F7000BC04FE1F024B53F82000C840704700BF0E
:105F8000BC04FE1F30B5044683B001200D4603F06B
:105F900095FA02A8002300F8013D02F099FE94F85A
:105FA000AA30D806FBD494F8A030D906F7D494F8D8
:105FB000AA3023F0010384F8AA3094F8AA30DA0654
:105FC000FBD494F8A030DB06F7D4042D2BD094F842
:105FD000A02005F0030322F00302134384F8A0304D
:105FE00094F8AA30D806FBD494F8A030D906F7D498
:105FF00094F8AA30042D0CBF43F0010323F00103F1
:1060000084F8AA3094F8AA30DA06FBD494F8A030C9
:10601000DB06F7D49DF8070002F06EFE012003F0C6
:106020001DFA03B030BD94F8A03043F0030384F8A8
:10603000A030D5E790F8AA30DB075ABF90F8A0004F
:1060400000F003000420704710B50446002003F060
:1060500035FA94F8403063F07F0384F8403094F8C8
:10606000403043F0010384F840300020BDE8104088
:1060700003F0F4B910B50446002003F01FFA94F8B9
:10608000403023F0010384F8403094F8403003F0AE
:106090007F0384F840300020BDE8104003F0DEB9F3
:1060A00090F84000C009704790F8410000F00100EE
:1060B000704700BF38B590F8413013F0010401D1AA
:1060C000002038BD0546002003F0F8F995F841306E
:1060D00023F0010385F84130002003F0BFF920468A
:1060E00038BD00BF38B5054600200C4603F0E6F980
:1060F00095F8301004F0010421F001010C4385F8FB
:1061000030400020BDE8384003F0A8B910B504467F
:10611000002003F0D3F994F8523043F0010384F8DF
:1061200052300020BDE8104003F098B910B5044685
:10613000002003F0C3F994F8523023F0010384F8EF
:1061400052300020BDE8104003F088B970B5044615
:1061500000200D46164603F0B1F994F83E3003F0E6
:106160007F0384F83E3094F83E3006F0070223F0B7
:10617000700343EA021284F83E2094F83E1005F0C2
:10618000070521F007010D4384F83E500020BDE8CB
:10619000704003F063B900BF10B50446002003F05F
:1061A0008DF994F83E3063F07F0384F83E30002090
:1061B000BDE8104003F052B910B50446002003F0CA
:1061C0007DF994F83E3003F07F0384F83E300020E0
:1061D000BDE8104003F042B910B50446002003F0BA
:1061E0006DF994F8533043F0010384F853300020E4
:1061F000BDE8104003F032B910B50446002003F0AA
:106200005DF994F8533023F0010384F853300020F3
:10621000BDE8104003F022B938B5054600200C4611
:1062200003F04CF995F8243004F0070123F07003D3
:1062300043EA011185F824100020BDE8384003F03E
:106240000DB900BF70B40F4B0F4C1D6800211960D1
:1062500094F823200138B0F1807FD2B20DD2F0261D
:10626000072502F0F002586084F8236099601D60F1
:1062700084F82320012070BC70471D60084670BC64
:10628000704700BF10E000E000ED00E090F85030F3
:1062900001F00F0123F00F03194380F850107047ED
:1062A00090F8500000F00F00704700BF90F8503099
:1062B00063F07F0380F85030704700BF90F8503093
:1062C00003F07F0380F85030704700BF90F8500013
:1062D000C009704790F8D13021B123F0010380F854
:1062E000D130704743F0010380F8D130704700BFD0
:1062F00090F8D13063F07F0380F8D130704700BF51
:1063000090F8D13003F07F0380F8D130704700BFA0
:1063100090F8D100C009704738B5054600200C46FA
:1063200003F0CCF895F8A51004F0070421F007015C
:106330000C4385F8A5400020BDE8384003F08EB836
:1063400020B1034B1B680360002070470120704799
:106350006CE6000030B52A4C87B0204602F014FEEF
:1063600006A8284B002503220095DB6800F8182DAD
:1063700002A90295039504950595984702986060D7
:106380004FF6FF7329460193FFF7F0FB28B910E0A1
:10639000019B43B1019B013B019360680021FFF722
:1063A000CFFB0028F4D0019B1BB94FF4CD7007B090
:1063B00030BD60680621FFF7AFFF4FF6FF73019312
:1063C000FFF74EFA60680421FFF76AFB04E0019BC7
:1063D00043B1019B013B019360680421FFF7C6FBB9
:1063E0000028F4D1019B002BDFD060680421052236
:1063F000FFF7FAFB60680021FFF7E4FA0020D6E718
:10640000D404FE1F50E5000070B169B170B5074EAD
:10641000044670680D46FFF729FC29462070706815
:10642000FFF728FD002070BD01207047D404FE1F37
:1064300070B582B0002940D0054600283AD0344CCF
:106440006068FFF7F7FD0428064633D060686946A8
:10645000FFF710FD23689A680AB1032E37D0DA6877
:10646000F2B1022E1CD193F829205969160733D4B2
:10647000D00638D496063BD450063ED4120603D537
:106480009DF805208A422BD393F82A30DB0703D5E9
:106490009DF804308B4223D39DF806308B421FD3E6
:1064A0002946012002F082FD6068FFF7CDFD002043
:1064B00002B070BD012002B070BD154D6868FFF7D5
:1064C000F3FD0446F0B14FF4CB7002B070BD93F809
:1064D000292019691007CBD59DF800008842C7D242
:1064E000052002B070BD9DF801008842C2D2F7E7D6
:1064F0009DF802008842BFD2F2E79DF8030088426F
:10650000BCD2EDE76868FFF7B5FD2046D3E700BFD2
:10651000D404FE1F38B5124C6068FFF7C5FD78B192
:106520006068FFF7A3FB236893F8283013F0300F5F
:10653000054603D05B0608D405280DD0032D0BD0EB
:106540006068FFF7B7FD002038BD6068FFF7A8FB63
:10655000052DF3D10328F3D140F2971038BD00BFC9
:10656000D404FE1F08B5034B01465868FFF7BAFD77
:10657000002008BDD404FE1F08B5034B5868FFF780
:10658000C5FD002008BD00BFD404FE1F08B5034BA5
:106590005868FFF7CBFD002008BD00BFD404FE1FE4
:1065A00008B5044B0A4601465868FFF7CFFD0020A6
:1065B00008BD00BFD404FE1F08B5034B5868FFF7A1
:1065C000EBFD002008BD00BFD404FE1F08B5034B3F
:1065D0005868FFF7F1FD002008BD00BFD404FE1F7E
:1065E00010B5114C2368606893F8283013F0300F11
:1065F00006D00521FFF7BAFA08B1002010BD606887
:106600000321FFF7B3FA0028F7D101466068FFF7CE
:10661000ADFA0028F1D160680121FFF7A7FA80F0F8
:106620000100C0B210BD00BFD404FE1F38B504463F
:10663000FFF708FB08B9032038BD631E012B11D9F1
:10664000042C0FD02CB1032C03D0052C01D000203A
:1066500038BD114D21466868FFF788FA78B94FF4C4
:10666000C87038BD0C4B21465868FFF77FFA40F2DE
:106670009113002814BF18464FF4C87038BD6868DD
:106680002146FFF75DFA40F2931300280CBF18462D
:106690004FF4C97038BD00BFD404FE1F70B5064664
:1066A0004FF6FE7440F2931501E0013C0CD03046E9
:1066B000FFF7BCFFA842F8D038B16FF4C873C31815
:1066C000022B38BF002070BD284670BD052814D0AD
:1066D00070B51F4D2B6893F8282012060C4612D473
:1066E0009A68944216D95B689C4200D970BD68686C
:1066F0000121BDE87040FFF745BC154B1A68526890
:10670000914212D97047FFF76BFFD8B92B689A688E
:106710009442E8D893F8283013F0300F09D1686814
:106720000321BDE87040FFF72DBC58680121FFF739
:1067300029BC6868064E0521FFF718FA0028EED03C
:106740003368D0E768680421BDE87040FFF71ABCE1
:10675000D404FE1FF0B583B00D460446FFF772FA6D
:1067600010B9032003B0F0BD5F4E052C21467068C0
:1067700006D0FFF7FBF9D0B140F2911003B0F0BDA5
:10678000FFF7F4F910BB3DB37068FFF76FFA052807
:10679000F2D02846FFF78CFB0028E2D070682978F9
:1067A000FFF7E4F900286CD14FF4CA70DAE770689B
:1067B000FFF740FC042811D0631E012B36D9042CAE
:1067C0003AD0A4B1032C1AD00020CBE77068FFF7B1
:1067D00061F840F29110C5E70120C3E7012C01D90F
:1067E000032CE9D170680321FFF7CCFBE4E7706864
:1067F0002146FFF7A5F9C8B140F29310B2E77068DF
:10680000394F2146FFF79CF905460028F4D13B6833
:10681000786893F82710FFF7B7F829467868FFF7EC
:10682000E7F9786821460522FFF7F8F970682146F4
:10683000FFF7E6F8002095E74FF6FF7321467068F2
:106840000193FFF793F9284B0146B0B1706804211A
:10685000FFF7D6F804E0019B43B1019B013B019394
:1068600070680421FFF782F90028F4D0019B002B07
:106870000CBF4FF4CD70002074E75868FFF7A2F802
:10688000E4E721467068FFF75BF90028B4D133686C
:1068900093F828305B0603D570682978FFF712FA61
:1068A00069787068104CFFF769FA95ED010A706815
:1068B000FFF71CFA7068FEF7EDFF336893F82810B5
:1068C000052001F00F01FFF755FB33685B68984224
:1068D00088BF0021606898BF0121FFF753FB7068F3
:1068E0000521FFF78DF86FE7D404FE1F70B582B065
:1068F0000446FFF7A7F910B9032002B070BD2E4D72
:106900006868FFF7B3F984421ED0052817D068687D
:106910000521FFF72BF990B9012C6868264E17D096
:106920002146FFF723F940B1022C26D0042C29D0B0
:10693000A4B1032C12D0052C10D00020DDE768682C
:10694000FFF7AEF9A042E7D140F2911002B070BD5E
:10695000FFF7A6FB58B140F29510CEE76868164DD8
:106960002146FFF7EDF840B940F29310C5E7706893
:106970002146FFF7FBF80028DFD068682146FFF7C3
:106980008FF8DAE770682146FFF78AF84FF6FF7351
:10699000019304E0019B43B1019B013B01936868B3
:1069A0000421FFF7E3F80028F4D1019B002B0CBF72
:1069B0004FF4CD700020A0E7D404FE1F01280FD0B3
:1069C000022801D00020704708B508460021FFF7D3
:1069D000C1FE40B140F29113984208BF002008BDAB
:1069E0000846FFF783BF002008BD00BF38B581B35C
:1069F00006282CD005281CD0042809D000B3012873
:106A000032D0022837D0032826D00323184638BDB9
:106A10001C4B1A6892F82A20D407F6D50D4600249C
:106A200001462C605868FFF795FA234628601846FF
:106A300038BD144B1A6892F829201506EED4E4E705
:106A4000104B1A6892F829201207E7D4DDE70D4BA6
:106A5000E4E70123184638BD0A4B1A6892F829204A
:106A60005206DBD40346D1E7064B1A6892F8292078
:106A7000D506D3D4C9E7034B1A6892F829209406A7
:106A8000CCD4C2E7D404FE1FF0B587B00C4605464F
:106A9000FFF7D8F810B9032007B0F0BD6CB3564E1D
:106AA000326892F82930190721D52778A079B842A1
:106AB000F1D861788F42EED894F803E0BE45EAD869
:106AC0008142E8D323F07F0303F0FF0113B1637920
:106AD0008342E0D392F82A30DB0702D52379834240
:106AE000D9D3042D0BD1002862D00520D4E76178DA
:106AF000E0788842CFD8A079E2E70120CCE770683F
:106B00003D4FFFF7B3F8854208D0002D47D0032D45
:106B100045D0052D43D06B1E012B60D97068364FD0
:106B20006946FFF7A7F970680021FFF72BFA0023E9
:106B3000A1798DF8083028468DF81430FFF71AFA3D
:106B4000062103907068FFF705FA049002A802F08E
:106B500057F90028A0D19DF80620A3799A4235D292
:106B600021467868FFF74EF978682946FFF784F8E0
:106B700006217068FFF7EEF90123049002A88DF852
:106B8000083002F03DF90446002885D102F028F9CA
:106B90001A4B0146186048BB4FF4C8707CE7706818
:106BA0002946FEF7CDFF0028B8D140F2931073E7D5
:106BB00063790BB1002998D170680F4FFFF770FA15
:106BC000002892D17868FFF751F8A7E7786829463E
:106BD000FFF752F878682146FFF714F9C8E778689C
:106BE0002946FEF7C3FF0028D6D097E72846FFF7CF
:106BF0006DFD204650E700BFD404FE1F6005FE1F58
:106C0000002800F086802DE9F047054686B006A8EA
:106C100000232F7800F8113D04A98DF810308DF86D
:106C200011308DF812308DF813308DF814308DF846
:106C300015308DF81630FFF7E7FB95F815E0EE7C80
:106C4000297DEA7DAB7D2C7E8DF808E038468DF8F5
:106C50000A608DF809108DF80B208DF80C308DF836
:106C60000D40FEF7EFFF18B9032006B0BDE8F0872E
:106C70002B7806AA134413F8103C012BF4D0022CF5
:106C800054D0DFF81081D8F8003093F8283013F092
:106C9000300F14BF06260526002440F2911905F195
:106CA000040A052CE1B25CD002AB185DFFF786FE4A
:106CB00008B14845D9D10134B442F2D13846FFF782
:106CC000EDFC0028D1D1052F25D0FFF789FC80F0FD
:106CD0000100C4B205F10C013846FFF7D5FE0028CB
:106CE000C3D19DF80750AF4210D006AB2B4413F828
:106CF000100C01282FD0D8F80400FEF7D1FF06AB06
:106D00000344014613F8100C012806D0DCB92046D4
:106D1000ABE7012070470446DCE7052DF6D18F4232
:106D2000F4D0FFF74BFE0028F0D09EE72879FEF75D
:106D300089FF002898D02B7906AA134413F8103C39
:106D4000012B9ED190E702F04BF801463846FFF741
:106D5000BDFC002089E72946FFF730FE0028CAD095
:106D600083E79DF80D30022B9ED128790021FFF793
:106D7000F1FC10B148457FF478AF2879FFF78EFC1D
:106D8000514600287FF471AF0520FFF7E3FC00288F
:106D900091D08EE7D404FE1F38B5114D2B6893F8BF
:106DA0002930DB0701D4062038BD002002F086FB25
:106DB00068680C4CFFF77AFA01E06CB1013C686836
:106DC000FFF784FA0028F8D0002002F047FB002CDF
:106DD0000CBF1420002038BD02F040FB142038BD49
:106DE000D404FE1FFFFF0F0038B5114D2B6893F838
:106DF0002930DB0701D4062038BD002002F05EFBFD
:106E000068680C4CFFF75AFA01E064B1013C68680D
:106E1000FFF75CFA0028F8D102F020FB002C0CBF31
:106E20001420002038BD204602F018FB142038BD85
:106E3000D404FE1FFFFF0F00F8B51B4D2B6893F81D
:106E40002930DB0701D40620F8BD184B1E5CFF2E4D
:106E500001D10320F8BD002002F030FB6868144C1B
:106E6000FFF734FA0746FFF7BFFF68683146FFF7C0
:106E70000DFA01E08CB1013C6868FFF711FA864217
:106E8000F8D13FB9002002F0E9FA002C0CBF142021
:106E90000020F8BDFFF780FFF4E7002FFAD1384655
:106EA00002F0DCFA1420F8BDD404FE1F64E60000F2
:106EB000FFFF0F0010B5094C236893F82A309B0799
:106EC00001D4062010BD002002F0F8FA6068FFF738
:106ED0000FFA002002F0C2FA002010BDD404FE1FF9
:106EE00010B5094C236893F82A309B0701D406207B
:106EF00010BD002002F0E2FA6068FFF701FA0020FE
:106F000002F0ACFA002010BDD404FE1F70B5124C84
:106F1000236893F82A309B0701D4062070BD03280C
:106F200002D008B1032070BD0546002002F0C6FA69
:106F30006068FFF7EDF90646FFF7D2FF6068294663
:106F4000FFF7C8F926B9002002F088FA002070BDCA
:106F5000FFF7B0FFF7E700BFD404FE1F08B5064BEC
:106F60001A6892F82920920701D4062008BD5868B3
:106F7000FFF732F9002008BDD404FE1F08B5064B08
:106F80001A6892F82920920701D4062008BD586893
:106F9000FFF732F9002008BDD404FE1F08B5074BE7
:106FA0001A6892F82920520701D4032008BD01462F
:106FB0005868FFF731F9002008BD00BFD404FE1F58
:106FC00008B90320704738B50D46044601F008FFA4
:106FD00007EE900AF8EE676AF7EE007AC7EEA66A47
:106FE00007EE905A07EE104AF8EE677AB8EE477A45
:106FF00066EEA77AC7EE277AFCEEE77A17EE900ADC
:10700000FFF720F900280CBF1220002038BD00BF78
:1070100038B5B0F8403823F48063A0F84038B0F8B1
:10702000403823F44073A0F84038B0F8423803F4F5
:10703000E063054673B141F2873401E0013C09D0B9
:107040000120014602F022F9B5F8423803F4E0636A
:10705000002BF3D1B5F8420800F4E060B0FA80F0FC
:10706000400938BD38B5B0F8403823F48063A0F843
:107070004038B0F8403823F4407343F40073A0F86C
:107080004038B0F8423803F4E063B3F5007F0546BA
:107090000FD041F2873401E0013C0AD001200146C3
:1070A00002F0F4F8B5F8423803F4E063B3F5007F7A
:1070B000F2D1B5F8420800F4E060A0F50070B0FA33
:1070C00080F0400938BD00BF38B5044607290AD80A
:1070D000DFE801F00C171F436E63A304FFF7C2FF44
:1070E000002840F0A6804EF6612038BD002380F8CD
:1070F0005838FFF78DFF00284EF6612018BF00209A
:1071000038BDFFF7AFFF00284EF6612018BF002002
:1071100038BDFFF7A7FFB4F8403843F48063A4F804
:107120004038B4F842385D0558BF41F2873502D582
:1071300009E0013D07D00120014602F0A7F8B4F8AC
:1071400042385805F5D5B4F84208C0F3802000282D
:107150004EF6612018BF002038BDB0F8403823F447
:107160008063A0F84038B0F84238590548BF41F272
:10717000873502D409E0013D07D00120014602F025
:1071800085F8B4F842385B05F5D4B4F842385A05AE
:10719000A9D42046FFF73CFFADE7FFF763FF0028C7
:1071A000A1D0032384F858382046FFF731FFA2E727
:1071B000B0F8403823F48063A0F84038B0F8403885
:1071C00023F4407343F48073A0F84038B0F8423899
:1071D00003F4E063B3F5807F18BF41F2873502D135
:1071E0000CE0013D0AD00120014602F04FF8B4F84E
:1071F000423803F4E063B3F5807FF2D1B4F842087B
:1072000000F4E060A0F58070B0FA80F0400900283A
:107210004EF6612018BF002038BDFFF723FF00287D
:107220003FF461AF072384F858382046FFF7F0FE9B
:1072300061E7052384F85838ABE700BF2DE9F04734
:1072400000294BD00024A04616464FF0400C2BE0FE
:1072500050F80A7027F0FF5952F8347029F4E019F9
:10726000C7F30A0749EA874740F80A702D014759D2
:1072700027F00047475196F80590475909F0010952
:1072800027F0804747EA897747518EF820C8377939
:10729000012F08BF051904F1010408BF85F82088F3
:1072A0008C4206F1080617D0377900EB040E002F48
:1072B000EED104F120054FEA051A8EF82078002B54
:1072C000C6D052F8347004F120054FEA051927F0B2
:1072D000604740F80970C9E71F2906D80022431803
:1072E0000131202983F82028F9D1BDE8F08700BFBB
:1072F000890831D02DE9F0474FF0000EDFF86480A7
:10730000043A74460F266FF0604912E040F82C9062
:1073100050F82C7027F0FF5525F4E01545EA8A4512
:1073200040F82C504EEA060E01348C424FEA061605
:107330000CD052F8045F4545F6D804F5807CC5F3BF
:107340000A0A002BE2D040F82C50EBE76FEA0E035C
:10735000C0F82834BDE8F0874FF0FF33C0F8283478
:10736000704700BFFEFFFF1F38B5B0F8403843F04C
:107370002003A0F84038B0F840389A0605460CD5EE
:1073800041F2873401E0013C07D00120014601F0C1
:107390007DFFB5F840389B06F5D4B5F84008C0F33A
:1073A000401080F0010038BD70B50646D0F84408A2
:1073B00082B0002310F0010401930D4616D011494C
:1073C000D6F84438D6F84428D6F84408C2F3022246
:1073D00002EB1373C0F30942012003330132B1FB06
:1073E000F2F2B2FBF3F32B6002B070BD064B01204A
:1073F0009B6901A9984708B90199E1E7204602B0C5
:1074000070BD00BF00127A00F8E5000070B40025DE
:107410002C462E4605F120031B01C218C450537997
:1074200023F00F03537100EB05110023CA18013339
:10743000082B82F80642F9D10135202DA1F80E6201
:10744000E8D170BC704700BF014491F8200880F07B
:107450004000C0F38010704770B401F12004260191
:107460008559C5F380755D7302BB8259C2F38A42A8
:1074700000EB04141A60657905F00F05082D28BF8C
:1074800008251D7165B10433002200EB0116B41804
:1074900004F500740132A47903F8014FAA42F6D131
:1074A0000144402381F8203870BC70478259DFE7DF
:1074B000F0B5002B3FD101F1200E4FEA0E151468F4
:1074C000435923F0FF5323F4E013C4F30A0443EABF
:1074D0008443435100EB0E1513796E7903F00F04CA
:1074E00026F00F0323436B71137963B1151D00233D
:1074F00000EB0117FC1815F8016F84F80662147987
:1075000001339C42F6D84FEA0E1E527B50F80E30E3
:1075100002F0010223F08043014443EA827340F801
:107520000E30002381F8203891F8203863F07F0373
:1075300081F82038F0BD136801F1200E4FEA0E14D7
:1075400023F060430351C5E790F84D38DBB20B6080
:1075500013B1002380F84D38704700BF30B5B0F844
:1075600042280C4692B283B003464FF0000500203B
:1075700060F3C705D1B262600190A571CD0708D54F
:1075800083F8530893F85208A279217960F3C7026F
:10759000A271E2796FF30402E271CA0608D50222F1
:1075A00083F8532893F85218E27961F30402E271E8
:1075B00093F85828A179A2F10302B2FA82F2520993
:1075C00062F30001A17193F85828C9B2A2F1070231
:1075D000B2FA82F2520962F38201A17193F858283B
:1075E000C9B2A2F10502B2FA82F2520962F3410174
:1075F000A17193F84E28627393F84F28227393F881
:107600005028D2B282F07F012261184683F85018C8
:1076100001A9FFF7C9FE10B1019BA360012003B0CF
:1076200030BD00BFB0F8423890F84D28C3F3C01306
:107630001AB1002380F84D38012390F850285206E3
:1076400003D0002380F8503801231846704700BF4C
:1076500020B1034B1B680360002070470120704776
:107660008CE6000038B590F82430056A044658B21C
:1076700010F1210F22D000280FDB40092030012219
:107680003A4903F01F0302FA03F341F82030BFF335
:107690004F8FBFF36F8F94F9240001F023FE94F80D
:1076A000242053B2002B09DB5B09603302F01F0278
:1076B00001212E4801FA02F240F8232094F82530E7
:1076C00058B210F1210F22D000280FDB40092030E2
:1076D0000122264903F01F0302FA03F341F8203088
:1076E000BFF34F8FBFF36F8F94F9250001F0FAFDC0
:1076F00094F8252053B2002B09DB5B09603302F0BC
:107700001F020121194801FA02F240F8232094F8DF
:10771000263058B210F1210F22D000280FDB40098B
:1077200020300122114903F01F0302FA03F341F84C
:107730002030BFF34F8FBFF36F8F94F9260001F015
:10774000D1FD94F8262053B2002B09DB5B0960338E
:1077500002F01F020121054801FA02F240F823203D
:10776000002385F84C38C5F82C3438BD00E100E022
:107770002DE9F04F8BB00AAB002223F8242D0C46E4
:1077800005461846039201F0E9FB276A002D7AD0DE
:10779000002F78D0A369002B75D0E368202B05D982
:1077A0004EF6622420460BB0BDE8F08F9A07F7D161
:1077B000B549686888426BD09B080FD07968086823
:1077C000B0F1005FECD201EB8303043104E051F827
:1077D000040BB0F1005FE3D29942F8D1616800294F
:1077E00051D00B68013BB3F5806FD9D24B79087942
:1077F0009842D5D989799942D2D80DF1280B002326
:107800004BF8143DA14E04935946BDF80430D6F808
:107810001890ADF8083001209DF805A0C84780BB3E
:107820009DF8088018F0020F47D118F0010838D1F0
:107830003B78012B35D00AA80DF1180900F8258DE9
:10784000494673699847E0B99DF80330052BA7D1E5
:107850002368DFF84082ADF80E30302000238DF829
:107860000C00D8F80C208DF80D304946069307938C
:107870000893099303A89047DDF818A0C5F820A045
:1078800040B104468EE7012420460BB0BDE8F08FDE
:10789000082487E703A801F065FD0746D0B10A2454
:1078A00080E76368059A1968794BB3FBF1F393425B
:1078B0003FF676AF0DF11809CAE7504604A9C8474C
:1078C0000028DED1049B0599B3FBF1F3022B7FF472
:1078D00067AFAAE703A801F0CDFC8AF84C78BDF8A1
:1078E00004E0CAF82C742068E368A169E26994F89E
:1078F00008C0EB601EF0010F236A2860207DADF800
:1079000010E0A961EA6185F809C028752F7218D0C6
:107910000123D4F804A02F6A6B75F36903209847FC
:10792000B0F5C97F14D098B104462846FFF79AFEF7
:1079300003A801F09BFC03A801F048FD00236B6045
:1079400030E71B786B75012BD4F804A02F6AE4D0C4
:1079500038460421FFF7B8FB0028E5D1B7F84038D6
:1079600023F4C053A7F84038B7F8403823F0010398
:10797000A7F84038B7F840386A7A23F0060302F0D7
:10798000030243EA4203A7F84038B7F840382A7D9B
:1079900023F0080302F0010243EAC203A7F84038CB
:1079A000B7F8403823F01003A7F84038B7F840384C
:1079B00043F0C003A7F84038D7F84438DAF800207D
:1079C00023F07F73013A02F03F0223F4403343EA8D
:1079D0000243C7F84438D7F844389AF8042023F013
:1079E000704343EA0273C7F84438D7F844389AF82A
:1079F000052023F4E06302F0070243EA0223C7F8FC
:107A00004438D7F844389AF8062023F4405302F05B
:107A1000030243EA0233C7F844386B7DD7F84428A1
:107A200003F0010322F001021343C7F8443838463B
:107A30000121FFF749FB0646002840F0E280D5F817
:107A40002090276A4846FFF7E1FC802389F85038E8
:107A5000E1682269237A4846FFF7F0FB48467A68D6
:107A6000E168237AFFF744FC2F6A31463846FFF776
:107A70002BFB00287FF458AF3846FFF775FC58B948
:107A80004EF6622451E700BF4E414352F8E5000034
:107A900000127A0050E500003846FFF7C3FD0146AA
:107AA0000028EDD10590D8F810802E6A03A85A4618
:107AB000C0479DF8140085F8240041B211F1210F50
:107AC00021D0514A94F8243017680029C0F28180EF
:107AD00001F160401B0100F56140DBB280F800332A
:107AE00095F8240057F8312043B2002B156007DBCE
:107AF00000F01F005B0901224449824041F8232025
:107B00003E2386F84C3803A803215A46C0479DF807
:107B1000143085F8253058B210F1210F1ED03A49A3
:107B200094F825200F6800285BDB00F1604E1301FC
:107B30000EF5614EDBB28EF8003395F8252057F82C
:107B4000301053B2002B0D6008DB02F01F025B09FE
:107B500001212E4801FA02F240F8232003A85A46D8
:107B60000421C0479DF8143085F8263058B210F132
:107B7000210F1ED0244994F826200968002838DBFC
:107B800000F16044130104F56144DBB284F8003372
:107B900095F8262051F8301053B2002B0D6008DB09
:107BA00002F01F025B090121184801FA02F240F8B5
:107BB00023206B6A164A23F07F4323F0FF0393428E
:107BC0001CBF4FF0FF33C6F82C34124B6B600024FF
:107BD000E8E5114A00F00F001B010244DBB2137606
:107BE0007EE70D4903F00F0319441201D3B20B765F
:107BF000A3E7094C03F00F031C441201D3B2237610
:107C0000C6E7044691E600BF4CEB000000E100E04F
:107C100000DFDF004E414352FCEC00E038B132B1EE
:107C200038B50B4B44689C4203D0072038BD012077
:107C30007047012918BF032000D038BD15780446CD
:107C40002946006AFFF740FA0028F6D1257238BDB0
:107C50004E41435228B10F4A4168914203D0072058
:107C600070470120704710B5002482B0026844605C
:107C700030230194ADF806208DF80430FFF7F2FCB4
:107C800001A801F0F3FA01A801F0A0FB204602B020
:107C900010BD00BF4E41435238B132B1F8B5294B47
:107CA00044689C4203D00720F8BD01207047076A52
:107CB000044638460E461546FFF7C6FB10B14EF691
:107CC0006520F8BDBB1993F82028D00727D593F875
:107CD0002038990723D42B46627A38463146FFF77D
:107CE000BBFB236AB3F84228D20602D5217D0129C5
:107CF0001AD0B3F8423813F0010313D094F82520BA
:107D000053B2002B0EDB5B09403301210E4802F019
:107D10001F0201FA02F240F823200020F8BD4EF6BF
:107D20006020F8BD0020F8BD94F8240042B2002A7B
:107D3000DFDB5209403200F01F00034D814045F85F
:107D40002210D6E74E41435200E100E050B14AB163
:107D5000F0B51C4C4568076AA54283B004D00720E3
:107D600003B0F0BD012070471F2902D9032003B0E2
:107D7000F0BD0546384601920E46FFF765FB012827
:107D8000019A02D04EF66420EAE71379082BEDD869
:107D9000286A831993F82018C90907D093F8201886
:107DA000C90703D44EF6632003B0F0BD002483F866
:107DB000204883F8204831466B7AFFF779FB20464C
:107DC00003B0F0BD4E41435238B138B539B10B4A1A
:107DD0004468944205D0072038BD01207047012037
:107DE00038BD0446006A0D46FFF7B8FB10B94EF6E1
:107DF000602038BD237A2B70002038BD4E4143529D
:107E000070B586B0EFF30380103840B201F06AFA23
:107E1000EFF303832E4A103B5BB2126852F8333003
:107E20001D68FDB12E6AEEB106A90024304641F866
:107E3000144D0294039404940594FFF785FB9DF878
:107E4000042002F0080303F0FF006BB102238DF859
:107E50000C30AB6933B12968EA6902910592049448
:107E600002A8984706B070BD02F0100101F0FF03B0
:107E700049B902F0040101F0FF0449B104221C4693
:107E80008DF80C20E5E7032304468DF80C30E0E77D
:107E9000910718D4930606D42B6AB3F84248C4F36A
:107EA0000014002CD5D006238DF80C30022296F851
:107EB000533886F8532896F85248DBB204F01F0472
:107EC00086F85338C5E705238DF80C30C1E700BFAD
:107ED0004CEB000010B584B0EFF30380103840B2D3
:107EE00001F000FAEFF30383114A103B5BB2126812
:107EF00052F833301B68CBB11A6ABAB19969A9B18B
:107F000092F85308002482F8534892F85218C0B2ED
:107F100082F853081868009001F01F02D969029294
:107F20008DF8044003919B696846984704B010BDE2
:107F30004CEB000030B585B0EFF30380103840B251
:107F400001F0D0F9EFF303831F4A103B5BB21268D4
:107F500052F833301C68002C33D0236A8BB3A269EB
:107F6000E2B1012093F8531883F8530893F852288C
:107F70008DF8040002F01F029818C9B2002583F89A
:107F8000531880F8205880F820582168E36903933B
:107F90000292A369009168469847236AB3F8423871
:107FA0009B070ED594F8262053B2002B09DB5B0902
:107FB000403302F01F020121044801FA02F240F8A6
:107FC000232005B030BD00BF4CEB000000E100E015
:107FD00020B1034B1B6803600020704701207047ED
:107FE000C4E6000006207047E8B110B584B0002355
:107FF00004466846009301930293039300F096FFB2
:108000009DF80C30990702D4062004B010BDE36936
:108010001A88120409D41B8813F4007F0CBF0020B7
:108020001B2004B010BD012070471B2004B010BD00
:1080300088B1104B826A9A4201D007207047C36909
:108040004BB190F82420022A07D01A8842F400721B
:108050001A8000207047012070471888C0F3C03094
:1080600030B91A886FEA42426FEA52421A8070476A
:10807000082070474344415298B10B4B826A9A42A0
:1080800001D007207047C3695BB190F82420022A11
:108090001A8814BF22F40072C2F30E021A80002064
:1080A00070470120704700BF4344415270B1084BF4
:1080B000826A9A4201D007207047C36933B11B8896
:1080C00013F4004F0CBF00200820704701207047B8
:1080D00043444152D0B1CB1CDBB21E2B01D903204B
:1080E0007047002930B40ADB104C0588012354F88E
:1080F00025408B40234202D1032030BC70470C4BFB
:10810000846A9C4204D0072030BC7047012070472D
:108110003AB1C3693BB11031002033F811301380FC
:10812000EBE70220E9E70120E7E700BF0C05FE1FAF
:108130004344415230B583B00023ADF806309AB1C4
:1081400014460DF106020546FFF7C4FFBDF80630E0
:1081500010B1236003B030BDEA88B2F5004F06D0FD
:108160000020236003B030BD022003B030BD1B04EB
:10817000F6E700BF30B129B1144B826A9A4203D0AE
:1081800007207047012070470B78DA1CD2B2122A00
:1081900016D85BB2002B30B407DB0D4C05880122EA
:1081A00054F825409A4022420CD04A78062A09D930
:1081B000C16949B10B44002083F8E02030BC70470E
:1081C000032070470320F9E70120F7E743444152B9
:1081D0000C05FE1F30B129B13A4B826A9A4203D096
:1081E00007207047012070470379012B56D0F0B566
:1081F000C76983B0002F62D0C46A002C50D04FF002
:10820000FF330122013302FA03F52542FAD0B5F11A
:10821000805F51D0B5F1005F08BF6FF001031033EC
:1082200007EB43030B6020220126013A06FA02F510
:108230002542FAD0B5F1805F3BD0B5F1005F08BFB1
:108240006FF00102103207EB4202D31A5B100133C8
:108250004B60054602A800230C4620221A4E0193CB
:10826000012100F8042D2A8800932172ADF8062020
:10827000336902216A46984770B92B78BDF802200D
:10828000628104335B004FF0FF326372E260EB7A8D
:10829000012B07D06B88238203B0F0BD0320704709
:1082A0004C60D6E76A695178137843EA0123E360AA
:1082B000F0E76FF00202C5E76FF00203AFE70120BD
:1082C000EAE700BF4344415250E5000030B5B0F842
:1082D000803023F00103A0F880300388C3F34133DA
:1082E000012B038A43F47C5383B00D4603821CD0D8
:1082F00000240480448220232A88009468468DF854
:108300000030ADF8022000F0B1FFEB6ADB000AD5C7
:108310002B6903B11C7002A800222223019200F8ED
:10832000043D00F0A3FF03B030BD038A43F03F03D8
:108330000382DDE7002877D03C4B826A9A4201D065
:1083400007207047C369002B6ED030B590F83030ED
:10835000044658B2002210F1210F83B0A26225D04A
:10836000904219DB400920300121314D03F01F03F9
:1083700001FA03F345F82030BFF34F8FBFF36F8F3F
:1083800094F8303058B2904206DB420903F01F03E4
:108390006032994045F8221000F0A4FF254B94F973
:1083A00030201B6853F8323000221A6094F83130C4
:1083B00058B210F1210F25D0002819DB40092030D8
:1083C00001211B4D03F01F0301FA03F345F8203090
:1083D000BFF34F8FBFF36F8F94F8313058B200283E
:1083E00006DB420903F01F036032994045F8221072
:1083F00000F078FF0F4B94F931201B6853F83230AE
:1084000000221A60E0692146FFF760FF02A80025FC
:108410002023019500F8043D2388ADF8063000F0D4
:10842000D5FF284603B030BD012070474344415278
:1084300000E100E04CEB000030B129B1AA4B826AA8
:108440009A4203D007207047012070472DE9F04180
:10845000C66986B05EB30D46A44A01882B6852F8FF
:108460002120044623B90320E36206B0BDE8F08171
:1084700042F04052D2431A42F5D13188C1F3413122
:10848000012916D06A68002AEDD1002302A80293C0
:1084900003930493059300F049FD9DF8082093078A
:1084A0000ED46B6813F0405F0AD02B68DBE7012025
:1084B000DBE769680029D6D01A430A42D3D1E4E742
:1084C0002B6813F0405109D030880706CBD45007F1
:1084D00000F1718196F87A20002AC4D1327B5207CC
:1084E00000F064816A68E9681A4331EA0202BAD18D
:1084F0000029B8D02A7C002A40F06B819BB2B3805F
:10850000AB88B382AB8933816B88F380EB88F382CD
:10851000EB8973812B6813F0405F03D16B6813F014
:10852000405F66D0002302A802930393049305934F
:10853000019300F0FBFC6E4B9DF810009B6901A9B4
:108540009847019B6B4A934202D803202B688BE724
:108550000028FAD16849039A684FA1FB03139B0CCA
:1085600002FB03F3A7FB0337BF09FB1FF82BECD873
:108570002B68DA0002D46A68D2001CD5FBB286F8F8
:10858000DE30A37A012B00F0F3802B6813F0805FBC
:10859000738A00F0B58043F480737382738A23F486
:1085A00080637382EB68728AC3F3007322F0010266
:1085B000134373822B68980002D46B68990018D516
:1085C000FFB286F8DF702B6813F0005F738A00F04B
:1085D000828043F400737382738A23F4006373828E
:1085E000EA68738AC2F3407223F0020343EA42034B
:1085F00073822B7C6A7C03F0030342EA4323A6F8D0
:1086000066302B8948F2010293422ED0A6F88030C2
:108610002379D4F81C80022B1FD0B8F80070C7F360
:108620004137012F2BD094F9300010F1210F14D0D5
:1086300000F058FE94F8302053B2002B0DDB5B099C
:108640009B0003F1604303F5614302F01F02012127
:1086500001FA02F2C3F880211A602A8948F2010364
:108660009A4207D02B680020FEE62379D4F81C80BC
:10867000022BD2D148F20103A6F88030F2E72A8912
:1086800048F201039A4243D094F9310010F1210FCE
:1086900012D000F027FE94F8312053B2002B0BDBF0
:1086A0005B099B0003F1604303F5614302F01F0285
:1086B0009740C3F880711F60B8F8003043F0400362
:1086C000A8F80030B8F8103023F03F0343F00A0355
:1086D000A8F81030A7E723F400737382738A43F479
:1086E000006373827CE700BF434441520C05FE1FC8
:1086F000F8E500003F420F0083DE1B43D34D6210BC
:1087000023F480737382738A43F48063738249E72E
:10871000B8F8103043F03F03A8F8103094F8312037
:1087200050B210F1210F1CD0002818DB4309203370
:10873000444902F01F0207FA02F241F82320BFF376
:108740004F8FBFF36F8F94F8312050B2002806DBB3
:10875000430902F01F026033974041F8237000F094
:10876000C1FDB8F8003023F04003A8F800305AE704
:108770003548002322220193029303930493059327
:1087800002A9C3688DF8042001A8984700287FF447
:10879000DDAE01A800F06EFD23691A7862F07F0259
:1087A0001A701A7842F010021A70EEE6EA68002A8F
:1087B0007FF459AE9EE6B1F1405F3FF454AE23F032
:1087C0007042002A7FF44FAE2279002A7FF44BAE2C
:1087D00084E60021102202A803F09EFC02A800F00B
:1087E000A5FB9DF80830DB077FF55FAE2A7C072AE2
:1087F0003FF65BAE6B7C032B7FF657AE37882B685A
:108800006968C7F34137012F02EA030001EA020158
:108810000DD082427FF427AE328817060DD400298E
:108820003FF46CAE2A89002A7FF41DAE66E68242D0
:10883000F2D08A427FF417AEEEE700287FF413AE41
:10884000EDE700BF00E100E050E50000002838D06F
:10885000002936D0F0B58B888E78C3F30E038DB027
:1088600013B103200DB0F0BD0C46054608A80893CF
:1088700009930A930B9300F059FBA37933B19DF848
:108880002C20D70740F17C81852BEAD0E27912F0C9
:10889000DF0FE6D1277AA278022FE2D8022AE0D8A9
:1088A000E17809B1052BDCD023690BB1022AD8D0BD
:1088B000012E00F08081B849A86A884203D10820BF
:1088C000D0E701207047B54E20886169B4F804C034
:1088D0002B624FF0200E00230293089309930A9312
:1088E0000B932880ADF80A00A961F3682A71A5F8F6
:1088F00006C085F824708DF808E002A80DEB0E0183
:1089000098470028AED1BDF82620089BEB61C2F342
:1089100082035B00C2F3401208332B726A72A049D3
:10892000228851F8220040B90B9F788841F8220034
:10893000FF8840EA074041F822000C2B00F04281FA
:108940000E2B00F02181102B00F0308102A800F0E6
:1089500009FD002886D1089008AA376902A80221DB
:10896000B8479DF82030226985F8303058B2002A87
:1089700000F0678110F1210F00F03181894AA17A5E
:10898000126801920028C0F2738100F1604E0B0161
:108990000EF5614EDBB28EF8003395F83030019A57
:1089A00052F8302058B2002815601ADB42092032F4
:1089B00001217D4F03F01F0301FA03F347F8223032
:1089C000BFF34F8FBFF36F8F95F8303058B2002848
:1089D00006DB420903F01F036032994047F822107A
:1089E000376900F07FFC08AA02A80321B847A378E2
:1089F0009DF8202085F83120012B50B200F0E7804F
:108A000010F1210F31D06749E37A09680028C0F2DC
:108A1000278100F160421B0102F56142DBB282F85E
:108A2000003395F8312051F8303050B200281D60E5
:108A300019DB4309203301215B4F02F01F0201FAC9
:108A400002F247F82320BFF34F8FBFF36F8F95F8E3
:108A5000312050B2002806DB430902F01F026033C8
:108A6000914047F8231000F03DFC0027AF72EF72F1
:108A70006F612F6104A8049705970697079700F088
:108A800055FA9DF81030039722228DF80C20DA0653
:108A900000F1AA80190700F1C180BDF812306B8087
:108AA0002946E869FFF712FC002620222388049655
:108AB00004A88DF81020ADF81230089609960A9691
:108AC0000B9600F0D7FBEB691E805E82E969A27805
:108AD0000B8802F0030223F4C04343EA42330B80C5
:108AE000EA69138823F080031380237A012B00F0B6
:108AF0008D804BB9EA69138843F480731380EA6967
:108B0000138A23F47C531382EB69E178DA8901F04C
:108B1000030122F0060242EA4102DA81DA89A188E1
:108B2000C2F30E02A1F50041B1FA81F1490942EA0E
:108B3000C132DA81DA89E17922F02002A1F1200143
:108B4000B1FA81F1490942EA4112DA81A2791A7334
:108B500008A800F0EBF99DF82C30C3F3400313F0A4
:108B6000FF0F2B7303D0217B002900F089806B7AE3
:108B7000012B6BD00023084AEB621846AA6271E60B
:108B800018067FF56EAE81E6E378032B3FF4DEAE88
:108B9000002B7FF466AED9E64344415250E5000015
:108BA0000C05FE1F4CEB000000E100E0E378042B15
:108BB0007FF457AECAE6208940F2011188427FF463
:108BC00050AE78E6E378022B3FF64BAEBEE6236963
:108BD000002B3FF415AF10F1210F7FF414AF02A862
:108BE00000F0F4FB0B203DE6089709970A970B97D6
:108BF000F36803A808A9984700287FF451AF012122
:108C0000089A9DF81030A9722A6143E7EA69138A2D
:108C100023F47C5343F41063138275E70023012788
:108C2000F2688DF80D70089309930A930B9303A8CB
:108C300008A9904700287FF433AF089BEF726B615F
:108C40002BE710F1210F3FF4CEAE97E6EB6900223F
:108C5000A3F8B021EB6949F69912A3F8A02189E79E
:108C6000194F02F00F021B011744DBB23B76D8E626
:108C7000154A03F00F031A440901CBB213768CE6B0
:108C80002846FFF7B1F9044640B102A800F09EFB68
:108C9000E8692946FFF71AFB2046E3E595F930001D
:108CA00000F020FB95F8302053B2002BFFF65FAFA9
:108CB0005B09603302F01F020121044801FA02F24D
:108CC00040F8232053E700BFFCEC00E000E100E0A7
:108CD00068B1084AB2F8003103F00103037092F85A
:108CE00000316FF3000382F800310020704701204B
:108CF000704700BF00C00140104991F8043143F0B3
:108D0000010381F80431B1F80431DB070CD54FF0D1
:108D1000FF3300E033B1B1F80421D20703F1FF3390
:108D2000F8D40BB914207047044A92F8003160F36C
:108D3000000382F800310020704700BF00C00140EE
:108D400070B5254D82B02B6898470120FFF7D4FFFE
:108D50000021AE680320B0470021204AEC698DF85D
:108D60000110032301928DF800300320A047B0F5D5
:108D7000C97FFAD169460520B04720B140F291136E
:108D8000984200D000BE0520A047B0F5C97FFAD1B7
:108D900001230222002405208DF800308DF80330D5
:108DA0008DF8043069468DF806408DF801208DF865
:108DB00005208DF802002B69984700B100BE2B6E8C
:108DC00004209847AB6A01209847EB6A9847AB6D3F
:108DD000984702B070BD00BFF8E500000000F04108
:108DE00000B583B002A9002341F8043D034B0620DF
:108DF0009B699847019803B05DF804FBF8E5000013
:108E0000037870B423B1012B3CD0002070BC7047B4
:108E100042683E498A426BD93D4B3E4EF1251D7159
:108E2000197A41F004011972197A41F00801197296
:108E3000197A41F001011972197AF02441F0020106
:108E4000B24219721C7105D91D71197A41F01001D5
:108E500019721C71304B31499A4294BF012302238D
:108E600003731C4691F81C3103F00703A3423FBF74
:108E700091F81C3123F00703234381F81C31037858
:108E8000012BC2D18368214A93423BD8204BF12267
:108E90001A711A7A22F004021A721A7A22F008025F
:108EA0001A721A7A22F001021A721A7AF02122F04A
:108EB00002021A721971164BF1221A711A7AF021F4
:108EC00022F010021A7219711449037B91F81C21C7
:108ED00002F00702934298D091F81C2103F0070397
:108EE00022F00702134381F81C31002070BC704748
:108EF0000B498A42AED8094A037392F81C3100200C
:108F000070BC7047034A9342DED8D4E7000E2707AF
:108F10000020004000C2EB0B0068890900C001403E
:108F200000B4C40400230370704700BF0378027BC1
:108F300041F2360103F0E00342F0010210B4416057
:108F4000022443F0130341F204016FF341028460F1
:108F50000370418002735DF8044B7047037803F09F
:108F6000FE0300226FF3410342700370704700BF9D
:108F700003786FF300030370704700BF037843F07A
:108F800003030370704700BF014B0360704700BFCD
:108F9000C8E60000044B002103F1300243F8041B33
:108FA0009342FBD1704700BF1405FE1F024B43F8EC
:108FB00020100020704700BF1405FE1F08B57A4B33
:108FC000B3F84031D90700F1C180774BB3F8403195
:108FD0009A0700F1B080744BB3F840315B0700F1A1
:108FE0009F80714BB3F84031180700F18E806E4BB3
:108FF000B3F84031D9067CD46B4BB3F84001C0F3D1
:109000008010002869D1684BB3F840311A0658D453
:10901000654BB3F84031DB0547D4634BB3F84031BF
:10902000980536D4604BB3F84031590524D45E4BD3
:10903000B3F840311A0512D45B4BB3F84031DB046E
:1090400000D408BD594BDB6A002B40F0AA80564A79
:10905000B2F8303143F48053A2F8303108BD534B9D
:109060009B6A002B40F09A804F4AB2F8303143F4AB
:109070000063A2F83031DFE74C4B5B6A002B40F015
:109080008A80494AB2F8303143F48063A2F8303123
:10909000CDE7464B1B6A002B7AD1434AB2F83031F8
:1090A00043F40073A2F83031BCE7404BDB69002B7E
:1090B0006BD13D4AB2F8303143F48073A2F83031BD
:1090C000ABE73A4B1B68002B5CD1374AB2F8303122
:1090D00043F08003A2F830319AE7344B5B68002BF1
:1090E0004ED1314AB2F8303143F04003A2F830316A
:1090F00089E72E4B9B69002B3FD12B4AB2F83031C8
:1091000043F01003A2F8303176E7284B5B698BBB44
:10911000254AB2F8303143F00803A2F8303166E74F
:10912000224B1B691BBB204AB2F8303143F00403C9
:10913000A2F8303155E71D4B9B68ABB91A4AB2F81B
:10914000303143F00203A2F8303144E7174BDB68BB
:109150003BB9154AB2F8303143F00103A2F830317F
:1091600033E703209847F4E702209847E6E7042016
:109170009847D8E705209847CAE706209847BCE7F4
:109180009847AEE7002098479FE70720984790E769
:109190000820984781E70920984772E70A209847F6
:1091A00062E70B20984752E7006000401405FE1F5D
:1091B00030B4124902784588895C447801F01F0375
:1091C000890614D501212B2A01FA03F008D0332A8D
:1091D00004D1012C04BF5A1C04FA02F030BC7047C1
:1091E000072DFBD9013301FA03F030BC70472C4442
:1091F0001B1B0120984030BC704700BF04EB0000EF
:109200000378452B12D870B5164CE65CFF2E0BD0B8
:1092100015460C46FFF7CCFF134BB20953F822302A
:1092200034B1B20611D585B9032070BD0120704755
:10923000EFF31082012181F31088196821EA000000
:10924000186082F31088204670BDEFF31082012170
:1092500081F3108819680843186082F31088002091
:1092600070BD00BF04EB0000F4EA00000121002201
:10927000FFF7C6BF00210A46FFF7C2BF704700BF15
:10928000A0F101000028FBD1704700BF2DE9D043B9
:1092900001FB00F4FFF7A4FD4FF47A71A4FB0189F0
:1092A00000274FF0FF364F4508BF46450C4BB3FB38
:1092B000F0F005D3B8FBF0F0800860B9BDE8D083CA
:1092C0008000B4FBF0F0A0FB01018F4208BF864292
:1092D000F3D24FF0FF30BDE8D043FFF7D1BF00BF5E
:1092E00000CA9A3B002808DB800000F1804000F5AE
:1092F000C640036823F48033036070470B4A0C4B6D
:1093000010B49B1A0B4CDB08236063B10A480021A0
:109310009388C3F3090340F8043F236801318B426B
:1093200002F10802F4D85DF8044B70470005000014
:10933000E00500004405FE1FFC620040012202E03F
:10934000C0E8432F43B1D0E84F3F13F0FF0FF7D0F1
:10935000BFF32F8F08207047184670470023037013
:10936000704700BF164B10B41C687CB1154B0068E9
:109370001A681368984218BF002304D10AE052F813
:10938000041F814207D00133A342F8D103205DF8C6
:10939000044B704700230C4A12680121134403E078
:1093A000C3E8401F0028F2D0D3E84F2F12F0FF0F80
:1093B000F6D0BFF32F8F08205DF8044B704700BF35
:1093C0004805FE1F4C05FE1F5005FE1F0F4B10B435
:1093D0001C687CB10E4B00681A681368984218BF6D
:1093E000002304D109E052F8041F814206D0013362
:1093F000A342F8D15DF8044B70470023054A126878
:109400000021D1545DF8044B704700BF4805FE1F92
:109410004C05FE1F5005FE1F38B50A4C0A4D0B487F
:109420000B490C4B0C4A04602D1BAD080D601A60F3
:109430003DB104EB850520460434FFF7C7FFAC427D
:10944000F9D138BDE0050000900700004C05FE1F73
:109450004805FE1F5005FE1F3804FE1FEFF3108164
:10946000012383F31088124B33F8102092B22AB1F3
:1094700033F81020013A92B223F8102033F810305C
:109480009BB293B910B40B4A0B4CB2F8FE3334F8CC
:1094900010009BB243F4254323EA0003A2F8FE33F5
:1094A00081F310885DF8044B704781F31088704792
:1094B0005405FE1F00E0014050EB000030B4EFF314
:1094C0001084012383F310880D4A32F810309BB2C8
:1094D0005BB90C4D0C49B5F8FE3331F810109BB256
:1094E00043F425430B43A5F8FE3332F81030013323
:1094F0009BB222F8103084F3108830BC704700BF54
:109500005405FE1F00E0014050EB0000024B00221A
:109510001A805A809A8070475405FE1F0C4A08B57D
:1095200013688BB1033020F003000A4918448842C5
:1095300002D81060184608BD02F0E8FD0C23036055
:109540004FF0FF33184608BD034B1360EAE700BF36
:109550005C05FE1F2021FE1F2011FE1F00BE70476C
:1095600008B500F005F800F073F8FEE7704700BF9B
:10957000284A38B5D2F8883043F47003C2F88830EE
:109580000020FFF7F3FFFFF705FD234B1B6898470B
:10959000FFF7BCFFFFF7D4FB204A214B21481B6893
:1095A000002414809847204A204B9B1A05D013446E
:1095B000214603F8011D9A42FBD11D481D4BC01ADC
:1095C00007D01D4A184412F8011B03F8011B8342FF
:1095D000F9D1FFF705FC194C194B1A4D18602D1BDA
:1095E0000120FFF7C3FF032DC8BF2D1904DD54F878
:1095F000043B9847AC42FAD1FFF70EFFFFF77EFE1F
:10960000114B12481B6898470020BDE83840FFF70F
:1096100035BE00BF00ED00E050E50000F804FE1F7D
:1096200058E400007CEE0000DC04FE1F2011FE1F49
:10963000A404FE1FC001FE1F9CFA00002C04FE1FA4
:109640006005FE1F3004FE1F6CE5000058EB0000B3
:1096500008B500F029FE002008BD00BFF8B50E4C8B
:109660000E4DE76826683B686168304698470C49AC
:10967000286000F0B5FD7B68A1683046984709492D
:10968000286000F0ADFDBB68304698470649286069
:10969000BDE8F84000F0A4BDF0EB0000B40DFE1FE3
:1096A00094EF0000A8EF0000C0EF0000FFFFFFFFF5
:1096B0002DE9F04782B002AC374BDFF8E4A01D681B
:1096C000DE68DFF8E0907369DFF8DC80002724F8BB
:1096D000027D284622466FF002019847BDF8060039
:1096E00007EE900AF8EE677A17EE900A01F046FF4F
:1096F00023A3D3E9002301F095FF23A3D3E900239B
:1097000001F0DCFD02F0C8F97369CAF800002246D6
:10971000284601219847BDF8060007EE900AF8EEAA
:10972000677A17EE900A01F029FF19A3D3E9002305
:1097300001F078FF02F0B0F97369C9F80000224621
:10974000394628469847BDF8060007EE900AF8EE1D
:10975000677A17EE900A01F011FF0DA3D3E90023F9
:1097600001F060FF00220D4B01F0A8FD02F094F91A
:10977000C8F8000002B0BDE8F08700BFAFF300807A
:1097800034F8DF703D0FC33F5602733E06577140F9
:10979000E7ABE4637781623FF0EB000000001B4021
:1097A0001406FE1F1C06FE1F1806FE1FF8B5114DFD
:1097B000114CAF682E68FB683046984794F920003A
:1097C000013800F071F969680869002294F92030C5
:1097D0001F3302EBC30340F832300132042AF5D1C3
:1097E0003B6830469847054B05491860BDE8F8408E
:1097F00000F0F6BC68EE00008C10FE1FB40DFE1FDA
:10980000D8EF000008B51E4B1868002831D11D4B59
:109810001A683ABB1C4B1A78EAB91C4B1A789AB9E9
:109820001B4B1A784AB91B4B1A782AB100221A48E6
:109830001A7001F025FC062008BD002217481A7096
:1098400001F01EFC0520EEE7002215481A7001F019
:1098500017FC0420E4E7002212481A7001F010FC03
:109860000320DAE7002210481A6001F009FC022008
:10987000D0E700220D481A6001F002FC0120C6E783
:109880003006FE1F2806FE1F3406FE1F2C06FE1F94
:109890003506FE1F2006FE1F80F0000060F000006D
:1098A00044F0000028F000000CF00000F0EF000091
:1098B0002DE9F84F1C4D1D4F1D4CDFF878B0DFF837
:1098C00078A0DFF87890DFF87880DFF878C0DFF8EC
:1098D00078E02E46002346F8050B6B73086849684C
:1098E000C5F80500B868716023602A71CBF80030B4
:1098F0002A46CAF80030856889F80030386888F848
:1099000000301F218CF800308EF80030A84718B1C5
:1099100007E0FFF777FF10B92368002BF9D0BDE807
:10992000F88FBDE8F88F00BFBC0DFE1F68EE000089
:109930002406FE1F3006FE1F2806FE1F3406FE1FEB
:109940002C06FE1F3506FE1F2006FE1F036870B59D
:10995000044643B92379062B4FD8DFE803F00D3ACC
:109960003E42464A09000020384900F039FCF1E740
:10997000374B01221A7070BD364B374D9A68A1687B
:10998000186854682A46A047344B354918600020AF
:1099900000F026FC334A2B681268934231D0324AD9
:1099A000126893423DD0314A1268934244D0304A03
:1099B0001268934230D02F4955F8056F0A682E4837
:1099C0002E4C6D68456042F0F80206600A60236024
:1099D00070BD2B4B01221A6070BD2A4B01221A6008
:1099E00070BD294B01221A6070BD284B01221A70EC
:1099F00070BD274B01221A7070BD264B01221A70D0
:109A000070BD55F8050F1B4C6968234B226803C3D2
:109A100042F00102226070BD204B42F20F721A60C8
:109A200070BD55F8050F134C69681D4B226803C3C0
:109A300042F00202226070BD0E4A1A491368B5F85E
:109A40000500088043F00403136070BD98F0000027
:109A50003506FE1F68EE0000880FFE1FB40DFE1FC6
:109A6000D4F00000C00FFE1F1C10FE1FA80FFE1F29
:109A7000D00DFE1F3806FE1F8010FE1F740FFE1F44
:109A80002406FE1F3006FE1F2806FE1F3406FE1F9A
:109A90002C06FE1F2006FE1F0C10FE1FCC0DFE1F05
:109AA0001410FE1F6810FE1F2DE9F84F00210F2231
:109AB00001F0AAFBDFF858A0DFF85880DFF858E083
:109AC0000F4E104C104A114BC00000F5807B00F285
:109AD000011900F5817C00F2031700F5827500F290
:109AE000051100F58370CAF800B0C8F80090CEF8F0
:109AF00000C03760256011601860BDE8F88F00BFB6
:109B0000D00DFE1F2010FE1F7010FE1FBC0FFE1F89
:109B1000C00FFE1F1C10FE1FA80FFE1F2DE9F04FE7
:109B2000394BDFF8F8B05D68384C2B6A83B04FEAE8
:109B3000202C4FF0060E002602278DF805C08DF868
:109B400000E08DF806008BF800608DF804708A46FE
:109B500040F203103146914698472D49206000F0AD
:109B60003FFB2C4BD3F808801E68D8F80870012200
:109B7000694630461346B8472749206000F030FB5D
:109B80009BF80030254F002BFAD02B6A012140F2C0
:109B900003109847002139702B6A206040F20310AF
:109BA00098471B49206000F01BFB01A9D8F80870FA
:109BB000304603220123B8471749206000F010FB0C
:109BC0009BF80030154A002BFAD000231370514641
:109BD000D8F8087030464A460123B847104920603B
:109BE00000F0FEFA9BF80030002BFBD02B6A01211D
:109BF00040F2031098470B49206000F0F1FA20680A
:109C000003B0BDE8F08F00BF64EB0000B40DFE1F91
:109C1000ECF0000004ED000010F100003C06FE1F17
:109C20002CF1000048F100002DE9F04F234B244CAB
:109C3000D3F8048083B0031200264FF0030B8DF895
:109C400006008DF805302670D8F820308DF804B065
:109C50008A4640F20310314691469847194900F070
:109C6000BFFA194B9F681E68BD6801A95A46304665
:109C70000123A847154900F0B3FA2378104A002BB6
:109C8000FBD00023137051467F6830464A460123BB
:109C9000B8470F4900F0A4FA2378002BFCD0D8F87D
:109CA0002030012140F2031098470A49044600F091
:109CB00097FA204603B0BDE8F08F00BF64EB0000C8
:109CC0003C06FE1F6CF1000004ED00008CF100006A
:109CD000A8F10000C0F1000010B5014604462122A1
:109CE0004FF4E060FFF7A0FF064B0749186000F053
:109CF00077FA94F920000121102201F085FA84F806
:109D0000200010BDB40DFE1FE4F1000008B50146AF
:109D100021224FF4E060FFF701FF034B0349186075
:109D2000BDE8084000F05CBAB40DFE1FF8F1000079
:109D3000084B10B4421E03F1200413F8011F02F86F
:109D4000011FA342F9D1012380F820305DF8044BB4
:109D5000704700BF93F70000014B01221A70704753
:109D60003C06FE1F08B5014610220020FFF75CFFED
:109D7000034B04491860BDE8084000F031BA00BF49
:109D8000B40DFE1F10F2000008B50146102200209D
:109D9000FFF7C4FE034B04491860BDE8084000F01B
:109DA0001FBA00BFB40DFE1F28F2000030B583B00B
:109DB00002AC552304F8013D012221464FF4807086
:109DC000FFF7ACFE284D2949286000F009FA21462A
:109DD00001224FF48070FFF727FF2549286000F02B
:109DE000FFF99DF80730552B02D0012003B030BD9C
:109DF000AA23012221464FF480708DF80730FFF727
:109E00008DFE1C49286000F0EBF9214601224FF439
:109E10008070FFF709FF1849286000F0E1F99DF80C
:109E20000730AA2B18BF0220E0D1002301222146CF
:109E30004FF480708DF80730FFF770FE0F492860EF
:109E400000F0CEF9214601224FF48070FFF7ECFEBE
:109E50000B49286000F0C4F99DF80730002B14BFAF
:109E600003200020C2E700BFB40DFE1F44F2000033
:109E70005CF2000074F200008CF20000A4F200001A
:109E8000BCF2000008B5074B9A6859681868126858
:109E90009047054900F0A4F9FFF788FF034B1860CD
:109EA00008BD00BF04ED0000D4F200002410FE1F26
:109EB0002DE9F84F224BDFF894E09F681D68DFF82A
:109EC0009080204E3A6859680024CEF80040284619
:109ED000C8F80040346090471B4AD2F808A0D2F876
:109EE00000905168DAF80030484698472146C8F893
:109EF0000040BB682846984740F6FF7B2146346007
:109F00000CE0C8F80040BB6898476100B1F5805F7D
:109F100012BF3160C6F800B040F6FF71DAF80830C1
:109F200089B248469847012164200C44FFF7AEF9F6
:109F300040F601039C422846A1B2E2D1BDE8F88F69
:109F400018EC0000B010FE1FA8ED00006810FE1F06
:109F5000B00FFE1F2DE9F041051E22DB40F6FF7316
:109F60009D42A8BF1D46104C21688D4214D015DCBF
:109F70004FF0FF380D4B9F681E68BB6889B23046B2
:109F8000984701210820FFF781F9216841448D425B
:109F90002160F2D1BDE8F081BDE8F0814FF0010809
:109FA000E8E70025DFE700BFB00FFE1F18EC000058
:109FB000114B2DE9F0475F68104D3B6A104C884605
:109FC0000646002135F82000914698470D4B9968C8
:109FD0001868D1F808C00023237041464A4601237F
:109FE000E0472378002BFCD03B6A35F8260001219E
:109FF000BDE8F047184700BF64EB00007803FE1F80
:10A00000B410FE1F80EC00002DE9F04F1C4C1D4FDA
:10A0100066681D4C83B002AD804605F8011D37F817
:10A02000200000219B46336A92469847174BD3F88D
:10A0300008901B68009318460122002329462370CC
:10A04000D9F808501346A84723780F4A002BFBD0B5
:10A05000BBF1000F0BDD00231370D9F804500098FA
:10A0600051465A460123A8472378002BFCD0336A77
:10A0700037F828000121984703B0BDE8F08F00BFF2
:10A0800064EB00007803FE1FB410FE1F80EC00009C
:10A090002DE9F041224B234F9A68596818681268DD
:10A0A000214E82B09047214900F09AF800242546BD
:10A0B0004FF018082046694601228DF80050FFF73E
:10A0C00077FF2046694601228DF80080FFF770FF78
:10A0D00020232046694601228DF80030FFF768FFF3
:10A0E0004FF0880E03232046694602228DF800E0D7
:10A0F0008DF80130FFF75CFF90232046694601345C
:10A1000002228DF801508DF80030FFF751FF042C2A
:10A1100047F8045B46F8045BCCD102B0BDE8F0819F
:10A1200080EC0000640FFE1F980FFE1FF8F2000085
:10A13000F0B5002183B0032201F066F80F4B53F80D
:10A1400020308DF8043004461F121E1469461B0E81
:10A15000982505228DF801308DF803708DF8026086
:10A160008DF80050FFF724FFE023204669460122C6
:10A170008DF80030FFF71CFF03B0F0BD0C10FE1F80
:10A1800070B5134E82B00024E825204669460122AE
:10A190008DF80050FFF70CFF204668216A46042323
:10A1A000FFF732FF9DF801109DF802309DF8032063
:10A1B0009DF80000090441EA03231343013443EAF4
:10A1C0000063042C46F8043BDFD102B070BD00BF31
:10A1D000640FFE1F014B01221A707047B410FE1F5E
:10A1E00000B970472DE9F0410546B2B00C462A4649
:10A1F00023462949294E684602F028FC684600F0AB
:10A200003FFF00F067F9264800F07EF92A4625490D
:10A21000684602F01BFC0027684600F075F9B84656
:10A22000651E16E015F8017F03F8C87C00F0ECFF0E
:10A2300086FB08324FEAE873C3EBA20303EB430348
:10A24000C3EBC303C3EB0803142B074618D008F174
:10A250000108204600F06AFF32AB80453B444FF0D6
:10A2600000014FF0C70207F10100DBD332AB1F44FE
:10A27000684607F8C81C00F047F900F0FFF8FEE751
:10A2800032AB03440A2701300021C72203F8C87CFF
:10A2900000F0BAFF0746DAE710F30000310CC330D4
:10A2A00028F3000034F3000000F09ABBFFFFFFFF2B
:10A2B0002DE9F04F644FDFF898A1BD683C686B69E9
:10A2C000DFF89C8183B001224021204698470DF1A0
:10A2D000080979682B6820469847012209F8052D5E
:10A2E00000273B468AF8007020464946EE68B04792
:10A2F000564BC8F800701F609AF80030544A002B83
:10A30000FAD0002717703B4601A920460222AE680A
:10A31000B0474E4BC8F800701F609AF800304C4FA1
:10A32000002BFAD09DF805309DF8040003EB0020C7
:10A3300001F012F940A3D3E9002301F073F901F011
:10A34000ABFB444A4FF0000B022310608DF8033042
:10A3500087F800B05B46EF68204649460122B847BF
:10A360003A4BC8F800B0C3F800B09AF80030384A49
:10A37000002BFAD0002717703B46204601A9022285
:10A38000AE68B047314BC8F800701F609AF80030D3
:10A390002F4F002BFAD09DF805309DF8040003EBF9
:10A3A000002001F0D9F824A3D3E9002301F03AF901
:10A3B00001F072FB284A4FF0000B032310608DF868
:10A3C000033087F800B05B464946EF68204601221B
:10A3D000B8471E4BC8F800B0C3F800B09AF8003078
:10A3E0001B4A002BFAD0002717703B4601A92046D4
:10A3F0000222AE68B047154BC8F800701F609AF88B
:10A400000030002BFBD09DF805309DF80400134E62
:10A4100003EB002001F0A0F809A3D3E9002301F029
:10A4200001F901F039FB6B6830602046984703B0B2
:10A43000BDE8F08FAFF300807B14AE47E17A543F64
:10A440007B14AE47E17A843FE8ED0000FC10FE1F6C
:10A450003D06FE1F0411FE1F0C11FE1F0811FE1FFA
:10A46000C80FFE1F034A044B017A117001221A70B3
:10A47000704700BF0011FE1F3D06FE1F114B70B557
:10A480005D68114C2B6A00262670012140F6010000
:10A49000984731462B6A40F2071098470B4B0C49FE
:10A4A0009A681868966801234FF48062B047237851
:10A4B000002BFCD02B6A40F207100121BDE8704050
:10A4C000184700BF64EB00001011FE1F8CEC000069
:10A4D0004006FE1F084B002003F5806103F8010FC2
:10A4E0008B424FF00002F9D104480549054B026048
:10A4F0000A701A70704700BF3F06FE1F1411FE1F3E
:10A500001111FE1F1811FE1F2DE9F0412D4F3B7850
:10A51000072B55DCDFF8B880027898F800E00EEBE6
:10A52000C31312B30446284D284E0AE00D2A22D147
:10A530003B784FF0000EDB0188F800E014F8012FA3
:10A540009AB152B20A2AF1D138780722002101309B
:10A5500000F05AFE4FF0000E387088F800E014F852
:10A56000012FC3B2DB01002AEBD103F07F0388F88F
:10A570000030BDE8F0811F2A1BDD203A02EB4202C9
:10A580005100BEF17A0F01F1080117DDCEF1800014
:10A590000028D3DD31440022B3F5806FBCBF11F831
:10A5A00002C003F805C00132824203F10103F3DB6C
:10A5B000C4E7BEF17A0F4FF00801E7DC0620E9E7B7
:10A5C000BDE8F0811811FE1F4006FE1F50F3000089
:10A5D0001111FE1F014B01221A7070471011FE1F4E
:10A5E0002DE9F0411C4D1D4C1D4895E848001A12FC
:10A5F0004FEA262C4FEA264E23704FEA2348370EA7
:10A600001B0E214662700068E3700822267184F8F0
:10A6100005C084F806E0E77184F80280FFF748F986
:10A62000AB68EA680F4823704FEA234E17121614DE
:10A63000150E4FEA232C1B0E2271214684F801C00F
:10A6400084F802E0E3706771A671E5710068082282
:10A65000BDE8F041FFF72CB9640FFE1F7810FE1F14
:10A660002010FE1F7010FE1F2E4B2F4A1B68106813
:10A6700010B52E4C23701B12637000F07FFF2C4B23
:10A68000002200F0CFFF01F0DFF9FF22002100F0EF
:10A69000BBFD284BA070186800F070FF264B00220D
:10A6A00000F0C0FF01F0D0F9FF22002100F0ACFD66
:10A6B000224BE070186800F061FF214B002200F08F
:10A6C000B1FF01F0C1F9FF22002100F09DFD1D4BFB
:10A6D0002071186800F052FF154B002200F0A2FF15
:10A6E00001F0B2F9FF22002100F08EFD164B6071DF
:10A6F000186800F043FF154B002200F093FF01F0B3
:10A70000A3F90021FF2200F07FFD114B114A1B68C5
:10A71000A071E371106821460822BDE81040FFF7E0
:10A72000C7B800BFB00FFE1F0C11FE1F7810FE1F30
:10A73000000044400411FE1F000069401806FE1F7F
:10A74000000044C01C06FE1F1406FE1F000014403B
:10A750002410FE1FBC0FFE1F38B51E4C2368D907FE
:10A7600011D423681B4D9A071BD42368194D5B072E
:10A7700025D42368174A13F0F80F03D0136823F089
:10A78000F803136038BD0020FFF7D2FC0120FFF76B
:10A79000CFFC23680F4D23F00103236023689A0741
:10A7A000E3D50220FFF7C4FC0320FFF7C1FC2B68B0
:10A7B00023F002032B602368064D5B07D9D5064BB7
:10A7C0001868FFF7C7FB2B6823F004032B60FFF723
:10A7D0004BFFCEE73806FE1F6810FE1FC2B222F004
:10A7E0002003413B192B01D8112070472328FBD0AF
:10A7F0005F28F9D03F2805D0A2F13003092B03D8F8
:10A8000021207047482070472B2807D02D3A012A75
:10A8100004D92A280CBF442000207047222070470A
:10A820002DE9F04F664B674D674C684E83B0194673
:10A830000093002307461A466320F2541433B3F5FD
:10A84000967F45F8042F41F8042F44F8040FF4D103
:10A850003D46DFF8808115F90109FFF7BFFF07F1D9
:10A860004F03D8F800B0019381464FF0000A15F865
:10A87000014F67B23846FFF7B1FF002C44D00D2FCF
:10A8800042D080EA090213070CD0B9F1220F1DD083
:10A890000BEB8B020AEB82024FF00003B354B9F1C9
:10A8A000000F1CD160B12C78D8F8003003EB830383
:10A8B0000AEB83030AF1010ABAF1130FF45475DCB1
:10A8C000019B9D428146D2D158462CE02128EBD0F5
:10A8D0000BEB8B020AEB82014FF0000373543C4BED
:10A8E00043F82B900BF1010BBBF10F0FC8F800B030
:10A8F0005CDC38B10BEB8B032A7806F823204FF091
:10A90000010ADDE78246DBE70BEB8B020AEB8201F3
:10A910002F4A00245846745442F82B90B9F1000F86
:10A9200049D10F2842DC002842DDDFF8ACB0DFF867
:10A93000ACA0264C4FF0000904260125632719E03E
:10A94000CAF8003094F900302A2BA3F1610128D015
:10A950000029CBF8001001DACBF80070D8F800001D
:10A9600009F1010981450BF1040B0AF1040A04F114
:10A9700014041DDA009A52F8043F009213F02003E9
:10A98000DED0204600F0D2FB0A2820460ED800F088
:10A99000D9FB94F90030CAF800002A2BA3F1610119
:10A9A000D6D1CBF80060CAF80050D7E74FF0FF309F
:10A9B00003B0BDE8F08F0BF10100C8F80000B0E76C
:10A9C000C80FFE1F2410FE1FFC0EFE1FD40DFE1F1D
:10A9D000CC0FFE1FB40FFE1F000FFE1F2810FE1F1E
:10A9E0002DE9F04F9BB000F0F3FBFFF761FA00F0A8
:10A9F00033FBB34800F044FBB24800F041FBB248DF
:10AA000000F03EFB00F008FCFEF728FEFFF73AFAE4
:10AA1000AE48FFF761F9AD4BAC4993F9052093F9C6
:10AA2000040093F9074091F9005093F90830A2F11E
:10AA30003001642202FB01F230384FF47A71303C6D
:10AA400001FB002104EB840401EB4402303B432D65
:10AA5000134404D19D4A92F90120532A7AD09C4A8A
:10AA60009C48144600F00CFB9848FFF761F99748A2
:10AA7000FFF74CF90023204623606360A360E36086
:10AA8000FFF782F9FEF792FEFFF702FB924B904A26
:10AA90005B68029301211B6A019240F20C7015461B
:10AAA00098474FF4FA7000F039FB2846FFF75AF93F
:10AAB0008A4E002455F8043B46F8043B20460134F6
:10AAC000FFF736FB042CF5D100231946844AD154F4
:10AAD0000133282B4FF00002F8D1824CDFF854B23A
:10AAE0002270DFF85482804F804E814DDFF84CA2F7
:10AAF000CBF8002027E02378ABB17A4A7D490023C8
:10AB0000CBF800301370764A0B601278232A07D0F6
:10AB1000734A794992F900200B601F2A89464BDC61
:10AB2000764800F0ADFA3B686F4AB3F5C87F3CDC6D
:10AB300032686E4940F2C9239A4215DC2B686C4A90
:10AB4000B3F57A7F1DDCD8F80030002BD3D0FFF7A7
:10AB500003FED0E75D4A92F90220312A7FF47FAFED
:10AB6000643B012B8ED97AE700230B60FEF7A0FD32
:10AB7000FFF79EFBFFF778FD2B685D4AB3F57A7F00
:10AB8000E1DD0198DAF80030036000211160DAF8A5
:10AB9000041041600199DAF80820DAF80C304C48CA
:10ABA0008A60CB60FFF7F0F8CDE700231360FFF772
:10ABB000E7FAFFF715FDBBE74948FFF731FE00282C
:10ABC000C9F800002BDBABD04D494E4800F0E0FA4D
:10ABD00078B306A84C493B4A01F038FF06A800F0BC
:10ABE0004FFAA0E74846494900F0D2FA002840F061
:10ABF0003E814846464900F0CBFA002840F03781B4
:10AC00004846444900F0C4FA002800F04C813A4B11
:10AC10001B68012B00F07081022B00F050813E4830
:10AC200000F02EFA374800F02BFA274800F028FAF7
:10AC300079E73448394900F0ABFAB0B1D9F80030BF
:10AC4000022BECD12F4B93F914303F2B78D0344B9F
:10AC50005868344940F2FF7200F0D6FA00F50060FF
:10AC6000FFF778F9FFF700FD5AE726482E4900F074
:10AC70008FFA80B1D9F80030032BD0D1214B93F952
:10AC80001430652BCBD11F4B93F928303F2B57D075
:10AC9000234B9868DDE71B48244900F079FA002827
:10ACA00064D01F4B5B68002B56D1029B00211B6AAE
:10ACB00040F20C7098471E4800F0E2F933E700BFFD
:10ACC00098F5000094F700006CF700008C10FE1F50
:10ACD000780FFE1FA4F5000064EB00000C10FE1FAF
:10ACE000480AFE1F440AFE1FCC0DFE1FC40FFE1FA4
:10ACF0006C10FE1FB80FFE1FB40FFE1F78F7000088
:10AD0000C4F50000D40DFE1FCCF50000D0F6000005
:10AD1000D8F60000E4F600007CF70000DCF5000047
:10AD20002810FE1F00F8FFFFE8F50000F0F5000016
:10AD3000FCF50000400AFE1F3806FE1F640FFE1FD0
:10AD40009E4B9F491A6806A8A2F5006201F07EFE9C
:10AD500006A800F095F9E6E6029B01211B6A40F285
:10AD60000C709847974800F08BF9DCE696489749B5
:10AD700000F00EFA20B3964B1B68012B13D14FF055
:10AD80000009944B4A4643F8042B484609F101094F
:10AD9000049203930593FFF7CBF9B9F1040F039BDA
:10ADA000049AF0D1BCE68C4B00215868032200F0D5
:10ADB0002BFA8849002241F82020FFF7B9F9AFE6C5
:10ADC000DFF804928549484600F0E2F9B8B1804BBB
:10ADD0001B68052B7FF423AF814BDFF8F89100202F
:10ADE00053F8042F49F8042B421C04930392FFF7F5
:10ADF0009FF9039A049B042A1046F1D190E6484635
:10AE0000784900F0C5F968B1FEF7D0FF0246002886
:10AE10003FF486AE06A8744901F018FE06A800F0BB
:10AE20002FF980E64846714900F0B2F9C0B1704888
:10AE300000F11009FEF796FF6E4800F021F9A9F124
:10AE4000100353F8042B6C49039306A8049301F0F4
:10AE5000FDFD06A800F014F9039B4B45F1D1E4E693
:10AE60004846664900F094F900283FF4BBAE6448B8
:10AE700000F006F96349644A06A801F0E7FD06A858
:10AE800000F0FEF8614800F0FBF8614B614993F96E
:10AE9000202006A801F0DAFD06A800F0F1F85E48CF
:10AEA00000F0EEF83FE648465C4900F071F930B337
:10AEB000FEF7FEFBFFF7FCF9FFF7D6FB30E699F94A
:10AEC00014303F2B18D0464B01211022586800F057
:10AED0009BF94F4B83F820001846FEF717FFFEF74B
:10AEE00065FC4F4906A84A4B93F9202001F0AEFDBE
:10AEF00006A800F0C5F816E606A83149F3E748466B
:10AF0000484900F045F9002848D0FEF7D1FBFFF78B
:10AF1000CFF93B4800F0B4F8434B186800F02EFB23
:10AF200002460B4606A8414901F090FD06A800F034
:10AF3000A7F83F4B186800F021FB02460B4606A815
:10AF40003C4901F083FD06A800F09AF83A4B1868D6
:10AF500000F014FB02460B4606A8384901F076FDC6
:10AF600006A800F08DF8364B186800F007FB024683
:10AF70000B4606A8334901F069FD06A800F080F8E9
:10AF8000314B186800F0FAFA02460B4606A82F4922
:10AF900001F05CFD06A800F073F8C4E548462C49B2
:10AFA00000F0F6F800283FF43AAE2A4800F068F8BE
:10AFB00041F2883000F0B2F8B5E500BFB00FFE1FD7
:10AFC000E0F5000004F60000D40DFE1F0CF60000B2
:10AFD000B40FFE1F0C10FE1F000FFE1F1CF600001A
:10AFE0002810FE1F2CF6000038F6000048F600007E
:10AFF000780FFE1F58F600005CF6000064F60000B3
:10B0000068F600006CF6000094F7000084F600007B
:10B010008C10FE1FC0F600006CF7000008F700005F
:10B02000F0F600000CF700000C11FE1F14F70000F2
:10B030000411FE1F24F700001806FE1F34F700005D
:10B040001C06FE1F44F700001406FE1F58F7000000
:10B0500070F7000078F70000074B70B51C689D681A
:10B0600059682A68204690476B6804492046502258
:10B07000BDE87040184700BF50EC0000480AFE1FB2
:10B0800070B5054600F052F8021E0EDD074B084C65
:10B09000996818688B6800264F2A2946A8BF4F2256
:10B0A000267098472378002BFCD070BD50EC000030
:10B0B0008803FE1F38B58388022B16D0802B17D14A
:10B0C000007A0C2814D90D2813D001F0EBFC0E4B9C
:10B0D0000E491A68C0B288541A6801321A601A6898
:10B0E0004F2A05DD4F221A6038BD094B01221A7024
:10B0F00038BD054B054C18680649074A00252554FC
:10B1000001230B60137038BD400AFE1F480AFE1F62
:10B110008803FE1FB80FFE1F440AFE1F002803DD30
:10B120004FF47A71FEF7B2B8704700BF431E00209B
:10B1300002E00130502803D013F9012F002AF8D182
:10B14000704700BF03785AB2202A1EDD30B40021B8
:10B15000012506E003EB440110F8013F5AB2202A12
:10B160000FDD303B092B01EB8104A2F13003F1D953
:10B1700010F8013F2D2A5AB208BF4FF0FF35202AA0
:10B18000EFDC01FB05F030BC70470020704700BFCA
:10B19000F8B50D46044601F07DFC0746284601F04F
:10B1A00079FC874201D00020F8BD002F0EDD274436
:10B1B000013D14F9010B01F075FC064615F9010F6C
:10B1C00001F070FC8642EED1BC42F2D10120F8BD04
:10B1D00070B40748074E084C084D0949094A002336
:10B1E00033602B60237003600B60136070BC70478A
:10B1F000CC0DFE1FB80DFE1F640DFE1F8810FE1F34
:10B20000C40FFE1F6C10FE1F884203DB9042A8BFD4
:10B21000104670470846704738B50B4B0B4D9A687F
:10B220005968126818680A4C90470A4B0A49186016
:10B23000FEF7D6FF09480A490A4A00232B6023601B
:10B2400003600B60136038BDC8ED00008810FE1F5E
:10B25000C80FFE1FB40DFE1FB4F70000CC0DFE1F7B
:10B260006C10FE1FC40FFE1FF0B5DFF840C0DFF802
:10B2700040E00B4F0B4E0C4DDCF80040DEF80000B8
:10B28000396832682B6801340130013101320133F1
:10B29000CCF80040CEF80000396032602B60F0BD81
:10B2A000CC0DFE1F6C10FE1FC40FFE1F8810FE1F6A
:10B2B000C80FFE1F81F0004102E000BF83F0004391
:10B2C00030B54FEA41044FEA430594EA050F08BF41
:10B2D00090EA020F1FBF54EA000C55EA020C7FEA05
:10B2E000645C7FEA655C00F0E2804FEA5454D4EB82
:10B2F0005555B8BF6D420CDD2C4480EA020281EA4C
:10B30000030382EA000083EA010180EA020281EA83
:10B310000303362D88BF30BD11F0004F4FEA0131D5
:10B320004FF4801C4CEA113102D0404261EB4101E4
:10B3300013F0004F4FEA03334CEA133302D052426A
:10B3400063EB430394EA050F00F0A780A4F1010426
:10B35000D5F1200E0DDB02FA0EFC22FA05F2801860
:10B3600041F1000103FA0EF2801843FA05F3594146
:10B370000EE0A5F120050EF1200E012A03FA0EFCC5
:10B3800028BF4CF0020C43FA05F3C01851EBE371EF
:10B3900001F0004507D54FF0000EDCF1000C7EEB0C
:10B3A00000006EEB0101B1F5801F1BD3B1F5001F4A
:10B3B0000CD349085FEA30004FEA3C0C04F1010469
:10B3C0004FEA445212F5800F80F09A80BCF1004F92
:10B3D00008BF5FEA500C50F1000041EB045141EA14
:10B3E000050130BD5FEA4C0C404141EB010111F415
:10B3F000801FA4F10104E9D191F0000F04BF0146C0
:10B400000020B1FA81F308BF2033A3F10B03B3F19D
:10B4100020020CDA0C3208DD02F1140CC2F10C022D
:10B4200001FA0CF021FA02F10CE002F11402D8BF8B
:10B43000C2F1200C01FA02F120FA0CFCDCBF41EA57
:10B440000C019040E41AA2BF01EB0451294330BD26
:10B450006FEA04041F3C1CDA0C340EDC04F1140403
:10B46000C4F1200220FA04F001FA02F340EA0300DA
:10B4700021FA04F345EA030130BDC4F10C04C4F120
:10B48000200220FA02F001FA04F340EA0300294600
:10B4900030BD21FA04F0294630BD94F0000F83F44A
:10B4A000801306BF81F480110134013D4EE77FEA2D
:10B4B000645C18BF7FEA655C29D094EA050F08BF79
:10B4C00090EA020F05D054EA000C04BF194610465A
:10B4D00030BD91EA030F1EBF0021002030BD5FEA9E
:10B4E000545C05D14000494128BF41F0004130BDC6
:10B4F00014F580043CBF01F5801130BD01F000451A
:10B5000045F0FE4141F470014FF0000030BD7FEA8C
:10B51000645C1ABF194610467FEA655C1CBF0B4687
:10B52000024650EA013406BF52EA033591EA030F9E
:10B5300041F4002130BD00BF90F0000F04BF002196
:10B54000704730B54FF4806404F132044FF00005C9
:10B550004FF0000150E700BF90F0000F04BF002142
:10B56000704730B54FF4806404F1320410F00045A8
:10B5700048BF40424FF000013EE700BF42004FEAA3
:10B58000E2014FEA31014FEA02701FBF12F07F4320
:10B5900093F07F4F81F06051704792F0000F14BF1D
:10B5A00093F07F4F704730B54FF4607401F0004561
:10B5B00021F0004120E700BF50EA010208BF7047B8
:10B5C00030B54FF000050AE050EA010208BF7047AD
:10B5D00030B511F0004502D5404261EB41014FF416
:10B5E000806404F132045FEA915C3FF4DCAE4FF01A
:10B5F00003025FEADC0C18BF03325FEADC0C18BF01
:10B60000033202EBDC02C2F1200300FA03FC20FA51
:10B6100002F001FA03FE40EA0E0021FA02F114449E
:10B62000C1E600BF70B54FF0FF0C4CF4E06C1CEAB3
:10B6300011541DBF1CEA135594EA0C0F95EA0C0F28
:10B6400000F0DEF82C4481EA030621EA4C5123EA9B
:10B650004C5350EA013518BF52EA033541F48011CA
:10B6600043F4801338D0A0FB02CE4FF00005E1FB7D
:10B6700002E506F00042E0FB03E54FF00006E1FBC7
:10B6800003569CF0000F18BF4EF0010EA4F1FF040A
:10B69000B6F5007F64F5407404D25FEA4E0E6D414A
:10B6A00046EB060642EAC62141EA55514FEAC5205B
:10B6B00040EA5E504FEACE2EB4F1FD0C88BFBCF5D7
:10B6C000E06F1ED8BEF1004F08BF5FEA500E50F188
:10B6D000000041EB045170BD06F0004646EA01014E
:10B6E00040EA020081EA0301B4EB5C04C2BFD4EB80
:10B6F0000C0541EA045170BD41F480114FF0000E79
:10B70000013C00F3AB8014F1360FDEBF002001F0E6
:10B71000004170BDC4F10004203C35DA0C341BDC60
:10B7200004F11404C4F1200500FA05F320FA04F032
:10B7300001FA05F240EA020001F0004221F0004166
:10B7400010EBD37021FA04F642EB06015EEA430ED9
:10B7500008BF20EAD37070BDC4F10C04C4F1200509
:10B7600000FA04F320FA05F001FA04F240EA0200BC
:10B7700001F0004110EBD37041F100015EEA430E8D
:10B7800008BF20EAD37070BDC4F1200500FA05F2AD
:10B790004EEA020E20FA04F301FA05F243EA02032C
:10B7A00021FA04F001F0004121FA04F220EA02003B
:10B7B00000EBD3705EEA430E08BF20EAD37070BD81
:10B7C00094F0000F0FD101F00046400041EB010161
:10B7D00011F4801F08BF013CF7D041EA060195F043
:10B7E000000F18BF704703F00046520043EB0303FD
:10B7F00013F4801F08BF013DF7D043EA06037047EA
:10B8000094EA0C0F0CEA135518BF95EA0C0F0CD0F4
:10B8100050EA410618BF52EA4306D1D181EA03013A
:10B8200001F000414FF0000070BD50EA410606BF34
:10B830001046194652EA430619D094EA0C0F02D179
:10B8400050EA013613D195EA0C0F05D152EA0336BE
:10B850001CBF104619460AD181EA030101F00041DC
:10B8600041F0FE4141F470014FF0000070BD41F025
:10B87000FE4141F4780170BD70B54FF0FF0C4CF4FF
:10B88000E06C1CEA11541DBF1CEA135594EA0C0F1E
:10B8900095EA0C0F00F0A7F8A4EB050481EA030E6B
:10B8A00052EA03354FEA013100F088804FEA033352
:10B8B0004FF0805545EA131343EA12634FEA022220
:10B8C00045EA111545EA10654FEA00260EF00041E1
:10B8D0009D4208BF964244F1FD0404F5407402D233
:10B8E0005B084FEA3202B61A65EB03055B084FEAC4
:10B8F00032024FF480104FF4002CB6EB020E75EBC1
:10B90000030E22BFB61A754640EA0C005B084FEAE8
:10B910003202B6EB020E75EB030E22BFB61A754665
:10B9200040EA5C005B084FEA3202B6EB020E75EBB0
:10B93000030E22BFB61A754640EA9C005B084FEA28
:10B940003202B6EB020E75EB030E22BFB61A754635
:10B9500040EADC0055EA060E18D04FEA051545EA24
:10B9600016754FEA06164FEAC30343EA52734FEACD
:10B97000C2025FEA1C1CC0D111F4801F0BD141EA46
:10B9800000014FF000004FF0004CB6E711F4801FAB
:10B9900004BF01430020B4F1FD0C88BFBCF5E06F8B
:10B9A0003FF6AFAEB5EB030C04BFB6EB020C5FEA9B
:10B9B000500C50F1000041EB045170BD0EF0004EF0
:10B9C0004EEA113114EB5C04C2BFD4EB0C0541EA22
:10B9D000045170BD41F480114FF0000E013C90E61F
:10B9E00045EA060E8DE60CEA135594EA0C0F08BFE3
:10B9F00095EA0C0F3FF43BAF94EA0C0F0AD150EAE2
:10BA000001347FF434AF95EA0C0F7FF425AF104674
:10BA100019462CE795EA0C0F06D152EA03353FF49C
:10BA2000FDAE1046194622E750EA410618BF52EA19
:10BA300043067FF4C5AE50EA41047FF40DAF52EAED
:10BA400043057FF4EBAE12E74FEA410212F5001214
:10BA500015D211D56FF47873B3EB625212D94FEA55
:10BA6000C12343F0004343EA505311F0004F23FA3F
:10BA700002F018BF404270474FF00000704750EA94
:10BA8000013005D111F0004008BF6FF00040704751
:10BA90004FF00000704700BF4FEA4102B2F1E043AF
:10BAA00024BFB3F5001CDCF1FE5C0DD901F0004CA5
:10BAB0004FEAC0024CEA5070B2F1004F40EB8300F5
:10BAC00008BF20F00100704711F0804F21D113F121
:10BAD0003872BCBF01F00040704741F480114FEA5A
:10BAE0005252C2F11802C2F1200C10FA0CF320FAE3
:10BAF00002F018BF40F001004FEAC1234FEAD32300
:10BB000003FA0CFC40EA0C0023FA02F34FEA430369
:10BB1000CCE77FEA625307D150EA01331EBF4FF0F2
:10BB2000FE4040F44000704701F0004040F0FE400D
:10BB300040F40000704700BF7BB972B90029BEBF56
:10BB400000204FF0004106E008BF00281CBF6FF046
:10BB500000414FF0FF3000F053B882B0EC462DE9C1
:10BB6000005000F01DF8DDF804E002B00CBC704796
:10BB700053B94AB9002908BF00281CBF4FF0FF3154
:10BB80004FF0FF3000F03CB882B0EC462DE9005099
:10BB900000F01EF8DDF804E002B00CBC704700BFF6
:10BBA0002DE9F041069C154606460F46984600F0E2
:10BBB00029F805FB01F300FB0838A5FB0023B21AA6
:10BBC000434467EB0303C4E90023BDE8F08100BFF1
:10BBD0002DE9F041069C904606460F461D4600F0B2
:10BBE0005FF900FB05F5A0FB082308FB0155B21A1D
:10BBF0002B4467EB0303C4E90023BDE8F08100BFD9
:10BC0000704700BF00292DE9F043C0F2A68000264E
:10BC1000002BC0F29C80884694469E4615460446FA
:10BC20000F46002B3DD18A4259D9B2FA82F33BB17B
:10BC3000C3F120029F4020FA02F29D4017439C402E
:10BC4000290C220CB7FBF1FEA8B201FB1E7742EAD9
:10BC5000074700FB0EF3BB420AD97F190EF1FF32F2
:10BC600080F00581BB4240F20281AEF1020E2F440A
:10BC7000FF1AA4B2B7FBF1F301FB137744EA0747BD
:10BC800000FB03F0B84208D97F1903F1FF3280F0BE
:10BC9000F080B84240F2ED80023B43EA0E430022BE
:10BCA00003E08B420FD900221346341C18BF012435
:10BCB00060424FF0000565EB4501584051400019C6
:10BCC0006941BDE8F083B3FA83F2002A40F0868030
:10BCD0008B4202D3844500F2DB800123E5E712B9F1
:10BCE0000123B3FBF2F5B5FA85F000283BD1781BB0
:10BCF0004FEA154E1FFA85FC0122B0FBFEF8210C1D
:10BD00000EFB180741EA07470CFB08F3BB4207D9B3
:10BD10007F1908F1FF3102D2BB4200F2BD80884694
:10BD2000FF1AA4B2B7FBFEF30EFB137744EA0747F2
:10BD30000CFB03FCBC4507D97F1903F1FF3102D28C
:10BD4000BC4500F2A7800B4643EA0843ADE75242E8
:10BD50006FEA060663EB43035DE7404261EB410196
:10BD60004FF0FF3654E7C0F1200224FA02F107FA3F
:10BD700000F385404FEA154ED7401943B7FBFEF25A
:10BD80000B0C0EFB12771FFA85FC43EA07430CFBF2
:10BD900002F79F4204FA00F407D95B1902F1FF3061
:10BDA00074D29F4272D9023A2B44DF1B89B2B7FB8F
:10BDB000FEF80EFB187341EA03430CFB08F79F42A1
:10BDC00008D95B1908F1FF315CD29F425AD9A8F11A
:10BDD00002082B44D81B48EA02428EE7C2F1200336
:10BDE0002CFA03F10EFA02FE20FA03F741EA0E0ED6
:10BDF00008FA02F028FA03F14FEA1E453843B1FB76
:10BE0000F5F8030C05FB18111FFA8EF743EA014100
:10BE100007FB08F38B420CFA02FC09D911EB0E0167
:10BE200008F1FF3930D28B422ED9A8F102087144B3
:10BE3000C91A80B2B1FBF5F305FB131140EA0141C9
:10BE400007FB03F78F4208D911EB0E0103F1FF3016
:10BE500016D28F4214D9023B714443EA0843C91BEE
:10BE6000A3FB0C89494509D305D000221DE796465E
:10BE7000FEE6134611E794404445F6D2013BF4E751
:10BE80000346EAE78846A5E7C846D1E702468CE7BD
:10BE900013460AE7023B57E7A8F102082F443FE7A1
:10BEA0002DE9F041002B44D18A42154604464FD972
:10BEB000B2FA82F70E464FB1C7F12003B94020FA1B
:10BEC00003F602FA07F50E4300FA07F44FEA154E9F
:10BED000230CB6FBFEF0AFB20EFB106143EA014348
:10BEE00007FB00F1994209D95B1900F1FF3280F09C
:10BEF000EC80994240F2E98002382B445A1AA4B2ED
:10BF0000B2FBFEF30EFB132244EA024207FB03F7E7
:10BF1000974208D9521903F1FF3180F0D880974237
:10BF200040F2D580023B43EA004000263146BDE89E
:10BF3000F0818B4247D8B3FA83F6002E48D18B426A
:10BF400002D3824200F2CD8001203146BDE8F0816B
:10BF500012B90125B5FBF2F5B5FA85F8B8F1000F75
:10BF600077D14A1B4FEA154EAFB20126B2FBFEF065
:10BF7000230C0EFB102143EA014107FB00F38B4227
:10BF800007D9491900F1FF3202D28B4200F2BA8080
:10BF90001046C91AA4B2B1FBFEF30EFB131144EA1A
:10BFA000014407FB03F7A74208D9641903F1FF32E4
:10BFB00080F08F80A74240F28C80023B43EA004031
:10BFC0003146BDE8F081002630463146BDE8F081BB
:10BFD000C6F1200422FA04F5B3402B4320FA04FCF6
:10BFE00001FA06F721FA04F54FEA134E4CEA070767
:10BFF000B5FBFEF8390C0EFB18551FFA83FC41EA1D
:10C0000005450CFB08F1A94202FA06F204D9ED1825
:10C0100008F1FF3467D3A0466D1ABFB2B5FBFEF43A
:10C020000EFB145547EA05410CFB04FC8C4504D972
:10C03000C91804F1FF355CD32C4644EA0844CCEB24
:10C040000101A4FB0223994248D344D02046002694
:10C050006CE7C8F1200401FA08F305FA08F520FAA4
:10C0600004F7E1404FEA154E1F43B1FBFEF63A0CD0
:10C070000EFB16111FFA85FC42EA01430CFB06F287
:10C080009A4200FA08F407D95B1906F1FF3137D25A
:10C090009A4235D9023E2B449B1ABFB2B3FBFEF045
:10C0A0000EFB103347EA03430CFB00F1994207D91A
:10C0B0005B1900F1FF3221D299421FD902382B447B
:10C0C0005A1A40EA0646674650E7104616E70B46FE
:10C0D00029E7134672E7B0409042B7D2601E0026AF
:10C0E00024E7304622E7A94295D9A8F102081D4469
:10C0F00092E78C45A0D9023C19449EE71046DFE741
:10C100000E46C9E70238294443E700BF014B1868CF
:10C11000704700BFEC03FE1F02440346934202D067
:10C1200003F8011BFAE770472DE9FF4755EC104B68
:10C130000D9FDDF830A0002D0E4691461946B8BF80
:10C1400022462B4627F02007BBBF05F100431D46C2
:10C1500000232D23B8BF1446462F0B7003D0452F64
:10C1600003D1013601E0032100E0022102AB00937C
:10C1700003AB019345EC104B3246534600F02CFDC7
:10C18000472F804602D119F0010F26D0462F08EB29
:10C19000060911D198F80030302B0AD120462946E3
:10C1A0000022002302F084F818B9C6F10106CAF88B
:10C1B0000060DAF800309944204629460022002326
:10C1C00002F076F808B1CDF80C90039B4B4504D2F1
:10C1D0005A1C039230221A70F7E7039B0E9AC8EBA1
:10C1E00003034046136004B0BDE8F08773B503460F
:10C1F0000029B8BF494203F8022BB4BF2D222B22DD
:10C200000929427019DD0DF1070426460A2291FB27
:10C21000F2F502FB15113031092D04F8011D2946F4
:10C22000F4DC3031651E04F8011CB5421A460AD20E
:10C2300015F8012B03F8012BF7E730241A462144A7
:10C2400002F8024B5970101A02B070BD2DE9F04F80
:10C250008BB08B4615461E46149F044601F07CFAAF
:10C26000D0F800A0504600F015FC002308933B686E
:10C270000590073323F0070303F108029BF81880A9
:10C280003A60D3E90023CBE912239BED120B00F0B7
:10C29000B1FB01281BD1DBE912010022002302F0CF
:10C2A00011F810B12D238BF84330B54BB54FB8F1D1
:10C2B000470F88BF1F460323CBF81030DBF8003050
:10C2C00023F00403CBF800304FF000099FE09BED12
:10C2D000120B00F08FFBDBF8002068B9AA4BAB4FC4
:10C2E00022F00402B8F1470F88BF1F460323CBF8A2
:10C2F0001030CBF80020E7E7DBF804104F1C9BED73
:10C30000120B01D1062309E0B8F1670F02D0B8F192
:10C31000470F05D1002940F0C1810123CBF804303B
:10C3200007AB8DE8080108AB42F48062029300235A
:10C330000393CBF800200DF11B032046DBF804101B
:10C34000FFF7F2FE08F0DF03472B07460AD1079BF1
:10C35000D81C03DBDBF80420934237DDA8F1020888
:10C360005FFA88F8B8F1650F079915D80139424688
:10C370000BF150000791FFF739FF089A8318012A43
:10C380008146CBF8103003DCDBF80020D10738D52C
:10C390000133CBF8103034E0B8F1660F18D1002922
:10C3A000DBF8043009DDCBF810101BB9DBF80020F6
:10C3B000D20721D501330B441CE01BB9DBF8002068
:10C3C000D00701D5023315E0012313E04FF06708D1
:10C3D000079B089A934207DBDBF80020CBF810306C
:10C3E000D10709D5013305E0002BD4BFC3F1020307
:10C3F00001231344CBF81030079BCBF858304FF093
:10C4000000099DF81B3013B12D238BF843300096A3
:10C410002046594609AA2B4600F056F9013002D1B0
:10C420004FF0FF304CE1DBF800305A0505D42046D0
:10C4300029463A46DBF8103008E1B8F1650F40F2C2
:10C44000D080DBE912010022002301F031FF50B35C
:10C45000204629464E4A0123B0470130E0D0089BD0
:10C46000079A9A4209DBDBF80030D80705D4DBF8DD
:10C4700000309F0700F1108107E12046294652460F
:10C48000059BB0470130CBD00027089B013B9F4262
:10C49000EDDA204629460BF11A020123B04701309C
:10C4A000BED00137F1E7079B002B29DC2046294647
:10C4B000374A0123B0470130B2D0079B2BB9089B04
:10C4C0001BB9DBF80030D907D1D5204629465246A2
:10C4D000059BB0470130A3D04FF00008079B5B429B
:10C4E00098452046294608DA0BF11A020123B04785
:10C4F000013095D008F10108F0E73A46089BA5E025
:10C50000DBF85820089B9A42A8BF1A46002A914699
:10C5100002DC4FF0000812E0204629463A464B461E
:10C52000B0470130F5D17BE7204629460BF11A02CE
:10C530000123B04701303FF473AF08F10108DBF885
:10C540005830B9F1000FACBFC9EB03021A46904551
:10C55000EADB07EB0308079A089B9A421ADBDBF831
:10C560000030DA0716D4089A1744C8EB0703079F70
:10C57000D21B9342A8BF1346002B1F4612DC18E0C3
:10C58000D6F70000D2F70000DEF70000DAF700006F
:10C59000E2F70000204629465246059BB04701308D
:10C5A000E1D13DE7204629464246B04701303FF4FD
:10C5B00037AF4FF000080AE0204629460BF11A0277
:10C5C0000123B04701303FF42BAF08F10108079A6F
:10C5D000089B002FA3EB0203A8BFDB1B9845EBDBF6
:10C5E00045E7089A012A01DCDB0736D520462946B3
:10C5F0003A460123B04701303FF412AF20462946A6
:10C600005246059BB04701303FF40AAFDBE9120107
:10C610000022002301F04CFEE8B9089B2046294681
:10C620007A1C013B1DE0204629460BF11A0201232A
:10C63000B04701303FF4F4AE0137089B013B9F4205
:10C64000F1DB204629460BF150024B46B047013042
:10C650007FF40DAFE4E60027EFE7204629463A468F
:10C660000123B0470130ECD1DAE6204629460BF130
:10C6700019020123B04701303FF4D2AE0137DBF895
:10C680000C30099A9B1A9F42EFDBDBF80C00099BE8
:10C690009842B8BF184613E00027F0E707AB8DE8D3
:10C6A000080108AB42F48062029300230393CBF8A5
:10C6B000002020460DF11B03FFF736FD074646E636
:10C6C0000BB0BDE8F08F00BF2DE9F84391461F463F
:10C6D0008A680B69DDF820809342B8BF1346C9F819
:10C6E000003091F8432006460C4612B10133C9F8D8
:10C6F00000302368990642BFD9F800300233C9F8E8
:10C700000030256815F006051CD094F843302268E7
:10C71000003318BF012392061FD5E1185A1C3020A0
:10C7200081F84300224494F8451082F84310023304
:10C7300013E03046394604F119020123C0470130A5
:10C7400007D00135E368D9F800209B1A9D42F0DB41
:10C75000DBE74FF0FF30BDE8F8833046394604F19F
:10C760004302C0470130F4D02268D9F80050E36892
:10C7700002F00602042A08BF5D1B2269A3680CBFF1
:10C7800025EAE57500259342C4BF9B1AED184FF0CA
:10C790000009A9450ADA3046394604F11A02012394
:10C7A000C0470130D5D009F10109F2E70020BDE80A
:10C7B000F883FFFF2DE9FF410C461746227E6E2AC3
:10C7C000984606460A9B01F1430100F0AF8012D85B
:10C7D000632A23D00AD8002A00F0BC80582A40F0EF
:10C7E000CB8084F84520DFF804E257E0642A1ED0AD
:10C7F000692A1CD0C0E0732A00F0B08009D86F2AE3
:10C800002ED0702A40F0B880226842F020022260C8
:10C810003FE0752A24D0782A3BD0ADE01A68111D7C
:10C820001960136884F8423004F14205A8E02068DA
:10C830001A6810F0800F02D0101D186008E010F088
:10C84000400F02F10400186002D0B2F9003000E09D
:10C850001368002B3EDA2D225B4284F8432039E036
:10C8600020681A6810F0800F02D0101D186007E0D1
:10C8700010F0400F02F10400186001D0138800E0AE
:10C880001368227EDFF864E16F2A0CBF08220A22B7
:10C890001CE07822DFF858E184F845202268186807
:10C8A00012F0800F00F104051D6003D1550601D57B
:10C8B000038800E00368D00744BF42F020022260F2
:10C8C0001BB9226822F0200222601022002084F886
:10C8D000430002E0DFF814E10A226568A560002D3C
:10C8E000A2BF206820F00400206003B965B10D46A6
:10C8F000B3FBF2F002FB10331EF8033005F8013DE4
:10C9000003460028F4D100E00D46082A0BD1236825
:10C91000DA0708D5236962689A42DEBF302305F83A
:10C92000013C05F1FF35491B21612EE025681A689D
:10C93000606915F0800F03D0151D1D60136808E0B5
:10C9400015F0400F02F104051D60136801D0188036
:10C9500000E01860002323610D4616E01A68111DDF
:10C960001960156862682846002100F001FF08B1CF
:10C97000401B6060636804E004F1420584F84220D3
:10C9800001232361002384F84330CDF80080304632
:10C99000214603AA3B46FFF797FE013002D14FF034
:10C9A000FF301FE0304639462A462369C047013030
:10C9B000F5D023689B0705D4E068039B9842B8BF75
:10C9C00018460FE00025E368039A9B1A9D42F3DAAC
:10C9D0003046394604F119020123C0470130DED048
:10C9E0000135F0E704B0BDE8F08100BFE4F70000D6
:10C9F000F5F7000053EC102B33F0004210B510EEA9
:10CA0000100A1BD00F49A3F580148C4210D903F1F2
:10CA1000FF430C4903F5E0038B4209D9B2F5801FAF
:10CA200008D3094B9A4207D1B0FA80F0400910BDF3
:10CA3000042010BD032010BD002010BD0028E6D149
:10CA4000022010BDFFFFDF7F0000F07F0EB400B5B5
:10CA50009CB04FF40271ADF814106FF000410491D6
:10CA600007914FF6FF711DABADF81610084953F84A
:10CA7000042B029006900868019302A901F074FA51
:10CA8000029B00221A701CB05DF804EB03B07047E3
:10CA9000EC03FE1F034613F8012B002AFBD1181AE2
:10CAA00001387047044B1B6803445B7803F00303B1
:10CAB000012B08BF20307047F003FE1F2DE9F74F10
:10CAC00003690C69A3428046C0F28180013C01F1F8
:10CAD00014074FEA840E00F1140657F8245006EBB1
:10CAE0000E030193013556F82430B3FBF5F507EB3F
:10CAF0000E09C5B34FF0000A3846B446D34650F885
:10CB0000043B9AB21B0C02FB05A26B4303EB1243DE
:10CB100092B2C2EB0B02BCF800B04FEA134A12FA11
:10CB20008BF21FFA83FBDCF80030CBEB134303EBF3
:10CB3000224392B242EA034248454FEA234B4CF863
:10CB4000042BDCD956F80E306BB9019B043BB34281
:10CB50001A4602D8C8F8104005E01268043B002AC3
:10CB6000F8D1013CF3E7404601F02FF800282CDB18
:10CB7000013530464FF0000E57F8041BD0F800C0C6
:10CB80008AB2C2EB0E03090C13FA8CF3C1EB1C4200
:10CB900002EB23429BB243EA02434F454FEA224E47
:10CBA00040F8043BE8D956F8242006EB840362B928
:10CBB000043BB3421A4602D8C8F8104005E0126898
:10CBC000043B002AF8D1013CF3E7284600E00020AE
:10CBD00003B0BDE8F08FFFFF2DE9F04F456A97B035
:10CBE000824608910B921293209C8DED000B45B963
:10CBF000102000F0B5FDCAF824004560856005608E
:10CC0000C560DAF82430196859B15A684A600123BE
:10CC100093408B60504600F0FAFDDAF82430002291
:10CC20001A60019B9E4A002BBFBF01232360019B1A
:10CC300023F00043B2BF019300232360019C24F042
:10CC400000431B0D1B0593421DD1129A42F20F7334
:10CC50001360009B43B9934A934BC4F3130000281D
:10CC600014BF1846104600E08F48219B002B00F0AF
:10CC70006D85C37813B100F1080300E0C31C219A4D
:10CC8000136000F063BDDDE900890022404649469B
:10CC9000002301F00DFB054658B1129A01231360E1
:10CCA000219B002B00F0408580481860013800F07F
:10CCB0004DBD504649EC108B15A914AA01F000F89F
:10CCC000C4F30A56049056B1C9F3130343F07F51DD
:10CCD000404641F44011A6F2FF3613951DE0159B26
:10CCE000149E1E446FF482639E42ADBF009A704B47
:10CCF000009A06F21243A3BF22FA03F06D4B9B1B6E
:10CD00009B1BAABF9C4002FA03F02043FEF714FCD1
:10CD10000123A1F1F871013E13930022664BFEF747
:10CD2000CDFA59A3D3E90023FEF77CFC58A3D3E93D
:10CD30000023FEF7C5FA044630460D46FEF70CFC0C
:10CD400055A3D3E90023FEF76DFC02460B462046AF
:10CD50002946FEF7B5FA04460D46FEF775FE29464C
:10CD6000834600222046002301F0ACFA58B1584611
:10CD7000FEF7F2FB02460B462046294601F098FAE0
:10CD800008B90BF1FF3BBBF1160F0DD84B4B03EB72
:10CD9000CB03D3E90001DDE9002301F0B1FA30B1A2
:10CDA0000BF1FF3B002300E001230D9300E00D9009
:10CDB000149B9E1B731E079345BF5B420693002383
:10CDC00000234CBF07930693BBF1000F07DB079BC3
:10CDD000CDF830B05B4407930023099308E0069B2D
:10CDE000CBEB03030693CBF10003099300230C93D1
:10CDF000089B092B28D8052BC4BF043B0893089B2C
:10CE0000A3F10203CCBF00250125032B21D8DFE8C5
:10CE100003F0020E0410002300E001230A930B9B91
:10CE2000002B20DC0123039302931A4619E0002310
:10CE300000E001230A930B9B5B4403930133012B16
:10CE40000293B8BF012311E00125002308930A953E
:10CE500001E001230A934FF0FF3303930293002272
:10CE600012230B9202E00B9B03930293DAF8244007
:10CE700000226260042101F114029A4220D8626803
:10CE8000013262604900F6E761436F63A787D23FD2
:10CE9000B3C8608B288AC63FFB799F501344D33FA9
:10CEA0000000F07F07F9000010F90000E3F7000030
:10CEB000EEFBFFFF0EFCFFFF0000F83F20F9000033
:10CEC0005046616800F06EFCDAF8243020601B6880
:10CED0000593029B0E2B00F24B81002D00F0488140
:10CEE0009DED007BBBF1000F8DED107B31DDB34A72
:10CEF0000BF00F034FEA2B1702EBC303F806D3E93D
:10CF000000450CD5AE4B51EC170BD3E90823FEF7C7
:10CF1000B3FC07F00F07CDE90001032600E002266D
:10CF2000DFF89C8277B1F90708D520462946D8E971
:10CF30000023FEF777FB013604460D467F1008F10B
:10CF40000808EFE7DDE9000122462B46FEF794FCD6
:10CF50001BE0CBF10004DCB1984B994D04F00F02BB
:10CF600003EBC203DDE91001D3E90023FEF75AFB0E
:10CF7000241102264CB1E20704D5D5E9002301367D
:10CF8000FEF750FB64100835F4E7CDE9000100E03E
:10CF900002260D9BDBB1DDE9004500222046294633
:10CFA000884B01F08FF990B1029B83B1039B002B5A
:10CFB00040F3DA80294620460022834BFEF732FBFD
:10CFC0000BF1FF37CDE900010136039D01E0029D21
:10CFD0005F469DED007B30468DED0E7BFEF7BCFA83
:10CFE000DDE90E23FEF71EFB0022784BFEF768F901
:10CFF0008046A1F15079CDB90022754BDDE90E01D3
:10D00000FEF75CF942464B46CDE9000101F078F9A4
:10D01000002840F04682424609F10043DDE9000164
:10D0200001F050F9002840F036829DE0634B0A99E8
:10D030006A1E03EBC203002949D0D3E90023002074
:10D040006449FEF719FC42464B46FEF737F9DDE925
:10D050000E89CDE90001059C49464046FEF7F4FCE7
:10D060000646FEF779FA02460B4640464946FEF769
:10D0700025F9303604F8016BDDE900238046894646
:10D0800001F020F9002840F0408342464B46002042
:10D090004C49FEF713F9DDE9002301F013F90028EC
:10D0A00040F0D380059BE31AAB425DDADDE9000175
:10D0B0000022454BFEF7B6FA0022CDE90001424BB3
:10D0C00040464946FEF7AEFA80468946C4E7D3E9B2
:10D0D000000142464B46FEF7A5FA059BCDE900014B
:10D0E000DDE90E895C191D4649464046FEF7ACFC59
:10D0F0000646FEF731FA303602460B4640464946B0
:10D10000FEF7DCF805F8016BA5428046894624D17C
:10D110000022304BDDE90001FEF7D2F802460B4653
:10D120004046494601F0ECF8002840F08E80DDE9E9
:10D13000002300202749FEF7C1F802460B4640466F
:10D14000494601F0BFF878B114F8013C302B04F1E6
:10D15000FF3240F0DA821446F6E700221A4BFEF75F
:10D1600061FA80468946BFE7DDE91023CDE9002357
:10D17000159B002BC0F28B80BBF10E0F00F3878054
:10D180000E4B03EBCB03D3E900670B9B002B23DA99
:10D19000029B002B20DC40F07D81304600220C4BAE
:10D1A0003946FEF73FFADDE9002301F09FF8029DC2
:10D1B0002E46002840F0708175E100BF20F9000084
:10D1C000E8F900000000F03F0000244000001C408F
:10D1D000000014400000E03FDDE90089059C324674
:10D1E0003B4640464946FEF747FBFEF72DFC054609
:10D1F000FEF7B2F932463B46FEF714FA0B460246FA
:10D2000049464046FEF75AF805F1300E059B04F8F2
:10D2100001EBC3EB040E029B9E452BD102460B464D
:10D22000FEF74EF832463B468046894601F068F8E4
:10D2300070B94046494632463B4601F039F800286D
:10D2400000F06482EB0703D460E2BB4600E01C46BA
:10D2500014F8012C392A04F1FF3307D1059A9342BF
:10D26000F5D1302313700BF1010B13461A780132FC
:10D270001A704BE20022A44BFEF7D4F900220023DF
:10D280008046894601F014F80028A8D03EE20A9AA8
:10D29000002A32D0089A012A0ADC139A12B103F24A
:10D2A000334302E0149BC3F13603099D069C18E04A
:10D2B000029B5D1E099BAB42BFBF099B0995EA1A01
:10D2C0000C9BB6BF9B185D1B0C93029BB8BF00253F
:10D2D000002BB9BF069B029A069C029BBCBF9C1AFE
:10D2E0000023069A1A440692079A50461A440121CE
:10D2F000079200F02EFB064602E0099D069C0A9E5E
:10D3000064B1079B002B09DDA342069AA8BF234600
:10D31000D21A0692079AE41AD31A0793099B002B94
:10D3200020DD0A9BC3B1002D10DD31462A46504650
:10D3300000F0AAFB06463146049A504600F012FB64
:10D3400004990746504600F062FA0497099B5A1B5D
:10D3500008D05046049902E00499099A504600F01A
:10D3600093FB04905046012100F0F3FA0C9B002B34
:10D3700005460ADD29461A46504600F085FB089B03
:10D38000012B054604DD00271BE0089B012B13DC65
:10D39000009B8BB9019BC3F313037BB9019B23F063
:10D3A00000473F0D3F0557B1069B01330693079B8E
:10D3B00001330793012702E0002700E0009F0C9B48
:10D3C00043B12B6905EB8303186900F075FAC0F1CE
:10D3D000200000E00120079B184410F01F0008D037
:10D3E000C0F12003042B02DDC0F11C0002E008D0D4
:10D3F00018461C30069B03440693079B03440444D1
:10D400000793069B002B05DD504604991A4600F051
:10D4100089FB0490079B002B05DD294650461A46E0
:10D4200000F080FB05460D9BEBB10498294600F007
:10D43000CCFB002817DA0023504604990A2200F09A
:10D44000FDF90A9B04900BF1FF3B002B00F070816B
:10D450003146002350460A2200F0F0F9039B002BCE
:10D46000064633DC6DE1029B002B26DC089B022B79
:10D4700023DD029B0393039B73B929460522504683
:10D4800000F0DCF905462946049800F09EFB0028D0
:10D4900009DC01E000252E460B9B059C6FEA030B7F
:10D4A00008E0BB462E46059B059A5C1C3123137091
:10D4B0000BF1010BB146002614E10A9B23B9029B34
:10D4C0000393059F049CCCE0029B0393002C05DD95
:10D4D00031465046224600F025FB0646B7B171683A
:10D4E000504600F05FF932690232044606F10C0141
:10D4F00092000C3000F04BF950462146012200F01A
:10D5000011FB814603E000BF00002440B146059FA7
:10D51000049C29462046FFF7D1FA3146069000F1D7
:10D520003008204600F051FB4A46029029465046FA
:10D5300000F067FBC26803463AB9194620460493D7
:10D5400000F043FB049B024600E0012250461946CE
:10D55000049200F05CF9049AA2B9089B93B9009B6D
:10D5600003F0010373B9B8F1390F3B46049440D07E
:10D57000029B002BC8BF069B07F10104C8BF03F143
:10D5800031083DE0029B002B04DA002AC4460494D3
:10D5900008DC21E024D1089B13BB009B03F00103AE
:10D5A000F3B9F2E72146012250460297CDF80080F8
:10D5B00000F0B8FA2946049000F007FB0028DDF8D7
:10D5C00000C0029B03DC07D118F0010F04D0B8F1B2
:10D5D000390F0ED008F1010C7C1C87F800C081E0E7
:10D5E000002A07F101020EDDB8F1390F3B46049421
:10D5F00003D1392201371A7057E0144608F10108A7
:10D6000087F800806EE0059B02F8018CD31A17465C
:10D61000039A93423AD021460A220023504600F052
:10D620000DF94E450446314650464FF00A024FF080
:10D63000000304D100F002F90646814669E700F0D4
:10D64000FDF8494606460A225046002300F0F6F847
:10D6500081465EE7214650460A22002300F0EEF89C
:10D66000044620462946FFF729FA00F1300807F85A
:10D67000018B059B039AFB1A9342EBDB059B012A66
:10D68000ACBF9B180133B1461F460026214601223C
:10D69000504600F047FA2946049000F096FA002818
:10D6A00003DC16D118F0010F13D03C4614F8013CEE
:10D6B000392B04F1FF3209D1059B9A4204D10BF1B9
:10D6C000010B3123059A02E01446EFE70133137092
:10D6D00008E03C4614F8013C302B04F1FF3201D144
:10D6E0001446F7E75046294600F091F8B9F1000FCB
:10D6F0000CD02EB14E4503D05046314600F087F88D
:10D700005046494600F083F800E0BB465046049975
:10D7100000F07DF80023129A23700BF101031360CF
:10D72000219B1BB11C6001E00A480FE005980DE049
:10D73000039B002B3FF7C5AE089B022B3FF79BAE28
:10D74000BFE6089B022B3FF796AEBFE617B0BDE8D9
:10D75000F08F00BFE2F7000000487047F403FE1F9F
:10D76000024B0146186800F04FBB00BFEC03FE1FE0
:10D7700010B5C9B202449042034606D01C788C42D0
:10D7800000F10100F7D1184610BD002010BD10B502
:10D79000431E0A44914204D011F8014B03F8014F93
:10D7A000F8E710BD70B5456A04460E463DB9102035
:10D7B000FFF7D6FF6062456085600560C560656AF9
:10D7C000EB6843B1636ADB6853F8260078B10268FE
:10D7D00043F8262017E020460421212200F0C2FA57
:10D7E000636AE860DB68002BECD1002070BD01218A
:10D7F00001FA06F56A1D2046920000F0B3FA0028EF
:10D80000F3D04660856000230361C36070BD70B5CE
:10D81000446A06460D463CB91020FFF7A1FF70622E
:10D82000446084600460C4603DB1736A6A68DB6808
:10D8300053F82210296043F8225070BD2DE9F041C1
:10D840000F69984606460C4601F1140E0023DEF8D7
:10D85000000085B2010C02FB0585514301EB154127
:10D860000133ADB24FEA1148BB4205EB01414EF81E
:10D87000041BECDBB8F1000F1BD0A3689F4212DB46
:10D88000616830460131FFF78DFF2269023204F1F1
:10D890000C01054692000C30FFF779FF2146304617
:10D8A000FFF7B5FF2C4604EB87030137C3F814805C
:10D8B00027612046BDE8F081030C1B0413B9000466
:10D8C000102300E0002310F07F4F04BF0002083354
:10D8D00010F0704F04BF0001043310F0404F04BF3C
:10D8E00080000233002803DB420003D5581C704738
:10D8F0001846704720207047036813F007020BD0CA
:10D90000D90722D49A074BBF5B089B0803600360CA
:10D910004CBF01200220704799B209B91B0C10229C
:10D9200013F0FF0F04BF1B0A0832190704BF1B09BD
:10D930000432990704BF9B080232D90702D45B085E
:10D9400005D0013203601046704700207047202048
:10D95000704710B50C460121FFF724FF01224461F6
:10D96000026110BD2DE9F74F14460A6923699A42F6
:10D97000B8BF0B468846BCBFA0461C46D8F81070FE
:10D98000D4F81090D8F80830D8F8041007EB09063E
:10D990009E42C8BF0131FFF705FF00F1140505EBFA
:10D9A000860C2B46634503D2002243F8042BF9E78B
:10D9B00004F1140208F1140102EB890301EB87075B
:10D9C0000093009B01929A4257D2B2F800B0BBF18B
:10D9D000000F23D08946AE464FF0000859F8044B9B
:10D9E000BEF800A0A3B20BFB03A34FEA144ADEF873
:10D9F000004043444FEA14480BFB0A8404EB1344F1
:10DA0000F2469BB243EA04434F454FEA14484AF8B2
:10DA1000043B01D9D646E1E7CEF80480019BB3F878
:10DA200002A00432BAF1000F21D02B682C4689469F
:10DA30004FF00008B9F800E0B4F802B00AFB0EBEDF
:10DA4000F044A3469BB243EA08434BF8043B59F821
:10DA5000043BB4F804E01B0C0AFB03E303EB18439C
:10DA6000B9454FEA134801D25C46E3E763600435E9
:10DA7000A7E75CF8043D13B9013E002EF9DC06610E
:10DA800003B0BDE8F08FFFFF12F003032DE9F04172
:10DA900006460F46154607D0013B214A52F823207F
:10DAA0000023FFF7CBFE0746AD1035D0746A3CB9B2
:10DAB0001020FFF755FE7062446084600460C4600B
:10DAC000D6F82480D8F808407CB9304640F271215D
:10DAD000FFF73FFF0023C8F808000446036004E096
:10DAE0006D1019D0206870B10446EB07F8D539469F
:10DAF00022463046FFF736FF394680463046FFF76C
:10DB000086FE4746ECE7304621462246FFF72AFFCD
:10DB1000002320600360E7E73846BDE8F08100BFDE
:10DB200010FA00002DE9F0470C464FEA621A23690B
:10DB300049680AEB0309A3680746164609F101057F
:10DB40009D4202DD01315B00FAE73846FFF72AFE0D
:10DB50000023804600F11401534504DA002241F805
:10DB600023200133F8E72AEAEA73206901EB8303F3
:10DB700016F01F0204F1140101EB800E14D0C2F163
:10DB8000200C00200E68964030439A4643F8040B60
:10DB900051F8040B714520FA0CF0F3D3CAF80400D5
:10DBA00048B109F1020506E0043B51F8042B43F8A3
:10DBB000042F7145F9D3013D3846C8F8105021466D
:10DBC000FFF725FE4046BDE8F08703690A699B1A06
:10DBD00010B511D192001430143183180A4453F84F
:10DBE000044D52F8041D8C4202D007D3012010BD11
:10DBF0008342F4D8002010BD184610BD4FF0FF300E
:10DC000010BD2DE9F84307460C4608461146154657
:10DC1000FFF7DBFF061E08D138463146FFF7C2FD8D
:10DC2000012303614661BDE8F883BCBF23462C464F
:10DC300038466168BABF1D4601260026FFF7B2FDCF
:10DC40002B69C660266905F11409143404EB8607B4
:10DC500009EB830800F114054FF0000C54F8043B65
:10DC600059F8042B1CFA83F11FFA82FE120CCEEB3A
:10DC70000101C2EB134303EB214389B24FEA234C6A
:10DC8000C84541EA0343A64645F8043BE6D8BE45ED
:10DC90000ED25EF8042B1CFA82F4120C02EB244222
:10DCA000A4B24FEA224C44EA024245F8042BEEE7C4
:10DCB00055F8043D0BB9013EFAE70661BDE8F8836B
:10DCC0002DE9F3410F46012155EC104B1646FFF7A5
:10DCD00069FDC5F31303C5F30A5580460DB143F43E
:10DCE00080130193ECB102A840F8084DFFF704FE41
:10DCF000009B50B1019AC0F1200102FA01F10B43DF
:10DD0000C240C8F81430019201E0C8F81430019BF9
:10DD1000C8F81830002B14BF02240124C8F81040A2
:10DD200009E001A8FFF7E8FD0124019BC8F81430C1
:10DD3000C8F81040203035B1A5F2334505443D60A8
:10DD4000C0F1350009E008EB8403A0F232403860EE
:10DD50001869FFF7B1FDC0EB44103060404602B0D7
:10DD6000BDE8F08138B502FB01F4214600F04CF823
:10DD7000054618B100212246FEF7CEF9284638BDE7
:10DD800030B500293DD051F8042C0B1F1D49002A45
:10DD9000B8BF9B180A680C4612B95A600B6030BDB8
:10DDA00093420DD219685818904201BF5A58521820
:10DDB0001A6042685A60236030BD994203D80A460F
:10DDC00051680029F9D1146815199D420AD11B68C0
:10DDD0002344D0188842136013D1086803441360A9
:10DDE0004B680DE002D90C23036030BD1C68181984
:10DDF000884204BF08684968596004BF0019186068
:10DE0000536030BD9C0AFE1F70B5CC1C24F0030487
:10DE100008340C2C38BF0C24002C064603DA0C23E3
:10DE20003360002070BD8C42F9D3204A136810463D
:10DE30001946A1B10A68121B0ED40B2A03D90A6035
:10DE40008B188C501FE08B420DBF5A684A685A608D
:10DE5000026018BF0B4616E00B464968E9E7144D0F
:10DE60002B681BB9304600F071F928603046214616
:10DE700000F06CF9421C0346D1D0C51C25F0030507
:10DE800085420AD11C6003F10B001A1D20F0070027
:10DE9000821A0AD05142995070BD3046E91A00F0FA
:10DEA00055F90130BBD02B46ECE770BD9C0AFE1F34
:10DEB000980AFE1F2DE9F0478E68B34282460C4651
:10DEC0009046994640D38A8912F4906F3AD02568DB
:10DED00009696F1A6569022305EB450595FBF3F5A2
:10DEE0007B1C4B449D4238BF1D4653050FD5294628
:10DEF000FFF78AFF064698B121693A46FFF747FCCB
:10DF0000A38923F4906343F08003A38113E02A469E
:10DF100000F047F9064670B950462169FFF730FF17
:10DF20000C23CAF80030A38943F04003A3814FF0CB
:10DF3000FF30BDE8F087266165613E44ED1B266039
:10DF4000A5604E46B14500D24E4632462068414655
:10DF500000F00CF9A3689B1BA36023681E44266095
:10DF60000020BDE8F087FFFF2DE9F0439DB0064695
:10DF700003938B891C060D4690460CD50B6953B94B
:10DF80004021FFF741FF2860286110B90C2333605E
:10DF9000CCE040236B610023099320238DF82930C6
:10DFA00030238DF82A3043461C4613F8012B1AB94A
:10DFB000B4EB08090FD002E0252AF5D1F8E7304686
:10DFC000294642464B46FFF775FF013000F0A98015
:10DFD000099B4B4409932378002B00F0A280002377
:10DFE0004FF0FF3204930793059206938DF8533058
:10DFF0001A9304F101084446DFF848912178484615
:10E000000522FFF7B5FB08F10108049B30B1C9EB0D
:10E0100000000122824013430493ECE7D80644BF7A
:10E0200020228DF85320190744BF2B228DF853204E
:10E0300022782A2A02D0079923460EE0039A111D5E
:10E0400012680391002ABBBF524243F002030792B9
:10E050000792B8BF049301340AE01C4601332278CA
:10E06000303A092A03D80A2000FB0121F5E707917D
:10E0700023782E2B1AD163782A2B0AD1039B1A1DE1
:10E080001B680392002BB8BF4FF0FF330234059397
:10E090000CE0611C00220C4601312378303B092B37
:10E0A00003D80A2000FB0232F5E70592DFF89880DA
:10E0B000217840460322FFF75BFB38B1049AC8EB96
:10E0C00000004023834013430493013421781A480D
:10E0D0008DF82810062204F10108FFF749FB88B1EA
:10E0E000164B33B9039B073323F00703083303931D
:10E0F00013E003AB0093304604A92A46104BFEF709
:10E10000A5F807E003AB0093304604A92A460C4B60
:10E11000FEF750FB421C074603D0099B3B44099382
:10E1200041E7AB895B0601D4099801E04FF0FF306D
:10E130001DB0BDE8F08300BF26FA00004DC200000C
:10E14000B5DE00001CFA000022FA000038B5064CCB
:10E150000023054608462360FBF7E0F9431C02D183
:10E16000236803B12B6038BD1C11FE1F814210B51E
:10E1700001EB020301D3421E0BE09842FBD281184F
:10E18000D21AD34204D013F8014D01F8014DF8E73B
:10E1900010BD994204D011F8014B02F8014FF8E785
:10E1A00010BDF8B5074615460E4621B91146BDE823
:10E1B000F840FFF729BE1AB9FFF7E2FD2846F8BD7F
:10E1C00000F015F8A8420ED238462946FFF71CFE8B
:10E1D000044650B131462A46FFF7D9FA384631464F
:10E1E000FFF7CEFD01E03046F8BD2046F8BD51F8FE
:10E1F000040C0028BEBF091851F8043CC0180438AC
:10E200007047FFFF4FF0FF3C06E000BF4FF0010CEE
:10E2100002E000BF4FF0010C4DF804CD4FEA410C75
:10E220007FEA6C5C4FEA430C18BF7FEA6C5C1BD042
:10E2300001B050EA410C0CBF52EA430C91EA030FC3
:10E2400002BF90EA020F0020704710F1000F91EA20
:10E25000030F58BF994208BF90422CBFD8176FEAEE
:10E26000E37040F0010070474FEA410C7FEA6C5CBC
:10E2700002D150EA013C07D14FEA430C7FEA6C5CC3
:10E28000D6D152EA033CD3D05DF8040B704700BFEF
:10E290008446104662468C461946634600E000BF3D
:10E2A00001B5FFF7B7FF002848BF10F1000F01BD0F
:10E2B0004DF808EDFFF7F4FF0CBF012000205DF8DA
:10E2C00008FB00BF4DF808EDFFF7EAFF34BF01205F
:10E2D00000205DF808FB00BF4DF808EDFFF7E0FFF8
:10E2E00094BF012000205DF808FB00BF4DF808ED49
:10E2F000FFF7CEFF94BF012000205DF808FB00BFB0
:10E300004DF808EDFFF7C4FF34BF012000205DF891
:10E3100008FB00BF4275696C7420776974682052ED
:10E32000656E657361732053796E65726779202815
:10E33000544D2920536F6674776172652050616374
:10E340006B6167652076657273696F6E20312E355B
:10E350002E332B6275696C642E64633334386432F7
:10E360006132323336000000312E352E330000008A
:10E3700000030501F8B500BFF8BC08BC9E46704715
:10E38000F8B500BFF8BC08BC9E4670470600000008
:10E390000100080001010000100001000000180049
:10E3A0000000010120000000000040000100000109
:10E3B0006000000001028000000000010001010077
:10E3C00000028001000001030002000000020004BE
:10E3D00001000003000800000003FFFF0004081014
:10E3E000E90B00005D0A0000A11300008D1400007D
:10E3F000A109000045120000ED07000021110000F6
:10E4000004000101010010000101010140000101AF
:10E4100001020001010101030B010401691B00005D
:10E4200099190000D5190000111A0000511A0000B6
:10E43000C1170000FFFFFFFF952E0000BD2C00005C
:10E44000D935000089360000C92D0000FD280000E4
:10E45000AD2700000C01040155410000754000008B
:10E46000CD4100004D3E0000F53C0000853D000020
:10E470001D4000005D3C0000F93D0000513F0000E0
:10E48000CD3C00004D3D0000A53C0000193F0000C0
:10E49000E13D0000020403040404FFFF854700007F
:10E4A000DD42000005430000114600002D4300003E
:10E4B0005D460000E1460000514300007945000040
:10E4C000D94300000A010401000103070F1F3F7F29
:10E4D000000101020102020301020203020303041C
:10E4E00001020203020303040203030403040405FC
:10E4F00001020203020303040203030403040405EC
:10E5000002030304030404050304040504050506CB
:10E5100001020203020303040203030403040405CB
:10E5200002030304030404050304040504050506AB
:10E53000020303040304040503040405040505069B
:10E54000030404050405050604050506050606077B
:10E55000594D0000814C0000A94C0000154E0000F0
:10E56000D94C0000454D000006010301ED500000AC
:10E57000BD500000595000006D5000008150000057
:10E5800095500000A950000003010201E153000072
:10E59000615500008D520000755100006D51000062
:10E5A00071510000BD51000035520000A95100001A
:10E5B000115300000A01020106010401F556000092
:10E5C0000D580000515600008D560000C156000045
:10E5D0002D56000041560000010002000400FFFF1C
:10E5E000010002000300FFFF000001000200FFFF26
:10E5F000000001000000020055630000016C0000F3
:10E6000055670000ED680000896A00000964000099
:10E61000ED6900002D660000316400001565000002
:10E6200065650000796500008D650000A16500004A
:10E63000B9650000CD650000396E0000996D0000DD
:10E64000E96D00000D6F0000B56E0000E16E000086
:10E650005D6F00007D6F00009D6F0000C16F0000C6
:10E660004163000004FF000201FFFFFF0C010301F2
:10E6700071770000997C00004D7D0000557C000002
:10E680001D7C0000C97D00005176000005010201DB
:10E690004D8800003984000031800000798000003E
:10E6A000AD800000D580000035810000758100003C
:10E6B000E97F0000E57F000035830000D581000080
:10E6C000D17F00000801090140420F000000000056
:10E6D00040420F00000000000400000002000000A3
:10E6E000002D310100127A0030040201020A1E02DC
:10E6F000D0FE010002000310040000001C00000016
:10E7000013000000030E0010FFFFFFFFFFFFFFFFDD
:10E71000FFFFFFFFFFFFFFFF5237465337473237F8
:10E72000483341303143464257533134343141311B
:10E73000303000000000000002906400F000000093
:10E7400001000810F3E0BFB6057933498B43F24F5F
:10E750001693A05D1E7A1DD8700D7A8242786A5E8B
:10E76000C35C0B190400501100000040FFFF0008BB
:10E77000FFC110081FFF1B057F0028073F002F0661
:10E780003E8047804C806A0064806B008200568027
:10E790006E00BD80B08083006F005B8070007200EF
:10E7A00071007300740075008A8086808D80CF8030
:10E7B00076006C006D00B5807B007A007C00A08044
:10E7C00077007800790090809A80978084009D80FF
:10E7D000A3807D00D580D880A6808500AD80A980EB
:10E7E000DE807E007F0080008100000006070210AE
:10E7F00000000000FFFF00000020000000010000FA
:10E8000000000100FFFF3F00008000000001000049
:10E810000607011000001040FFFF104040000000FC
:10E82000040000000A000410070B0B0F0000FE1F7D
:10E83000FFFFFF1F00000020FFFF03200000042057
:10E84000FFFF072000E00F20FFFF0F20010700104F
:10E850000800400000500040080301100052004032
:10E86000015F00100100000C00000040011F0010BB
:10E8700001000001000C0040000300100100000135
:10E88000000D0040010700100100000100E07F4082
:10E89000000300100100100000C07F40E0010310E1
:10E8A000B0010310C0010310200003105400031036
:10E8B00030000F1070040310000807101000031040
:10E8C000460403104105031040070310000C031019
:10E8D000400407104204031044040310D005031041
:10E8E000E0050B10F00503100F0707104009031097
:10E8F000000E0711400E0310600E03106000071099
:10E9000010040310B0070710800403100200001069
:10E91000030000010030054007030300000F001052
:10E920000A00200000000740000F00100200000154
:10E9300000200740020000100E0000010080074088
:10E940003F1F1F1F0F0F0F0F0707070707070000C5
:10E950000003001001001000F08F074000030010BA
:10E960000400000100200440000300100200000128
:10E970000040084000070010060000010050084059
:10E980000007001002000010000005400007001002
:10E9900002000004002006400200001002000002F5
:10E9A00000400640070700000007001102000001B8
:10E9B00000E0044001030010C0000400000804400F
:10E9C00008030110000D04400400021002000002C0
:10E9D00000C005402B2B00007F007F003F000F0090
:10E9E0007F0067001F000700040001100C002000DA
:10E9F00000000440070B0B0B0B0303030301010191
:10EA0000FFCFFFC3FFFFFFFFFF30FF30FFFFFF3FE0
:10EA1000FFFFFFFFFFFF7F18FFFF3F7FFFFF3F7FED
:10EA2000FF3F0300FFFF0000FFFF0000FF000000AA
:10EA30000400021001002000001008400300000044
:10EA4000FFFFFFFF030003000003001001000002AE
:10EA500000000064011700100100001000000940D0
:10EA6000001D00200100000200000640010300100C
:10EA700001000001004406400103001001000001F4
:10EA80000045064001030010010000080050064048
:10EA9000000300100200000400580640FFFFFFFFC3
:10EAA000FFFFFFFFFFFFFFFFFFFFFFFFFFFFFFFF76
:10EAB000FFFFFFFFFFFFFFFFFFFFFFFFFFFFFFFF66
:10EAC000FFFFFFFFFFFFFFFFFFFFFFFFFFFFFFFF56
:10EAD000FFFFFFFFFFFFFFFFFFFFFFFFFFFFFFFF46
:10EAE000FFFFFFFFFFFFFFFFFFFFFFFFFFFFFFFF36
:10EAF000727E30A21CE001400070044004700440AB
:10EB000008700440FFFFFFFFFFFFFF3636FFFF8E58
:10EB1000FFFFFFFFFF808D815F4953839FFFFFFF52
:10EB2000FFFFFFFFD0F4D6FFDCFFFFFFFFFFFFE595
:10EB3000EEFFFFC34245466B8C8988FFFFFFFFFF56
:10EB4000FFFFFFFF4F6D82848685FFFF00050000F9
:10EB5000010002000800FFFF0100000000000000AB
:10EB6000000000000000000058E400000803FE1F41
:10EB7000810100FF0000000024ED00000000000003
:10EB80004803FE1FA50100FF0000000048ED000043
:10EB9000000000009C0BFE1F10ED00008CE5000043
:10EBA000380CFE1FB4ED00008CE5000000000200F0
:10EBB000000083200201FFFF0000000000000000B1
:10EBC000F0EB00000000000002000000A086010041
:10EBD0004000010000000C0C0C0C0000A0EB000039
:10EBE00020EE000065A40000E8ED000000EC00004D
:10EBF000C00AFE1FACEB000060ED000090E60000D4
:10EC000001FFFFFF3803FE1F6D0000FF0000000042
:10EC100020EE000000000000300CFE1F74EE00002B
:10EC2000BCE500000000000000FFFFFF0200000044
:10EC300000C2010000000000050C0CFF00000000F5
:10EC400024ED0000B5B0000050EC0000F0EC000036
:10EC5000480CFE1F2CEC0000E0E30000060C0C0C3E
:10EC60000C0000000100000040420F0094EB000087
:10EC700074ED0000D5A1000080EC00001CEE000047
:10EC8000280DFE1F5CEC00001CE40000BC0CFE1F05
:10EC90002CEE00001CE40000000000000100000059
:10ECA000060000003200000001000A0169B2000005
:10ECB000C8ED000024EC0000000C0C0C0C0001015D
:10ECC0000100000040420F0030ED00003CED00006C
:10ECD000599D000004ED000018EE00002803FE1FFF
:10ECE000A40100FF0000000054ED0000000000003F
:10ECF0000000010001000000000000000100000011
:10ED0000D00700001C0BFE1FB8EC00001CE4000044
:10ED10001803FE1F990100FF0000000094EB0000A3
:10ED200000000000040BFE1F6CEB00008CE50000EF
:10ED3000AC0BFE1F50EE00008CE50000F40AFE1F35
:10ED4000D4ED00008CE50000A00AFE1F80EB00005F
:10ED50008CE50000780CFE1FDCEC00008CE5000068
:10ED60001F0000300000000000000000070000301D
:10ED700000180000F80CFE1FF4ED00008CE5000008
:10ED800000000000C002FE1F000000002000000084
:10ED9000C001FE1F000000004D99000068EE000059
:10EDA00010EE00000C0C0C00140BFE1F08EE00000F
:10EDB000BCE500005803FE1F6E0000FF00000000CD
:10EDC000A0EB0000000000009C05FE1F98EC000076
:10EDD0009CE40000D802FE1F740100FF0000000048
:10EDE0003CED000000000000CC0BFE1FC8EB000053
:10EDF00038E40000C802FE1F980100FF0000000078
:10EE000074ED00000000000001000001000000009F
:10EE100000000000E802FE1F01FFFFFF00FFFFFFF0
:10EE2000200CFE1F04EC00008CE50000080C0C0C0C
:10EE30000C000101010000008096980048ED0000E0
:10EE400054ED0000D5A500008CEC000064EE00003D
:10EE50006803FE1F750100FF0000000030ED000098
:10EE60000000000000FFFFFF6805FE1F80ED0000AE
:10EE700070E6000000000001000000002200000019
:10EE800084EE000000800000000000000080000010
:10EE900001000000008000000E0000000080000063
:10EEA0000F00000000000104000100000000010448
:10EEB0000101000000000104020100000500000043
:10EEC000030100000000010404010000000001042F
:10EED000050100000000010406010000050000001B
:10EEE000070100000000010008010000000001000F
:10EEF00009010000000001000A01000000000104F7
:10EF00000C010000000001040D010000050C0000D0
:10EF100002020000050C000003020000050C0000C6
:10EF2000070200000000010000030000000C0104C3
:10EF300004030000000C010405030000000C0104A0
:10EF400006030000050C00000D0300000000011086
:10EF50000104000000040110020400004000010749
:10EF60000B050000400001070C0500001000000028
:10EF70000C060000100000000D0600000400000058
:10EF80000C0700000500000000080000040000005D
:10EF900001080000675F616463302E705F61706913
:10EFA0002D3E6F70656E0000675F616463302E7088
:10EFB0005F6170692D3E7363616E43666700000098
:10EFC000675F616463302E705F6170692D3E7363AB
:10EFD000616E53746172740063616E5F696E69740F
:10EFE00020705F6170692D3E6F70656E00000000DB
:10EFF000690943414E5F4556454E545F4552525F45
:10F000004255535F4F46460D0000000069094341D9
:10F010004E5F4556454E545F4255535F5245434FF0
:10F02000564552590D000000690943414E5F45564F
:10F03000454E545F4552525F504153534956450D1A
:10F0400000000000690943414E5F4556454E545F3C
:10F050004552525F5741524E494E470D0000000045
:10F06000690943414E5F4556454E545F4D41494CF9
:10F0700059424F585F4F56455257524954450D001B
:10F08000690943414E5F4556454E545F554E4558BC
:10F090005045435445440D0063616C6C6261636B81
:10F0A0005F63616E20496E76616C69642043414EF6
:10F0B0002063616C6C206261636B206368616E6EBB
:10F0C000656C2C2027302720657870656374656433
:10F0D0002000000063616C6C6261636B5F63616E52
:10F0E000206170692D3E7265616400FF6672616D1A
:10F0F0005F77726974652070696E577269746520F4
:10F100004652414D2053534C206C6F770000000055
:10F110006672616D5F77726974652061706957729C
:10F120006974652068656164657200006672616D6E
:10F130005F777269746520617069577269746520C0
:10F1400064617461000000006672616D5F777269CE
:10F1500074652070696E5772697465204652414D1E
:10F160002053534C20686967680000006672616D27
:10F170005F726561642070696E57726974652046BC
:10F1800052414D2053534C206C6F77006672616D75
:10F190005F72656164206170695772697465206887
:10F1A00065616465720000006672616D5F72656121
:10F1B000642061706952656164206461746100005B
:10F1C0006672616D5F726561642070696E57726905
:10F1D0007465204652414D2053534C20686967683E
:10F1E000000000006366675F6C6F61642C206672CC
:10F1F000616D5F72656164006366675F7361766508
:10F200002C206672616D5F77726974650000000082
:10F21000737461727475705F6C6F61642C206672B8
:10F22000616D5F7265616400737461727475705FA3
:10F23000736176652C206672616D5F7772697465A3
:10F2400000000000636865636B5F6672616D2C206F
:10F250006672616D5F7772697465310063686563BA
:10F260006B5F6672616D2C206672616D5F726561A5
:10F2700064310000636865636B5F6672616D2C20AA
:10F280006672616D5F777269746532006368656389
:10F290006B5F6672616D2C206672616D5F72656175
:10F2A00064320000636865636B5F6672616D2C2079
:10F2B0006672616D5F777269746533006368656358
:10F2C0006B5F6672616D2C206672616D5F72656145
:10F2D000643300006672616D5F696E697420675FF8
:10F2E0007370695F6672616D2E705F6170692D3E2B
:10F2F0006F70656E00FFFFFF675F7370695F656E1B
:10F30000632E705F6170692D3E6F70656E00FFFF48
:10F310004552524F525F5452415020256C69203A59
:10F320002025730A000000004552524F525F54528C
:10F3300041500A00657272203D20256C690A000068
:10F34000446562756720256C69203A2025730A00A0
:10F350004656207F0608010600000000000000005D
:10F360005F000000000700070000147F147F1400F6
:10F37000242A7F2A1200231308646200364956208B
:10F380005000000807030000001C2241000000415B
:10F39000221C00002A1C7F1C2A0008083E080800C6
:10F3A0000080703000000808080808000000606055
:10F3B00000002010080402003E5149453E00004272
:10F3C0007F4000004261514946002141494D3300D0
:10F3D0001814127F10002745454539003C4A494919
:10F3E00030004121110907003649494936000649D4
:10F3F00049291E000000140000003C428185864718
:10F4000000081422410014141414140000412214A2
:10F4100008000201510906003E415D594E007C1270
:10F4200011127C007F49494936003E41414122008A
:10F430007F4141413E007F49494941007F09090917
:10F4400001003E4149497A007F0808087F000041D9
:10F450007F4100002040413F01007F08142241000D
:10F460007F40404040007F021C027F007F04081064
:10F470007F003E4141413E007F09090906003E41AF
:10F4800051215E007F091929460026494949320069
:10F4900001017F0101003F4040403F001F2040200C
:10F4A0001F003F4038403F0063140814630003040A
:10F4B00078040300615149454300007F4141410008
:10F4C000020408102000004141417F0004020102B3
:10F4D0000400404040404000000307080000205462
:10F4E000545478007F284444380038444444280069
:10F4F000384444287F0038545454180000087E09CA
:10F50000020018A4A4A47C007F080404780000442E
:10F510007D4000002040403D00007F102844000056
:10F5200000417F4000007C04780478007C080404DB
:10F530007800384444443800FC1824241800182467
:10F540002418FC007C080404080048545454240087
:10F5500004043F4424003C4040207C001C20402008
:10F560001C003C4030403C004428102844004C9093
:10F5700090907C004464544C4400000836410000E4
:10F58000000077000000004136080000020102047C
:10F5900002003C2623263C00690976657273696F78
:10F5A0006E2000006909496E697469616C697A6945
:10F5B0006E6720636F6E66696775726174696F6EDE
:10F5C0000D00000076657273696F6E006F097665D5
:10F5D0007273696F6E2025730D0000006D677300F4
:10F5E0006F0925690D00000066696E650000000066
:10F5F000656E636F6465725F6F6E00006F096F66A2
:10F60000660D00006F096F6E0D000000636F756E70
:10F61000746572726573657400000000636F756EC7
:10F6200074657277726974650000000063686563D1
:10F630006B5F6672616D000065096572726F723A88
:10F640002025690D00000000726561645F737461BC
:10F6500072747570000000006F090000256C69204D
:10F66000000000003F0000006F090A0023204669E7
:10F67000726D776172652D56657273696F6E3A208F
:10F6800025730A002320436F6D6D616E6420636FE4
:10F69000756E7465726964203C696420312E2E3168
:10F6A000363E2073746F72657320636F6E66696790
:10F6B000207065726D616D656E746C792E0A000044
:10F6C000636F756E74657269642025690A000000B5
:10F6D00068656C70000000007072696E74636F6E14
:10F6E00066696700636F756E746572696400000017
:10F6F0006F09636F756E7465726964207365742039
:10F70000746F2025690D000073656E6473746174F5
:10F71000757300007535706F73203D20252E32669D
:10F7200020560A006935706F73203D20252E336600
:10F7300020410A0075356E6567203D20252E326612
:10F7400020560A00753573656E736F72203D202553
:10F750002E326620560A000074656D706572617401
:10F76000757265203D20252E316620430D00000076
:10F7700075706461746500006F0D000065096E6F3F
:10F78000742076616C696420636F6D6D616E643A9C
:10F790002000FFFF4353312030312D30315F3231B3
:10F7A0003130313320202020202020202020202014
:10F7B00020202000675F74696D65725F316B687A25
:10F7C0002E705F6170692D3E6F70656E00000000E5
:10F7D0004300494E4600696E66004E414E006E6120
:10F7E0006E003000303132333435363738394142EB
:10F7F0004344454600303132333435363738396189
:10F8000062636465660000202020202020202020E4
:10F8100028282828282020202020202020202020C0
:10F8200020202020202020881010101010101010F0
:10F830001010101010101004040404040404040434
:10F8400004101010101010104141414141410101BC
:10F850000101010101010101010101010101010198
:10F8600001011010101010104242424242420202A6
:10F870000202020202020202020202020202020268
:10F880000202101010102000000000000000000014
:10F890000000000000000000000000000000000068
:10F8A0000000000000000000000000000000000058
:10F8B0000000000000000000000000000000000048
:10F8C0000000000000000000000000000000000038
:10F8D0000000000000000000000000000000000028
:10F8E0000000000000000000000000000000000018
:10F8F0000000000000000000000000000000000008
:10F9000000000000000000496E66696E69747900AD
:10F910004E614E00504F534958002E00FFFFFFFF2D
:10F92000000000000000F03F000000000000244044
:10F9300000000000000059400000000000408F401F
:10F94000000000000088C34000000000006AF8408A
:10F950000000000080842E4100000000D0126341AE
:10F960000000000084D797410000000065CDCD4124
:10F97000000000205FA00242000000E87648374205
:10F98000000000A2941A6D42000040E59C30A242A3
:10F990000000901EC4BCD64200003426F56B0C4318
:10F9A0000080E03779C3414300A0D88557347643BF
:10F9B00000C84E676DC1AB43003D9160E458E14320
:10F9C000408CB5781DAF154450EFE2D6E41A4B4495
:10F9D00092D54D06CFF08044F64AE1C7022DB544DA
:10F9E000B49DD9794378EA440080E03779C3414334
:10F9F000176E05B5B5B89346F5F93FE9034F384D95
:10FA0000321D30F94877825A3CBF737FDD4F157540
:10FA100005000000190000007D000000232D302BA0
:10FA20002000686C4C0065666745464700FFFFFF95
:10FA300000000000000000000000000000000000C6
:10FA400000000000000000000000000000000000B6
:10FA500000000000000000000000000000000000A6
:10FA60000000000000000000000000000000000096
:10FA70000000000000000000000000000000000086
:10FA80000000000000000000000000000000000076
:04FA90000000000072
:08FA940070C1FF7F01000000BA
:10FA9C000001000000000000010100000000000057
:10FAAC000201000000000000030100000000000043
:10FABC000400000000000000050000000000000031
:10FACC00060000000000000007000000000000001D
:10FADC000800000000000000090000000000000009
:10FAEC000A000000000000000B00000000000000F5
:10FAFC000C000000000000000D00000000000000E1
:10FB0C000E000000000000000F00000000000000CC
:10FB1C0010000000000000001100000000000000B8
:10FB2C0012000000000000001300000000000000A4
:10FB3C001400000000000000150000000000000090
:10FB4C00160000000000000017000000000000007C
:10FB5C001800000000000000190000000000000068
:10FB6C001A000000000000001B0000000000000054
:10FB7C001C000000000000001D0000000000000040
:10FB8C001E000000000000001F000000010100002A
:10FB9C00050000000E070100000008000000000036
:10FBAC000000000000000000000008000000000041
:10FBBC000000000000000000FFFFFF1FFFFFFF1F01
:10FBCC00FFFFFF1FFFFFFF1FFFFFFF1FFFFFFF1FB9
:10FBDC00FFFFFF1F0000FF1F0000100800000000C7
:10FBEC0000000000000000000000100800000000F1
:10FBFC0000000000000000000000080000000000F1
:10FC0C0000000000000000000000080000000000E0
:10FC1C0000000000000000000000100800000000C0
:10FC2C0000000000000000000000100800000000B0
:10FC3C0000000000000000000000100800000000A0
:10FC4C0000000000000000000D0300000202000094
:10FC5C000302000007020000010000000000000089
:10FC6C0030FA000050FA000070FA000000000000AA
:10FC7C00000000000000000000000000D0F70000B1
:10FC8C000000000000000000000000000000000068
:10FC9C000000000000000000000000000000000058
:10FCAC000000000000000000000000000000000048
:10FCBC000000000000000000000000008C03FE1F8C
:10FCCC0006F800001AF9000021FA000021FA0000E1
:10FCDC0021FA000021FA000021FA000021FA0000AC
:10FCEC0021FA000021FA000021FA0000FFFFFFFFBB
:10FCFC00FFFFFFFFFFFFFFFFFFFF0000B507000046
:10FD0C00910700000000000000000000000000004F
:10FD1C0000000000000000000000000000000000D7
:10FD2C0000000000000000000000000000000000C7
:10FD3C0000000000000000000000000000000000B7
:10FD4C0000000000000000000000000000000000A7
:10FD5C000000000000000000000000000000000097
:10FD6C000000000000000000000000000000000087
:04FD7C000000000083
:020000044012A8
:10005000FFFFFFFFFFFFFFFFFFFFFFFFFFFFFFFFB0
:040000030000956103
:00000001FF
